:020000040800F2
:10000000F0FF0120554F0408191F020801AE000837
:10001000C94F0408C94F0408C94F04080000000074
:10002000000000000000000000000000251F020882
:10003000211F0208000000001D1F020881A7000800
:10004000C94F0408C94F0408C94F0408C94F040820
:10005000C94F0408C94F040809AF000835B00008AB
:10006000F9AF0008BDAF000881AF000871100108AA
:100070006110010851100108411001082D100108FC
:100080001910010805100108C94F040800000000FC
:1000900000000000000000000000000045AF000864
:1000A000C94F04089599000879960008199B000823
:1000B000D59800081598000849970008C94F04080A
:1000C000C94F0408C94F0408C94F0408C94F0408A0
:1000D000C94F04085DA80008C1A70008000000007F
:1000E000CDAE0008C94F0408D96202080000000024
:1000F000000000000000000000000000F10F0108F7
:1001000000000000C94F0408C94F0408C94F040883
:1001100000000000000000000000000000000000DF
:10012000DD0F0108C90F0108B50F0108A10F010873
:100130008D0F01080000000000000000000000001A
:10014000000000000000000000000000992D0208DF
:10015000790F0108650F0108510F0108C94F040804
:10016000C94F0408C94F0408000000000000000047
:10017000000000000000000000000000000000007F
:1001800000000000C94F040800000000000000004B
:08019000C94F0408C94F04081F
:08019800EC4A04000100000024
:1001A00010020100982C0020942C00200000000078
:1001B000C80600081A023C00B42600209C2C00202F
:1001C000000000008D8B000827000400B0260020EE
:1001D000D82C002000000000CA06000803123300DB
:1001E000B0330020283B002000000000D0060008AB
:1001F00025009600DC390020723A00200000000043
:1002000000000000F6210C00A8370020583900201B
:10021000000000000407000815007000B43700203B
:10022000E838002000000000000000002A00600004
:1002300024380020883800200000000081D4020803
:100240002C001000083B0020183B0020000000009C
:10025000FD2F01082B0024007F3B00205B3B00208A
:1002600000000000CD2F010829107800B8360020CA
:1002700064390020000000000000000014000300AA
:10028000C43500208438002000000000100700085A
:10029000101002004C340020E83B00200000000059
:1002A00014070008281010003C340020EC3B00200C
:1002B000000000001513010823001000E4300020A6
:1002C000FC3B0020000000002D130108F82106006F
:1002D0002E3200200C3C0020000000001607000811
:1002E00016000800243C0020E43E0020000000002E
:1002F0001C07000805100600C0540020D459002037
:100300000000000024070008F53170002054002090
:10031000DC590020000000008D74020826000E0049
:100320005C5A00204C5A00200000000059120208BC
:100330000B20100020520020905A002000000000E6
:100340002A0700081F201C006C490020A05A00202A
:10035000000000003A07000805020400E8530020EE
:10036000BC5A0020000000005607000803010A00E4
:10037000D4510020C05A0020000000005A07000895
:100380001302030018480020CC5A0020000000008F
:10039000640700080C106C001E6D0020F87200202D
:1003A000000000004D7D03080E502001D46B00209A
:1003B0006473002000000000A9D4020813000400A8
:1003C000A07000208474002000000000680700086E
:1003D000010104004E6B0020887400200000000022
:1003E0000000000000010400466B00208C74002017
:1003F000000000006C07000802010300416B0020B0
:100400009074002000000000757D030809020100BF
:10041000AC720020947400200000000070070008F7
:1004200001020500566B00209874002000000000B7
:10043000496A02080002050050700020A0740020E4
:1004400000000000000000001B02080044700020B3
:10045000A874002000000000418600080120080068
:1004600084710020B07400200000000072070008B2
:100470001900050034720020B8740020000000004C
:100480007A07000837001E000C720020C07400209C
:1004900000000000800700081E000500246E0020F8
:1004A000E0740020000000009E0700081B00F4001C
:1004B000E05A0020E874002000000000217B0208C0
:1004C0000E0202001C710020DC75002000000000FC
:1004D000A40700082F001100D8720020E07500204A
:1004E00000000000A60700081A000E00D8790020BE
:1004F0001C7C002000000000B80700081802020061
:100500003C8700208C8700200000000000000000D5
:1005100017020B00318700209087002000000000A8
:100520004D86000802000C00408700209C870020B8
:1005300000000000000000000812090028870020C9
:10054000A88700200000000091860008F70106003F
:100550001E870020B487002000000000C6070008A6
:100560000A020A00E0810020BC8700200000000091
:10057000CC0700080300010020830020C88700206A
:10058000000000000000000004008000C0BC00204B
:1005900054BD002000000000000000000D002C00F1
:1005A00034BB0020D4BD002000000000C57D03083E
:1005B000F901040090B2002000BE002000000000FD
:1005C00025820008FD0124006CB2002004BE00203A
:1005D00000000000AD81000818202C003CB2002073
:1005E00028BE0020000000001D8C00080610180026
:1005F00088A5002054BE00200000000005D5020898
:10060000FB010100C0A400206CBE0020000000001F
:100610005D9F0008FC0109008CA3002070BE002033
:10062000000000006D9F00080A402000CC9C0020C4
:100630007CBE002000000000D60700083400100037
:10064000FC9B00209CBE002000000000D9D40208C2
:1006500011020800D49B0020ACBE00200000000066
:10066000F607000812120400CC9B0020B4BE002044
:1006700000000000FE07000812200D00BC9B0020B7
:10068000B8BE0020000000000208000802020300BB
:100690001C880020C8BE00200000000000000000F0
:1006A0000C020300D8870020CCBE00200000000010
:1006B000B1860008FE010900C0890020D0BE0020DC
:0806C00000000000C1860008E3
:1006C80000002003000000000000000000000000FF
:1006D8000000000000000000000000000000000012
:1006E8000000000000000000000000000000000002
:1006F80000000000000000000000010000000000F1
:1007080001000000020200000300000000050401CF
:10071800F4011900C4090000190128282000030168
:1007280000002B21231E64010100000001000A01C2
:10073800290000000000000100000005000001027F
:10074800030000000000000000000000000000009E
:100758000000040101006C16000000000000000009
:1007680048040430900100002900E8036400040AEA
:10077800000100002801000020003200C800D00756
:100788009600140032002800B0044006000550000E
:1007980014000F0008010000010000000000000024
:1007A8000000000000000000000000000000000041
:1007B8007E05EA05B4053200E803D00700002201EF
:1007C8000000000000004A01B400D601000000301B
:1007D80001000000000064002C010000000000007F
:1007E80000000000020000019E077D004632000064
:1007F800000001010101FFFFFFFF000000010000F0
:07080800054D4234310000F0
:10080F00010000008001000008000000040000004B
:10081F0000000000000000000102030406070809A1
:10082F00D6010100000101010001FFFFFFFFFFFFE3
:10083F0001010102FFFF000004030904120100027D
:10084F00EF0201408304563200020102030100004F
:10085F00120100020202004083044057000201020D
:10086F000301000009026400030100C03209040003
:10087F0000010300000009211101000122260007D9
:10088F0005830308000A080B010202020100090494
:10089F0001000102020100052400100105240100DE
:1008AF000204240202052406010207058203080040
:1008BF00FF09040200020A000000070501024000C0
:1008CF00000705810240000009024300020100C039
:1008DF003209040000010202010005240010010585
:1008EF0024010001042402020524060001070582E9
:1008FF00030800FF09040100020A000000070501B8
:10090F00024000000705810240000000FF000000C8
:10091F0000FFFF0000000000AA55050100000100C4
:10092F0005010905A101A1000501093009310932AD
:10093F00093309350934094009381581257F7508B0
:10094F0095088102C0C0000009022200010100E0E9
:10095F003209040000010301020009211101000105
:10096F002226000705830308000A0000000000008C
:10097F0001020304010203040607080961220208A9
:10098F0065210208A524020831070208750A02082A
:10099F00410702085D07020809070208F906020865
:1009AF0000000000000000002D202D2D202D2D2DEA
:1009BF002D202D2D2D2D0000000000000000000027
:1009CF0000000000000000AA550B010000AA550707
:1009DF00010000AA550902000000AA5503009F005C
:1009EF0001000000C0120000FF1FFF1F01000000E8
:1009FF006C5A002000000000E006002004000000F8
:100A0F00E4D0040810DD040800000000897D03080D
:100A1F00A08601000400000000000000000000009C
:100A2F0000000000000000000000000000000000B7
:100A3F0000000000E4D0040818DD040800000000E6
:100A4F0049800008E80300000400000000000000D7
:100A5F000000000000000000000000000000000087
:100A6F000000000000000000F4E304080CB40408C8
:100A7F000000000071A703087D00000006000000C1
:100A8F000000000000000000000000000000000057
:100A9F000000000000000000000000003CD004082F
:100AAF000000000000000000C1050108E80300007D
:100ABF000300000000000000000000000000000024
:100ACF000000000000000000000000000000000017
:100ADF0020DD0408000000000000000021D90208FA
:100AEF0010270000030000000000000000000000BD
:100AFF0000000000000000000000000000000000E7
:100B0F00000000002CDD040800000000152C010877
:100B1F00C1BE00085F760000050000000000000065
:100B2F0000000000000000000000000000000000B6
:100B3F000000000000000000A4D204080000000024
:100B4F0000000000A1EA00081027000001000000CB
:100B5F000000000000000000000000000000000086
:100B6F0000000000000000000000000030DD04085D
:100B7F0000000000000000004D800008E8030000A6
:100B8F000500000000000000000000000000000051
:100B9F000000000000000000000000000000000046
:100BAF003CDD04080000000000000000DD94030895
:100BBF00204E0000030000000000000000000000B5
:100BCF000000000000000000000000000000000016
:100BDF00000000004CDD04080000000000000000D1
:100BEF00B9920308204E000003000000000000002F
:100BFF0000000000000000000000000000000000E6
:100C0F0000000000000000005CDD04080000000090
:100C1F0000000000D5880008400D0300030000000D
:100C2F0000000000000000000000000000000000B5
:100C3F00000000000000000000000000A8D1040820
:100C4F000000000000000000A1E2030810270000D0
:100C5F000100000000000000000000000000000084
:100C6F000000000000000000000000000000000075
:100C7F0054D0040800000000000000002DAA020854
:100C8F00102700000300000000000000000000001B
:100C9F000000000000000000000000000000000045
:100CAF00000000006CDD04080000000000000000E0
:100CBF006DA40108A8610000010000000000000001
:100CCF000000000000000000000000000000000015
:100CDF000000000000000000ACD20408000000007B
:100CEF000000000059B70108A00F0000010000002C
:100CFF0000000000000000000000000000000000E5
:100D0F0000000000000000000000000078DD040873
:100D1F000000000000000000057702081027000007
:100D2F0001000000000000000000000000000000B3
:100D3F0000000000000000000000000000000000A4
:100D4F00B0D10408000000000000000011430208A9
:100D5F001A41000001000000000000000000000028
:100D6F000000000000000000000000000000000074
:100D7F00000000000CD30408000000000000000079
:100D8F000D0F0208102700000100000000000000F6
:100D9F000000000000000000000000000000000044
:100DAF00000000000000000084DD040800000000C7
:100DBF0000000000419602081A41000001000000E7
:100DCF000000000000000000000000000000000014
:100DDF0000000000000000000000000088DD040893
:100DEF000000000000000000893E0208400D0300D3
:100DFF0000000000000000000000000000000000E4
:100E0F0000000000000000000000000000000000D3
:100E1F0090DD0408000000000000000029A4010874
:100E2F00400D030000000000000000000000000063
:100E3F0000000000000000000000000000000000A3
:100E4F000000000098DD0408000000000000000012
:100E5F00F5B7020850C300000300000000000000B7
:100E6F000000000000000000000000000000000073
:100E7F000000000000000000A4DD040800000000D6
:100E8F00000000002D92030840420F0000000000F8
:100E9F000000000000000000000000000000000043
:100EAF00000000000000000000000000B0DD04089A
:100EBF00000000000000000009E5030850C3000017
:100ECF000000000000000000000000000000000013
:100EDF000000000000000000000000000000000003
:100EEF00000200051002700B00000100E00101017B
:100EFF00010000001D6E02080000000068080020BD
:100F0F004CEA040800000000000000000000000090
:100F1F0000000000C4DF0408000000000000000013
:100F2F00FE08002004000000F8E904080D0000008E
:100F3F00D1910208D02200200000000064E30408D1
:100F4F000D000000F9910208C422002000000000EB
:100F5F00CCE404080800000000000000B8220020C4
:100F6F0004000000D0E304080D000000D16E020859
:100F7F00AC2200200000000080E404080300000001
:100F8F00CD940208A0220020000000005CEA0408B3
:100F9F0003000000CD9402089422002000000000FE
:100FAF000CE0040801000000000000000000000039
:100FBF0000000000000000000E0000000000000014
:100FCF0000000000000000004CEA040800000000D0
:100FDF00000000000000000000000000C4DF040853
:100FEF000000000000000000FE08002004000000C8
:100FFF00A4E90408030000007D7502088822002080
:10100F0008000000D0E304080D000000D16E0208B4
:10101F00AC2200200000000080E404080300000060
:10102F00CD940208A0220020000000005CEA040812
:10103F0003000000CD94020894220020000000005D
:10104F000CE0040801000000000000000000000098
:10105F0000000000000000000E0000000000000073
:10106F00000000000000000064EA04080000000017
:10107F00000000000000000000000000C4DF0408B2
:10108F000000000000000000FE0800200400000027
:10109F00ACE9040803000000CD940208DC22002014
:1010AF00000000000CE00408010000000000000038
:1010BF000000000000000000000000000E00000013
:1010CF000000000000000000000000002070002061
:1010DF00702D7200FFFFFFFF010000000000803F36
:1010EF00080000000000000000000000441E002067
:1010FF00FA0000000100000001000000FFFF2D209A
:10110F002D2D202D2D2D2D202D2D2D0000000000FB
:10111F0000000000000000000000000000000000C0
:10112F000000803F0000803FFFFFFFFFE0DF04086B
:10113F00E8DF040804E004080000000000000000DD
:10114F000000000000000000E3DD040804000000C0
:10115F009B8F020800000000000000000CE0040854
:10116F00010000000000000000000000000000006F
:10117F00000000000E000000000000000000000052
:10118F0000000000D45400200100C409000000003A
:10119F00D25400200100C40900000000D0540020E8
:1011AF000100C40900000000CE5400200100C40952
:1011BF0000000000CA5400200100C4090000000014
:1011CF00CC5400200100C40900000000C8540020C6
:1011DF000100C40900000000C65400200100C4092A
:1011EF0000000000686B00200100C8000100000033
:1011FF00666B00203200307532000000646B0020F7
:10120F00055A0500616B002000FF0100636B002091
:10121F00010000002C0900205F6B0020020000007D
:10122F002C8B0408606B002000FF0100626B002014
:10123F00010000002C0900205E6B0020020000005E
:10124F002C8B0408546B002080C1803E05000000E9
:10125F00526B002080C1803E050000004C6B0020C7
:10126F0080C1803E050000004A6B002080C1803E97
:10127F0005000000446B002000FF0100406B0020C0
:10128F000A3201003F6B002004000000E88E0408C2
:10129F003E6B002002000000FC8E040800000000DE
:1012AF000000000034090020945300209CFF2C0103
:1012BF0000000000EE0600200A000000088F04085E
:1012CF00346B0020E0150C1700000000F006002022
:1012DF0008000000008B0408EF0600200500000046
:1012EF003C900408366B002002000000208F040899
:1012FF00A46D00200100FF7F01000000A36D0020FE
:10130F00020000002C8F0408C76B002003000000B0
:10131F003C8F0408C66B0020030000003C8F0408BC
:10132F00FE6C00200000F40101000000FC6C0020A6
:10133F000000F40101000000FA6C00200000F4012D
:10134F0001000000F86C00200000F4010100000013
:10135F00F66C00200000803E01000000F46C0020BD
:10136F000000803E010000001A6D0020E803D00746
:10137F000A000000186D0020006401000A00000040
:10138F000D6D0020006401000C6D00200064010051
:10139F00146D0020006401000A000000136D00208E
:1013AF00006401000A000000126D002000640100BB
:1013BF000A000000176D0020006401000A00000001
:1013CF00166D0020006401000A000000156D00205A
:1013DF00006401000A000000116D002000FF0100F1
:1013EF000A000000106D002000FF01000A0000003D
:1013FF000F6D002000FF01000A000000D06B0020DD
:10140F000000F40101000000CE6B00200000F40189
:10141F0001000000CC6B00200000F401010000006F
:10142F00CA6B00200000F40101000000C86B00200F
:10143F000000F401010000000A6D002000640100AB
:10144F00086D00201400E80301000000066D002065
:10145F00E80330750A000000046D002000C8010089
:10146F00036D002000C80100026D002000C80100BC
:10147F00016D0020006401000A000000986D00203B
:10148F000000D00701000000936D002000C801008C
:10149F00926D002000C80100916D002000C801006E
:1014AF00966D00200000D00701000000906D002015
:1014BF0000C801008F6D002000C801008E6D002054
:1014CF0000C80100946D00200000D007010000004B
:1014DF008D6D002000C801008C6D002000C8010038
:1014EF008B6D002000C8010034E0040800000000EC
:1014FF00000000000000000000000000F0B304082E
:10150F000900000000000000D809002004000000BE
:10151F00F8B304080900000000000000CC09002007
:10152F000400000084E70408090000000000000028
:10153F00C009002004000000B0DE0408090000000C
:10154F0000000000B40900200400000044E004087B
:10155F000900000000000000A8090020040000009E
:10156F004CE0040809000000000000009C09002066
:10157F000400000054E0040809000000000000000F
:10158F0090090020040000005CE00408090000003E
:10159F000000000084090020040000000CE0040893
:1015AF00010000000000000000000000000000002B
:1015BF00000000000E00000000000000000000000E
:1015CF000000000050E204080000000000000000CE
:1015DF00000000000000000098D004080700000081
:1015EF0000000000FC0900200000000060E2040879
:1015FF000800000000000000F009002000000000BB
:10160F006CE204080800000000000000E40900205C
:10161F00000000000CE004080100000000000000C2
:10162F000000000000000000000000000E0000009D
:10163F0000000000000000000000000074E2040839
:10164F00000000000000000000000000000000008B
:10165F0084E204080D00000000000000380A00209A
:10166F00000000008CE204080D00000000000000E4
:10167F002C0A00200000000094E20408070000007C
:10168F0000000000240A0020000000009CE2040873
:10169F000D00000000000000180A002000000000EC
:1016AF00A4E204080D000000000000000C0A002056
:1016BF0000000000ACE2040807000000000000007A
:1016CF00040A0020000000000CE0040801000000E4
:1016DF0000000000000000000000000000000000FB
:1016EF000E000000000000000000000000000000DD
:1016FF00B4E2040800000000000000000000000039
:10170F000000000098D004080C000000000000004A
:10171F006A6B002000000000C8E204080C00000003
:10172F00000000006C6B002000000000D8E20408ED
:10173F000C00000000000000A26B00200000000061
:10174F00E8E204080C00000000000000966B002087
:10175F0000000000FCE204080C0000000000000084
:10176F006E6B00200000000008E304080C0000006E
:10177F0000000000706B00200000000010E3040860
:10178F000C00000000000000726B00200000000041
:10179F0024E304080C00000000000000746B00201C
:1017AF00000000002CE304080C0000000000000003
:1017BF00766B00200000000034E304080C000000EA
:1017CF0000000000B46B0020000000004CE3040890
:1017DF000C00000000000000786B002000000000EB
:1017EF0058E304080C000000000000007A6B002092
:1017FF000000000000B404080C000000000000000E
:10180F007C6B00200000000060E304080C00000067
:10181F00000000007E6B0020000000006CE3040855
:10182F000C00000000000000806B00200000000092
:10183F0078E304080C00000000000000826B002019
:10184F000000000084E304080C000000000000000A
:10185F00846B00200000000090E304080C000000DF
:10186F0000000000866B0020000000009CE30408CD
:10187F000C000000000000009A6B00200000000028
:10188F00A4E304080C00000000000000986B002087
:10189F0000000000ACE304080C0000000000000092
:1018AF00A66B002000000000B8E304080C00000045
:1018BF0000000000A86B002000000000C4E3040833
:1018CF000C00000000000000AE6B002000000000C4
:1018DF006CDD04080C00000000000000886B002085
:1018EF0000000000D0E304080C000000000000001E
:1018FF00906B002000000000D8E304080C000000EB
:10190F00000000008A6B002000000000E4E30408E0
:10191F000C000000000000008C6B00200000000095
:10192F00F0E304080C000000000000008E6B0020A4
:10193F0000000000F8E304080C00000000000000A5
:10194F00926B002000000000B8D004080C000000CB
:10195F00000000009C6B00200000000004E404085D
:10196F000C00000000000000946B0020000000003D
:10197F004FDF04080C00000000000000A46B0020E3
:10198F000000000010E404080C000000000000003C
:10199F009E6B00200000000018E404080C000000FB
:1019AF0000000000A06B00200000000020E40408ED
:1019BF000C00000000000000AA6B002000000000D7
:1019CF0028E404080C00000000000000AC6B0020AD
:1019DF000000000030E404080C00000000000000CC
:1019EF00BE6B0020000000000CE0040801000000A6
:1019FF0000000000000000000000000000000000D8
:101A0F000E000000000000000000000000000000B9
:101A1F0038E404080000000000000000000000008F
:101A2F000000000044E404080D0000000000000066
:101A3F00900A0020000000004CE404080D00000094
:101A4F0000000000840A00200000000054E4040895
:101A5F0007000000000000007C0A002000000000CA
:101A6F0060E404080700000000000000740A002072
:101A7F00000000006CE404080900000000000000F2
:101A8F00680A00200000000078E404080900000044
:101A9F00000000005C0A00200000000084E404083D
:101AAF000900000000000000500A002000000000A4
:101ABF0094E404080900000000000000440A00201C
:101ACF00000000000CE0040801000000000000000E
:101ADF000000000000000000000000000E000000E9
:101AEF00000000000000000000000000A8E404084F
:101AFF0000000000000000000000000000000000D7
:101B0F00B8E404080500000000000000C56B0020C9
:101B1F00000000000CE004080100000000000000BD
:101B2F000000000000000000000000000E00000098
:101B3F00000000000000000000000000C0E40408E6
:101B4F000000000000000000000000000000000086
:101B5F00C4DF04080000000000000000A8010020FE
:101B6F0004000000ACDE04080D000000FD8F020829
:101B7F00E40A002000000000F8E904080D0000004E
:101B8F00D56D0208D80A00200000000064E30408A5
:101B9F000D000000B96D0208CC0A00200000000003
:101BAF00CCE404080800000000000000C00A002078
:101BBF0004000000D0E304080D000000016D0208CE
:101BCF00B40A002000000000D4E40408090000005B
:101BDF0000000000A80A00200400000080E40408B0
:101BEF0003000000CD9402089C0A002000000000B2
:101BFF000CE00408010000000000000000000000DD
:101C0F0000000000000000000E00000000000000B7
:101C1F000000000000000000DCE4040800000000E9
:101C2F00000000000000000000000000ECE40408C9
:101C3F000D00000000000000FC0A00200000000062
:101C4F00F4E404080A00000000000000D26D002038
:101C5F000000000000E504080A000000000000007A
:101C6F00DA6D00200000000008E504080A000000FB
:101C7F0000000000E26D00200000000010E50408E5
:101C8F000800000000000000F00A00200000000023
:101C9F000CE004080100000000000000000000003C
:101CAF0000000000000000000E0000000000000017
:101CBF00000000000000000018E50408000000000C
:101CCF000000000000000000000000002CE50408E8
:101CDF000D00000000000000140B002000000000A9
:101CEF003CE50408040000007592020800000000A3
:101CFF000000000044E504080D0000000000000093
:101D0F00080B00200000000058E504080400000044
:101D1F005192020800000000000000000CE00408CF
:101D2F0001000000000000000000000000000000A3
:101D3F00000000000E000000000000000000000086
:101D4F000000000060E50408000000000000000033
:101D5F00000000000000000074E504080800000007
:101D6F00000000005C0B00200000000080E504086C
:101D7F000800000000000000500B002000000000D1
:101D8F008CE504080800000000000000440B002050
:101D9F000000000098E504080800000000000000A3
:101DAF00380B002000000000A4E504080800000024
:101DBF00000000002C0B002000000000B0E504081C
:101DCF000800000000000000200B002000000000B1
:101DDF000CE00408010000000000000000000000FB
:101DEF0000000000000000000E00000000000000D6
:101DFF000000000000000000BCE504080000000027
:101E0F0000000000CF08002000000000C8E5040813
:101E1F000B00000000000000F00B0020000000008D
:101E2F00D4E504080B00000000000000E40B0020C4
:101E3F0000000000E0E504080B00000000000000B7
:101E4F00D80B002000000000ECE504080B00000098
:101E5F0000000000CC0B002000000000F8E5040893
:101E6F000B00000000000000C00B0020000000006D
:101E7F0004E604080B00000000000000B40B002073
:101E8F000000000010E604080B0000000000000036
:101E9F00A80B0020000000001CE604080B00000047
:101EAF00000000009C0B00200000000028E6040842
:101EBF000B00000000000000900B0020000000004D
:101ECF0034E604080700000000000000880B002023
:101EDF00000000003CE604080700000000000000BE
:101EEF00800B00200000000048E604080B000000F3
:101EFF0000000000740B00200000000054E60408EE
:101F0F000800000000000000680B00200000000027
:101F1F000CE00408010000000000000000000000B9
:101F2F0000000000000000000E0000000000000094
:101F3F00000000000000000060E604080000000040
:101F4F0000000000000000000000000074E604081C
:101F5F0008000000000000002C0C00200000000012
:101F6F0080E604080800000000000000200C00209C
:101F7F00000000008CE604080800000000000000CC
:101F8F00140C00200000000098E604080800000070
:101F9F0000000000080C002000000000A4E6040868
:101FAF000800000000000000FC0B002000000000F3
:101FBF000CE0040801000000000000000000000019
:101FCF0000000000000000000E00000000000000F4
:101FDF000000000000000000ACE604080000000054
:101FEF0000000000CC08002000000000BCE6040840
:101FFF000B00000000000000700C0020000000002B
:10200F00C8E604080700000000000000680C00206C
:10201F0000000000D4E604080700000000000000E4
:10202F00600C002000000000E0E60408070000003C
:10203F0000000000580C002000000000ECE604082F
:10204F0008000000000000004C0C00200000000001
:10205F00F4E604080800000000000000400C002017
:10206F0000000000FCE6040807000000000000006C
:10207F00380C0020000000000CE0040801000000F4
:10208F000000000000000000000000000000000041
:10209F000E00000000000000000000000000000023
:1020AF0008E704080000000000000000CC08002032
:1020BF000000000014E70408070000000000000003
:1020CF00E00C0020000000001CE7040807000000DF
:1020DF0000000000D80C00200000000024E70408D6
:1020EF000700000000000000D00C002000000000DE
:1020FF002CE704080800000000000000C40C0020BA
:10210F000000000034E70408070000000000000092
:10211F00BC0C0020000000003CE704080700000092
:10212F0000000000B40C00200000000044E7040889
:10213F000700000000000000AC0C002000000000B1
:10214F004CE704080800000000000000A00C00206D
:10215F000000000054E70408070000000000000022
:10216F00980C0020000000005CE704080700000046
:10217F0000000000900C00200000000064E704083D
:10218F000700000000000000880C00200000000085
:10219F006CE7040808000000000000007C0C002021
:1021AF00000000000CE00408010000000000000027
:1021BF000000000000000000000000000E00000002
:1021CF000000000000000000000000000000000000
:1021DF0045710208E80C0020C36B00202B000000A3
:1021EF004C8F0408C26B002000C80100C06B002098
:1021FF00E803D007010000004D414D424146343104
:10220F00310000005D6B0020000301005C6B0020BB
:10221F00000301008D70020865700208C40D0020D4
:10222F0021700208D56F02083C0E0020CD70020805
:10223F00B5700208F00E0020416F0208F56E02081B
:10224F00101200205B71020821920208EC1200208C
:10225F00416D0208000000003C130020BD7502080C
:10226F00DD730208181400208171020800000000BD
:10227F00B814002029720208F571020844150020D5
:10228F00B1720208FD720208F81500200B6D0020D4
:10229F0001060100C5710208957102083817002068
:1022AF005D72020899920208D81700202D73020858
:1022BF00E9920208A0180020006D00200103010020
:1022CF0074E7040800000000000000000000000098
:1022DF000000000080E70408080000000000000074
:1022EF00EC1900200000000088E704080700000038
:1022FF0000000000E41900200000000098E7040827
:10230F000D00000000000000D819002000000000A0
:10231F00A4E7040803000000CD940208CC190020A4
:10232F00000000000CE004080100000000000000A5
:10233F000000000000000000000000000E00000080
:10234F00000000000000000000000000ACE70408DF
:10235F00000000000000000000000000000000006E
:10236F00BCE704080A000000000000006CDB040852
:10237F0000000000C4E704080A000000000000008D
:10238F004CDB040800000000CCE704080A00000042
:10239F00000000009A6D002000000000D4E7040840
:1023AF000A00000000000000F819002000000000E3
:1023BF000CE0040801000000000000000000000015
:1023CF0000000000000000000E00000000000000F0
:1023DF000000000000000000DCE70408000000001F
:1023EF00000000000000000000000000E8E7040803
:1023FF0003000000CD9402082C1A002000000000FA
:10240F00F4E7040803000000CD940208201A00200E
:10241F0000000000FCE7040803000000CD94020850
:10242F00141A00200000000004E804080500000052
:10243F00000000005B6B0020000000000CE80408A7
:10244F0007000000000000000C1A00200000000030
:10245F0018E804080700000000000000041A00201C
:10246F00000000000CE00408010000000000000064
:10247F000000000000000000000000000E0000003F
:10248F0000000000000000000000000024E8040825
:10249F00000000000000000000000000000000002D
:1024AF0038E8040803000000CD9402085C1A0020ED
:1024BF000000000044E8040803000000CD94020867
:1024CF00F4060020000000004CE8040803000000A0
:1024DF00CD940208501A00200000000054E80408B0
:1024EF0003000000CD940208441A002000000000F1
:1024FF00D0E3040803000000CD940208381A00202E
:10250F00000000000CE004080100000000000000C3
:10251F000000000000000000000000000E0000009E
:10252F0000000000000000000000000060E8040848
:10253F00000000000000000000000000000000008C
:10254F0070E804080700000045930208B81A00203D
:10255F0000000000F4E3040803000000CD9402081B
:10256F00AC1A0020000000007CE804080300000003
:10257F00CD940208A01A00200000000084E804088F
:10258F0003000000CD940208941A00200000000000
:10259F008CE8040807000000299302088C1A002019
:1025AF00000000007CEC040803000000CD9402083A
:1025BF00801A00200000000098E8040803000000C3
:1025CF00CD940208741A002000000000A4E804084B
:1025DF0003000000CD940208681A002000000000DC
:1025EF000CE00408010000000000000000000000E3
:1025FF0000000000000000000E00000000000000BE
:10260F00000000000000000015710208E5700208CC
:10261F00C01A0020A9730208000000004C1B002004
:10262F00B16F02088D6F0208D81B00200000000058
:10263F00000000008C1C00208173020861930208C7
:10264F002C1D0020B0E8040800000000000000006E
:10265F000000000000000000BCE8040803000000B8
:10266F00CD940208381E002000000000C4E80408C2
:10267F0003000000CD9402082C1E00200000000073
:10268F00B0D1040803000000CD940208201E0020E2
:10269F0000000000D0E8040803000000CD940208F9
:1026AF00141E002000000000DCE8040803000000F6
:1026BF00CD940208081E002000000000E4E8040882
:1026CF00020000007D9302080000000000000000DF
:1026DF00ECE80408020000007D93020801000000EE
:1026EF0000000000F8E80408020000007D930208D3
:1026FF000200000000000000000000000E000000BB
:10270F000000000000000000000000003A6B0020F5
:10271F0088136F17010000003C6B002088136F17A0
:10272F000000000004E904080000000000000000A1
:10273F00000000000000000014E904080800000079
:10274F0000000000181F00200400000020E904080A
:10275F0008000000000000000C1F00200000000017
:10276F0080E4040804000000259002080000000027
:10277F00000000000CE00408010000000000000051
:10278F000000000000000000000000000E0000002C
:10279F00000000000000000000000000386B002067
:1027AF0088136F1701000000D453002088136F1790
:1027BF0000000000856E020800000000241F0020AA
:1027CF009E70002001000000FC8F0408D6530020EB
:1027DF000100000008900408CC5300200200000004
:1027EF0010900408BE490020000000000000000007
:1027FF00BC4900200000000000000000BA49002082
:10280F000000000000000000B84900200000000098
:10281F0000000000B649002000000000000000008A
:10282F00B44900200000000000000000E401002077
:10283F000000000000000000376B002002000000C5
:10284F001C9004085CE90408000000000000000070
:10285F00000000000000000014E904080800000058
:10286F0000000000A81F00200400000020E9040859
:10287F0008000000000000009C1F00200000000066
:10288F0080E4040804000000556E020800000000F8
:10289F00000000000CE00408010000000000000030
:1028AF000000000000000000000000000E0000000B
:1028BF000000000000000000000000006CE90408A8
:1028CF0000000000000000000000000000000000F9
:1028DF007CE904080D00000075910208D81F002044
:1028EF000400000088E904080D000000AD6E020826
:1028FF00CC1F00200400000094E904080D00000024
:10290F0039910208C01F002000000000A0E9040850
:10291F00030000009D750208B41F0020080000008E
:10292F00ACE9040803000000CD940208DC2200206B
:10293F00000000000CE0040801000000000000008F
:10294F000000000000000000000000000E0000006A
:10295F0000000000000000000000000004E0040878
:10296F000000000000000000000000000000000058
:10297F00E3DD0408040000003D90020800000000A1
:10298F00000000000CE0040801000000000000003F
:10299F000000000000000000000000000E0000001A
:1029AF0000000000000000000000000000EA040822
:1029BF000000000000000000000000000000000008
:1029CF00D0B704080D0000000000000038200020E0
:1029DF000400000010EA04080800000000000000D6
:1029EF002C200020040000001CEA0408080000004E
:1029FF0000000000202000200400000024EA04084A
:102A0F000800000000000000142000200400000057
:102A1F002CEA040808000000000000000820002035
:102A2F000400000034EA0408080000000000000061
:102A3F00FC1F0020040000003CEA0408080000000E
:102A4F0000000000F01F00200400000044EA04080A
:102A5F000800000000000000E41F00200400000038
:102A6F000CE004080100000000000000000000005E
:102A7F0000000000000000000E0000000000000039
:102A8F0000000000000000006D6E02080000000052
:102A9F00442000200000000000000000BC200020A7
:102AAF0000000000000000005C210020D253002035
:102ABF000400000028900408D0530020E0150C17E4
:102ACF0000000000CF53002008000000008B040816
:102ADF00CE530020050000003C90040800000000C9
:102AEF0000000000AC2100200000803F000000002B
:102AFF0000000000000000000000803F0000000008
:102B0F0000000000000000000000000000000000B6
:102B1F0000000000000000000000000000000000A6
:102B2F00010000000000803F0000000000000000D6
:102B3F00000000000000803F010000000000803F07
:102B4F00000000000000000000000000FF00000077
:102B5F00000000007C87002008000000000000003B
:102B6F006C87002008000000550C0208F9090208C4
:102B7F008124020800000000F50602085121020816
:102B8F00C10B0208C920020800000000000000006D
:102B9F00B1060208C50B0208B9090208C1230208D1
:102BAF0000000000C9060208CD200208950B02089C
:102BBF00292002080000000000000000BD060208E6
:102BCF003499040805080400000000003C90040834
:102BDF00008B04082890040800000000000000008B
:102BEF006099040805080A00000000003C900408E2
:102BFF00008B0408088F040800000000000000008C
:102C0F000800000015060208110602080D0602084A
:102C1F0001060208FD05020809060208050602085A
:102C2F00890602087D060208550602086906020891
:102C3F00410602082D0602081906020801000000CD
:102C4F000060024010600240000000000000000021
:102C5F00000B00000000000000000000000000005A
:102C6F0000600240286002400100000000000000E8
:102C7F00060C000000000000000000000000000033
:102C8F0000600240406002400200000000000000AF
:102C9F00100D000000000000000000000000000008
:102CAF000060024058600240030000000000000076
:102CBF00160E0000000000000000000000000000E1
:102CCF00006002407060024004000000000000003D
:102CDF00200F0000000000000000000000000000B6
:102CEF000060024088600240050000000000000004
:102CFF00261000000000000000000000000000008F
:102D0F0000600240A06002400600000000000000CA
:102D1F003011000000000000000000000000000063
:102D2F0000600240B8600240070000000000000091
:102D3F00362F00000000000000000000000000001F
:102D4F000064024010640240000000000000000018
:102D5F00003800000000000000000000000000002C
:102D6F0000640240286402400100000000000000DF
:102D7F000639000000000000000000000000000005
:102D8F0000640240406402400200000000000000A6
:102D9F00103A0000000000000000000000000000DA
:102DAF00006402405864024003000000000000006D
:102DBF00163B0000000000000000000000000000B3
:102DCF000064024070640240040000000000000034
:102DDF00203C000000000000000000000000000088
:102DEF0000640240886402400500000000000000FB
:102DFF00264400000000000000000000000000005A
:102E0F0000640240A06402400600000000000000C1
:102E1F00304500000000000000000000000000002E
:102E2F0000640240B8640240070000000000000088
:102E3F003646000000000000000000000000000007
:102E4F0001000000482600200000000000000000E4
:102E5F000000000000000000000000000000000063
:102E6F000000000000000000000000000000000053
:102E7F000000000000000000000000000000000043
:102E8F000000000000000000000000000000000033
:102E9F000000000000000000000000000000000023
:082EAF0000000000000000001B
:1080000090ED057A90ED004AD0ED066AD0ED014A78
:10801000D0ED047A90ED035AD0ED025AA4EE007A26
:10802000B0EE406AB0EE470AB0EE667AA4EE867A09
:1080300067EEC07AA5EE407AE5EE867A80ED057AA5
:10804000C0ED067A704700BF704700BF70B50C4C9A
:1080500023689BB15A68821A002A0FDB0546002666
:1080600003E05A68AA1A002A08DB99681E731A6886
:108070002160184690472368002BF2D170BD00BFE5
:10808000A8260020436A8269D154436A0169C26B01
:1080900001338B4228BF00234362DAB1EFF311832F
:1080A000502282F31288C26B1168C9070ED470B4D3
:1080B0005468FCB9D0E909518D4211D1012280F8F0
:1080C0006020DBB283F3118870BC7047DBB283F3AE
:1080D00011887047C26DD36843F08003D360704746
:1080E00086690E44D6600ED9691A516085620021F6
:1080F00080F86010116841F00101DBB2116083F378
:10810000118870BC70470569691A51608462EEE796
:10811000034610B4846BD968406954B11A6D8C1A47
:10812000013A005D5DF8044B08BF0A46C0B21A650B
:1081300070471A6A805C01328A4228BF2246C0B268
:108140001A625DF8044B7047C36B13B190F860007E
:108150007047D0E90903181AB0FA80F04009704757
:10816000D0E909120369914238BFC9188A1AC16B54
:10817000013B19B149680A449A4201D2981A7047E2
:1081800000207047836B43B1026D5B689A4291BFD8
:10819000981AC0689B1AC0187047D0E907239A4202
:1081A0002FBFD01AC0688018C01A70470A4B30B56C
:1081B00003F1100493F900205D78072AC8BF143A30
:1081C000811804330D7313F8025C855413F8012CE5
:1081D0000A769C42EED130BDF868040803682DE9A8
:1081E000F0415D6A1DB12B46BDE8F0411847002AF9
:1081F000174611DD04460E460F4400E023689B68D5
:10820000204698470028F9D0236816F8011B1B6800
:1082100020469847BE42F1D1BDE8F08103681B6952
:10822000184700BF00233D213E2201704270837039
:10823000C370704703685A1C02601970704700BF12
:108240002DE9F047089C2578002B804689460CBF15
:108250004FF0200A4FF0300A661C25B3002A26DDB5
:10826000334601E0024698B113F8011B501E002965
:10827000F8D1971E60B13D46013D51464046C84782
:108280006B1C002BF8DC257827EAE770013045B13C
:10829000041B29464046C847301916F8015B002DDB
:1082A000F7D1BDE8F087002A03DC2846F9E7002073
:1082B000EEE7571EDFE700BF0A44914215D030B405
:1082C0000139551E41F2210211F8014F082380EABD
:1082D000042004044CBF82EA40004000013B80B20D
:1082E000F7D18D42F0D130BC704770472DE9F0478F
:1082F00014461D4606464FF47A720023204629464E
:108300003CF05CFC4D4BDFF850814D4A4D4F03442F
:1083100088FB03101844D91782FB032CC1EB6010B3
:1083200088FB002887FB03279C44474AC1EBEC2CC1
:10833000C0EB001E82FB0C29A3EB8E0E1F44434AA8
:1083400086F806E0C1EB27474FEAEC7E08EB000A0F
:10835000CEEBA90E82FB07824FEAE0780EEB4E0EC1
:10836000C8EB6A18ACEBCE0CC8EB0818DFF8ECE0F1
:1083700086F804C0A0EB880070718EFB0303F81729
:10838000C0EBE21240F2B55000FB1272C1EBE353B6
:10839000B2F5896F4FEA83073FDA40F2DA239A4257
:1083A00043DCB2F5B77FB4BF4FF0000E4FF0010EC3
:1083B0004FEA4E08264B08EB0E0103EBC1031FFAF0
:1083C0008EFCD88C234908EB0E0301EBC301163158
:1083D0000B2301E031F8020D90421BDD013BF9D186
:1083E0001B4BC64403EBCE0E0123BEF81000B37046
:1083F00007F5FA670132121ABC44F270A6F800C001
:10840000204629464FF47A7200233CF0D7FB328194
:10841000BDE8F0870133DBB2E9E74FF0030CE64635
:1084200040F296504FF00608CCE74FF0020CE646BB
:1084300040F229404FF00408C4E700BF80BC92C757
:10844000C5B3A29107452EC2ABAAAA2A73B06D1676
:10845000F86804080869040889888888792D031158
:1084600030B403888278174DC478A3F5FA6303F01B
:10847000030101EB4101013A02EB810205EB4202EB
:10848000611E158A027940F2B5549B0804FB031360
:108490002B4403EB430302EBC303427984790A497B
:1084A0000089C3EB031302EB83032144C3EB0313E3
:1084B00001EB83034FF47A720021C2FB030130BC4D
:1084C000704700BFF868040880436D380028F0B496
:1084D00003DA2D230B7040420131092804464FF086
:1084E000010307DD03EB83035B00B0FBF3F2092A12
:1084F000F8D883B10F48A0FB0326B4FBF3F2092A96
:1085000002F1570C02F1300709DD03FB1244F308B6
:1085100001F801CBEFD100230B70F0BC704703FBD7
:108520001244F30801F8017BE5D100230B70F0BC85
:10853000704700BFCDCCCCCC884270B44FF0010462
:1085400042D301FB04F4B0FBF4F58D42F9D2ECB157
:1085500042BB092D04FB150005F1570605F1300259
:108560000EDDB4FBF1F403F8016B7CB1B0FBF4F564
:10857000092D04FB150005F1570605F13002F0DC6A
:10858000B4FBF1F403F8012B002CEFD100221A7098
:1085900070BC704703F8016BB4FBF1F4002CF5D00C
:1085A000B0FBF4F5092D04FB150005F1370605F1C4
:1085B0003002EFDCB4FBF1F403F8012B002CEFD117
:1085C00000221A7070BC70470546002AEAD1C0E745
:1085D000D0ED057A90ED013AD0ED003AD0ED064AA3
:1085E00090ED024A90ED077A90ED035A90ED086AFB
:1085F000D0ED045AC0ED067AF0EE406A27EE830A09
:10860000C0ED056AA3EEA60A80ED087AA4EE240A5E
:10861000A5EE470AA5EEC60A80ED070A704700BF1F
:10862000D0ED007A90ED017A30EE670AE7EE007A3D
:10863000B0EE670AC0ED007A704700BF704700BF18
:1086400006224FF47A73027043607047F0B400253D
:108650000E4E00F1FF3C2F46142165B103788B428A
:108660000BD003460CEB050403E013F8012F8A42FC
:1086700003D0A342F9D1C155013701350B2D02D0EA
:1086800016F8011FE9E7F0BC704700BF68690408ED
:1086900030B41523162517242D212E2203702F23E5
:1086A00045708470C1700271437130BC704700BF67
:1086B00001212C220223017042708370704700BF99
:1086C000012310B411211024212244704171C27081
:1086D00003720370037183705DF8044B704700BF31
:1086E0004FF4006383827047012380F85430704751
:1086F000F0B4037C456902681F2B37D9203B202149
:10870000546899400C4223D010249C40D160D4601E
:108710005168D940CE074ED4EFF31183502282F333
:108720001288EA6B1168C90709D45468002C52D129
:10873000D5E909618E4243D1012285F86020DBB280
:1087400083F31188037C02681F2B194614D9203B40
:10875000082150689940084200D0D1600421506837
:1087600001FA03F3184223D1F0BC704720241668A5
:108770009C4026420FD11946082310688B401842AE
:1087800000D093600423106803FA01F10842EBD093
:108790009160F0BC7047102199409460916011681D
:1087A000D940CC07B8D5012101FA03F39360B3E7B0
:1087B000D360F0BC7047012101FA03F3D360ABE74B
:1087C000AF690F44D7600ED82E69711A5160AC6240
:1087D000002185F86010116841F00101DBB21160E1
:1087E00083F31188AEE7711A5160AE62F0E700BF03
:1087F00070B4037C01681F2B26D9A3F12005202229
:108800004C68AA40224214BF01220022D2B1426920
:108810001B481C4C02EB420200EB421225785468C4
:108820002068CDB9E56856892C6824F001042C60D5
:1088300082891F2B22EA060282811AD8202202FA9C
:1088400003F38B6070BC704720220C689A40224270
:1088500014BF01220022D9E7A469226822F0010294
:108860002260828922F480721204120C1F2B8281F2
:10887000E4D9A3F1200220239340CB6070BC704761
:10888000B4A50020B0A5002010B5027C01681F2A05
:108890004FF020030ED94C68203A93401C4208D078
:1088A0000B4A406800241470026822F00102026042
:1088B000CB6010BD0C6893401C42FAD0044A40685B
:1088C00000241470026822F0010202608B60F0E75D
:1088D000705E00202DE9F0478C4A8D4B12781C7891
:1088E000D207064648D58B4D012C00F091801ED34F
:1088F000022C40F09B808849884A09881288884F5A
:10890000914201D901241C70EB7AFBB12B89EBB1A8
:10891000844B1B78D3B130F0A5FB002800F0E28037
:108920002B7B83422CBF012300233B700FE0DFF839
:10893000E8C17B4F7C4CBCF800002288697B521A4E
:108940008242DFDAEB7A0024002BDFD13B782A79F0
:10895000632A07D87549022C087800F0B8800028EF
:1089600040F0A0807249AA7A9C4238BF1C460C7025
:10897000002A44D1BDE8F087DFF89CC1654DBCF802
:108980000000BCF8021095F803E06A4F411A002974
:10899000A4F10302B8BF4942704597F80080D2B2F3
:1089A00011D32F7887420ED3012A45D9B8F1020F8F
:1089B0009AD15C48604A007890800229CCBF00219F
:1089C0000121D18090E7B0EB4E0FEDDC012A40F29F
:1089D0008C800229EADC0324514F524852494F4A05
:1089E0001C70B8F1020F4FF000033C7003700B8055
:1089F000138089D1504A01219380D18084E7012CD2
:108A00006BD0022CB6D10720BDE8F04731F022BB75
:108A1000424A41491288687B0988121A914207DD4F
:108A2000414A12888A423CBF00241C703C4F6BE7CD
:108A300002241C703A4F67E70229B7DC95F800E082
:108A400090FBFEFE0EF1010EBEF1080FDFF8D4A080
:108A5000AA786978DFF8C490334C314FA8BF4FF043
:108A6000080E8AF800E01FFA8EFA11FB0AF112FBD9
:108A70000AF2DFF8B8A0A9F8001092B200214FF076
:108A80006409B8F1020F228039701970CAF8041015
:108A90008AF801907FF452AF274A0121A2F804E03E
:108AA000D18048E74868301A244EB042C8BF4A70A7
:108AB0003FF758AFC2F16402214E00FB02F086FB83
:108AC0000062C017A0EBA250643048704AE700284B
:108AD000E8D101274E600F70ECE70820BDE8F047B1
:108AE00031F0B8BA02233B7031E7032C7FF471AF49
:108AF000B8F1020F9AD10B4A0F4B12789A800229D3
:108B0000CCBF00210121D980054FFDE6DE510020B8
:108B100024810020205200200452002028810020BF
:108B2000848100200A520020268100202C81002010
:108B3000F85400200D880020108800207F969800AF
:108B40006BCA5F6B70B544880546C4F30B042246BC
:108B500008460E4600213DF061FE2B69094A93420A
:108B600002D3094A934205D35BB121463046BDE8A2
:108B700070401847224630461946BDE870403CF028
:108B800059BA70BDC80600080F08000838B51D4B5B
:108B90001B78044600F1250593B104221A492030C0
:108BA0003DF07AFE2846142218493DF075FE012357
:108BB00084F83A30164B1B7873B984F83B3038BDD3
:108BC0002846142213493DF067FE012384F83A3009
:108BD0000F4B1B78002BF0D00F4B186859689A6820
:108BE000DD68E56020606160A260DD69186959692F
:108BF0009A69A2610123E5612061616184F83B30DB
:108C000038BD00BF95330020963300209B330020F1
:108C10007433002078A104087533002038B52C2265
:108C200000213DF0FBFD0346642140F2DC5240F29E
:108C3000022019745A821321202240F21A4540F270
:108C40006C74188399760E2002211A7701229D8276
:108C5000DC8240F2753540F6430483F82200197235
:108C600083F82A109A7383F82920DD831C8419461F
:108C70000248BDE838400FF053B800BF84A1040893
:108C8000022810B504460BD8084B0949094A00EBE5
:108C9000400003EB401318460B60147027F038FEB9
:108CA000601CC0B2BDE8104035F0DCBBD46B0020C6
:108CB000E4560020BC9B002038B53A4B3A481A785D
:108CC0005B783A493A4C3B4D02EB420203EBC3035B
:108CD00001EB430300EB42122B6022602AF0F2FD0D
:108CE0000021302234483DF099FD206827F010FE25
:108CF000324B03F1780102E006338B4250D01A78F0
:108D0000002AF9D19C78D878844202D35879002877
:108D1000F2D02B492B4B08792B492C4C0A70C822D6
:108D2000642111FB002100222948DA61C3E9011204
:108D3000C3E90322C3E9052283F8202083F8212018
:108D400060600EF08FFA23899FED225A224AA17AA1
:108D50009FED226A507906EE903AF8EEE66A1388A3
:108D6000C5EE265A07EE103A1D4B1960538812794A
:108D70001C4907EE903AB8EEC77AF8EEE77A1A4B3C
:108D8000C1ED005A27EE067A67EE867A18725A729B
:108D900083ED017AC3ED007ABDE8384021F054B983
:108DA0000122B6E7BC9B0020D46B00201E6D002082
:108DB000E4560020E8560020B87B0020B83600209A
:108DC00084710020E051002038230020A8260020D4
:108DD000EA300020C0C9FB48243C002017B7D13836
:108DE0004C7600205076002024760020074B1B781C
:108DF00053B9074B00F1200250F8041B43F8041B41
:108E00009042F9D101207047002070477433002050
:108E10007533002010B5154C94F84630002B144BD8
:108E200014BF012200221A700BD0042204F12C017D
:108E300010483DF031FD142204F131010E483DF09F
:108E40002BFD94F84730002B0C4B14BF012200225D
:108E50001A7009D00A4B0B4A03F1200153F8040B96
:108E600042F8040B8B42F9D110BD00BFA8260020A8
:108E700095330020963300209B330020743300206C
:108E8000B4260020753300200B4B1B7810B58BB92E
:108E90000A4B0B4A03F1200153F8040B42F8040B70
:108EA0008B42F9D1074B012483F84740FFF7B2FF0B
:108EB000204610BD0020FCE77433002075330020ED
:108EC000B4260020A826002038B50C4B1B789BB98F
:108ED0000B4D0C49042205F12C003DF0DDFC012472
:108EE0001422094905F131003DF0D6FC85F84640D1
:108EF000FFF790FF204638BD0020FCE795330020A7
:108F0000A8260020963300209B330020F0B50C29C2
:108F100034D8DFE801F08A3333335F33333334330B
:108F200033330700048C9689B2F802C01788744D59
:108F300024F480542404240C0484038C8488818BBE
:108F400023F4005321F4E6411B0409041B0C46EAF8
:108F50000C06090C43EA063341EA0721A8429BB2FA
:108F6000A4B289B200F09E8005F58065A84200F0A9
:108F7000998092688480818302640384F0BD048CAC
:108F80009589B2F802E017885D4E24F480742404B9
:108F9000240C0484038CB0F804C0818B23F4007388
:108FA0001B0421F0730145EA0E041B0C090443EA7B
:108FB0000423090CB0429BB21FFA8CF541EA070169
:108FC0005BD0504CA04258D0926885808183C263A8
:108FD0000384F0BD048C9589B2F802E0B2F800C0B9
:108FE000474E24F010042404240C0484038C878846
:108FF000018B23F0200321F4E6411B0409041B0C20
:1090000045EA0E04090C43EA041341EA0C21B0427C
:109010009BB2BFB289B25BD03A4CA04258D09268A2
:109020008780018382630384F0BD048C9589B2F844
:1090300002C01788324E24F001042404240C048456
:10904000018C8488038B21F0020123F0730309044F
:109050001B04090C45EA0C051B0CB04241EA050152
:10906000A4B243EA070324D0264DA84221D0926837
:109070008480038342630184F0BDD489168A578AB1
:1090800023F4006343EA04234FF6FF341C40938823
:1090900025F440553E4344EA032345EA06149BB2B7
:1090A000A5B291E7158A24F4804444EA8514A4B259
:1090B0005FE7D689158A578A21F0080131439688DF
:1090C00024F4407421F004013D4331432C43CEE7A6
:1090D000D489168AB2F812C023F0800343EA04133D
:1090E0004FF6BF741C40938827F4406546EA0C068F
:1090F00044EA031345EA86049BB2A7B28FE700BF98
:1091000000000140000401402DE9F84FF022DFF893
:1091100034B28248824E834FDFF82C82DFF82C92E3
:10912000DFF82CA200213DF079FB7F48DFF824C254
:10913000DFF824E20BF590755C462368B34200F03B
:10914000D080B3F1804F00F0CE80BB4200F0CD80E4
:10915000634500F0D880734500F0D780434500F0A8
:10916000D6804B4500F0D580534500F0D4806F4A3F
:10917000934200F0988002F58062934208BF092371
:1091800000F092802434A542D7D1694E694D4FF04A
:1091900003094FF002089BF80630002B7CD09BF8A7
:1091A00004301F09013F032F03F00F0374D836F872
:1091B000170040FA03F2D2076ED54FF0010A0AFAFF
:1091C00003F3013B18403BF049FD5B4BDB5D18446A
:1091D00015EBC00760D055F8303058489BF80810A0
:1091E00003F13F4202F57E02920A825C02F01F0008
:1091F0005209032A0AFA00FA7FD0042A77D0022AF9
:1092000004D14948426C4AEA02024264B7F804C0F9
:10921000BCFA8CF2C2F11F0292B2D00803EB8000BC
:1092200002F00702076A92004FF00F0E0EFA02FEDC
:1092300027EA0E070762076A01FA02F23A4302625E
:109240004FF0010E00220EFA02F737EA0C0120D18E
:109250005000D3F800A009FA00F1C9430AEA010A54
:10926000C3F800A0D3F800A008FA00F040EA0A0012
:10927000186098680840986098689860586820EA74
:1092800007075F6058685860D8680140D960D9689E
:10929000D9600132102AD6D10BF1240B5C457FF442
:1092A0007AAFBDE8F88F0823254A02EBC3030122F9
:1092B0001B7903F01F015B09032B02FA01F208D0AE
:1092C000042B0AD0022B7FF45DAF436C1A43426437
:1092D00058E7036C1A43026454E7036B1A430263B2
:1092E00050E70023E0E70123DEE70223DCE70E4836
:1092F000026B4AEA0202026388E70B48026C4AEA00
:109300000202026482E70323CEE70423CCE70523AD
:10931000CAE70623C8E70723C6E700BF3492002048
:1093200000000140000400400038024000440140B9
:10933000F49A040824880020FC9A04088C990408F4
:10934000009B0408D4990408001000400014004059
:109350000040014000080040000C004000B9704788
:1093600003682DE9F04F03F13F4404F57E04534EAA
:10937000A40A0125345D04F01F066409032C05FAD4
:1093800006F500F09580042C00F08D80022C45D06D
:109390008588B5FA85F0C0F11F0080B2C40803EBE0
:1093A000840400F00700266A80000F27874026EA21
:1093B00007062662276A01F003068240701E3A43C0
:1093C00001282262C1F3810EC1F300184FF00002A0
:1093D0004FEA51114FF0010C25D94FF0030E0CFA52
:1093E00002F0A84315D150001F680EFA00F4E443C0
:1093F00027401F60D3F8008006FA00F747EA080705
:109400001F60DF683C40DC60DC6801FA00F020434C
:10941000D8600132102AE2D1BDE8F08F284C666C8A
:1094200035436564B4E74FF003090CFA02F737EAF5
:10943000050033D15000D3F800A009FA00F4E4434A
:109440000AEA040AC3F800A0D3F800B006FA00FA4A
:109450004AEA0B0AC3F800A0D3F808A004EA0A0AF3
:10946000C3F808A0D3F808B00EFA00FA4AEA0B0ACB
:10947000C3F808A0D3F804A02AEA07075F60D3F86E
:1094800004A008FA02F747EA0A075F60DF683C4079
:10949000DC60DC6801FA00F02043D8600132102A59
:1094A000C3D1BDE8F08F064C266B354325636FE7CB
:1094B000034C266C354325646AE700BF8C99040889
:1094C0000038024003682DE9F04F03F13F4404F5F2
:1094D0007E04534EA40A0125345D04F01F0664097E
:1094E000032C05FA06F500F09580042C00F08D8021
:1094F000022C46D08588B5FA85F0C0F11F0080B2F5
:10950000C40803EB840400F00700266A80000F27DC
:10951000874026EA07062662276A01F0030602FA58
:1095200000F0721E3843012AC1F3810EC1F3001806
:1095300020624FEA51114FF000024FF0010C25D983
:109540004FF0030E0CFA02F0A84315D150001F682B
:109550000EFA00F4E44327401F60D3F8008006FAB7
:1095600000F747EA08071F60DF683C40DC60DC6802
:1095700001FA00F02043D8600132102AE2D1BDE8A0
:10958000F08F284C666C35436564B3E74FF00309F0
:109590000CFA02F737EA050033D15000D3F800A0E7
:1095A00009FA00F4E4430AEA040AC3F800A0D3F875
:1095B00000B006FA00FA4AEA0B0AC3F800A0D3F892
:1095C00008A004EA0A0AC3F808A0D3F808B00EFA03
:1095D00000FA4AEA0B0AC3F808A0D3F804A02AEA62
:1095E00007075F60D3F804A008FA02F747EA0A0702
:1095F0005F60DF683C40DC60DC6801FA00F020431B
:10960000D8600132102AC3D1B9E7064C266B354326
:1096100025636FE7034C266C354325646AE700BF7A
:109620008C9904080038024010B50409013C032C51
:1096300017D80E4B33F8142000F00F0042FA00F355
:1096400013F001030FD0012303FA00F0013810409A
:109650003BF004FB064A074B125D104403EBC000CD
:1096600010BD002010BD184610BD00BFF49A0408BC
:10967000FC9A0408248800202DE9F843304D2B8AF9
:10968000B5F80C8018EA030827D02E4E4FF000479B
:10969000B8FA88F327FA03F2D24391B21B3B08EAE7
:1096A00002082982042B15D8DFE803F0372D23198F
:1096B0000300D6F8EC30002B39D1EB6A1FFA83F99E
:1096C000D6F8E84034B12368204649469847646894
:1096D000002CF8D1B8F1000FDAD1BDE8F883D6F844
:1096E000C800696B036889B29847B8F1000FCFD101
:1096F000F3E7D6F8CC00A96B036889B29847B8F1B4
:10970000000FC5D1E9E7D6F8D000E96B036889B24C
:109710009847B8F1000FBBD1DFE7D6F8D400296C29
:10972000036889B29847B8F1000FB1D1D5E703F1CA
:10973000FF3900231FFA89F9C6F8EC30C0E700BFF3
:1097400000480140349200202DE9F8432F4D2B8A28
:10975000B5F80C8018EA030827D02D4E4FF00047CB
:10976000B8FA88F327FA03F2D24391B21B3B08EA16
:1097700002082982042B15D8DFE803F0352B2219C3
:109780000300D6F89C30002B37D1EB6A1FFA83F91F
:10979000D6F8984034B12368204649469847646813
:1097A000002CF8D1B8F1000FDAD1BDE8F883B06F22
:1097B000696B036889B29847B8F1000FD0D1F4E71C
:1097C000F06FA96B036889B29847B8F1000FC7D151
:1097D000EBE7D6F88000E96B036889B29847B8F1E7
:1097E000000FBDD1E1E7D6F88400296C036889B287
:1097F0009847B8F1000FB3D1D7E703F1FF39002341
:109800001FFA89F9C6F89C30C2E700BF0008004083
:10981000349200202DE9F8432C4D2B8AB5F80C80AA
:1098200018EA030825D02A4E4FF00047B8FA88F30B
:1098300027FA03F2D24391B21B3B08EA02082982BD
:10984000042B13D8DFE803F0322920170300736FCD
:10985000002B34D1EB6A1FFA83F9346F34B12368DB
:109860002046494698476468002CF8D1B8F1000FAB
:10987000DCD1BDE8F883306D696B036889B2984725
:10988000B8F1000FD2D1F4E7706DA96B036889B20B
:109890009847B8F1000FC9D1EBE7B06DE96B0368E9
:1098A00089B29847B8F1000FC0D1E2E7F06D296C9A
:1098B000036889B29847B8F1000FB7D1D9E703F12F
:1098C000FF3900231FFA89F97367C6E700040040D7
:1098D000349200202DE9F8434FF080452B8AB5F8EB
:1098E0000C8018EA030825D0294E4FF00047B8FA3B
:1098F00088F327FA03F2D24391B21B3B08EA02082D
:109900002982042B13D8DFE803F032292017030043
:10991000F36C002B34D1EB6A1FFA83F9B46C34B1C9
:1099200023682046494698476468002CF8D1B8F16E
:10993000000FDCD1BDE8F883B06A696B036889B2B7
:109940009847B8F1000FD2D1F4E7F06AA96B036829
:1099500089B29847B8F1000FC9D1EBE7306BE96BDA
:10996000036889B29847B8F1000FC0D1E2E7706B85
:10997000296C036889B29847B8F1000FB7D1D9E7CD
:1099800003F1FF3900231FFA89F9F364C6E700BF2A
:10999000349200202DE9F8435C4D2B8AB5F80C80F9
:1099A00018EA030826D05A4E4FF00047B8FA88F359
:1099B00027FA03F2D24391B21B3B08EA020829823C
:1099C000042B14D8DFE803F04C433A310300736AE8
:1099D000002B40F09480EB6A1FFA83F9346A34B1AB
:1099E00023682046494698476468002CF8D1B8F1AE
:1099F000000FDBD1474D2B8AB5F80C8018EA03081D
:109A00004BD0434E4FF00047B8FA88F327FA03F2E1
:109A1000D24391B21B3B08EA02082982042B39D8B1
:109A2000DFE803F05B51473D27003068696B03684E
:109A300089B29847B8F1000FB8D1DBE77068A96B1D
:109A4000036889B29847B8F1000FAFD1D2E7B06888
:109A5000E96B036889B29847B8F1000FA6D1C9E74E
:109A6000F068296C036889B29847B8F1000F9DD15E
:109A7000C0E7D6F8C430002B39D1EB6A1FFA83F95E
:109A8000D6F8C04034B123682046494698476468F8
:109A9000002CF8D1B8F1000FB6D1BDE8F883D6F8A4
:109AA000A000696B036889B29847B8F1000FABD189
:109AB000F3E7D6F8A400A96B036889B29847B8F118
:109AC000000FA1D1E9E7D6F8A800E96B036889B2D5
:109AD0009847B8F1000F97D1DFE7D6F8AC00296CB2
:109AE000036889B29847B8F1000F8DD1D5E703F12B
:109AF000FF3900231FFA89F9C6F8C430C0E703F123
:109B0000FF3900231FFA89F9736267E700000140FB
:109B100034920020004401402DE9F8432C4D2B8A5B
:109B2000B5F80C8018EA030825D02A4E4FF00047FC
:109B3000B8FA88F327FA03F2D24391B21B3B08EA42
:109B400002082982042B13D8DFE803F032292017FA
:109B50000300736A002B34D1EB6A1FFA83F9346A6D
:109B600034B123682046494698476468002CF8D1F0
:109B7000B8F1000FDCD1BDE8F8833068696B036889
:109B800089B29847B8F1000FD2D1F4E77068A96B99
:109B9000036889B29847B8F1000FC9D1EBE7B06804
:109BA000E96B036889B29847B8F1000FC0D1E2E7CA
:109BB000F068296C036889B29847B8F1000FB7D1F3
:109BC000D9E703F1FF3900231FFA89F97362C6E769
:109BD0000000014034920020F0B50668464CB30AFC
:109BE000A34200F0858009D9444CA34264D00134DB
:109BF000A3427AD0123CA34261D0F0BDB3F5801FDE
:109C000070D0013CA342F8D1702702254379B6F801
:109C10000CE0022023FA00F4A0401FFA80FCA80008
:109C20002346441903EB4403354C00294FD04CEA3A
:109C30000E0C03F1040E44F8231044F82E20A6F86D
:109C40000CC0E319EFF31181502282F312884219FC
:109C500004EBC202D2F810C0BCF1000F03D044F8EC
:109C600007C013690433421904EBC202576917B1E4
:109C70001F6053690433421904EBC202976917B19C
:109C80001F6093690433421904EBC202D76917B10C
:109C90001F60D36904330027CAB21F6082F31188A2
:109CA000284404EBC004236A63B9B38923F0010399
:109CB0001B041B0CB381F0BDC0270425A6E7202799
:109CC0000025A3E7B38943F00103B381F0BD2EEA79
:109CD0000C0C03F1040EA6F80CC044F8231044F851
:109CE0002E20AEE74827012590E7E82705258DE7D8
:109CF000982703258AE700BF0200100051001000DA
:109D00003492002030B50368584C594D18882468A7
:109D1000B4FBF2F20139013AAB4294B283B089B29A
:109D200082B211D0534883420ED0B3F1804F0BD092
:109D3000A0F58030834207D000F58060834203D0D5
:109D400000F58060834202D122F0700292B24A484C
:109D5000834269D000F58060834241D022F4407292
:109D600000F56C4092B283421A80D9621C8564D19E
:109D70000122002119869A821A883D4842F0010288
:109D800083421A8036D0B3F1804F60D03B4A934271
:109D90005FD002F5806293425DD002F5806293420B
:109DA0005BD002F58062934259D002F58062934203
:109DB00057D002F59632934255D002F58062934215
:109DC00017D002F58062934208BF092112D002A881
:109DD0004FF0012340F8043D35F0C8FA03B030BD20
:109DE00001201A80D9621C8598821A8802431A8041
:109DF000C9E70821224B03EBC10100224C798DF801
:109E00000440012301A88DF805308DF807308DF846
:109E1000062035F0ABFA1B2CE0D11A4B019301A8B8
:109E200035F0A4FA03B030BD01201A80D9621C8538
:109E300098821A8802431A80A8E70E4A934297D064
:109E400001229A821A8842F001021A809BE70121BE
:109E5000D0E70221CEE70321CCE70421CAE70521A0
:109E6000C8E70621C6E70721C4E700BF84A5002094
:109E700000000140000401400010004000040040C8
:109E8000009B0408190100011F4B98422CD0B0F12F
:109E9000804F2BD0A3F57C43984229D003F58063F3
:109EA000984227D003F58063984225D003F580635C
:109EB000984223D003F58063984221D003F596336E
:109EC00098421FD003F58063984207D003F5806362
:109ED000984208BF092202D00020704708220B4B8D
:109EE00003EBC203187970470022F8E70122F6E776
:109EF0000222F4E70322F2E70422F0E70522EEE76C
:109F00000622ECE70722EAE700000140009B040874
:109F1000002330B40F4A1D46012404E00133082B0E
:109F20000DD012F8244C30EA040402F12402F5D1D9
:109F3000A94207D001330135082BEDB2F1D1002041
:109F400030BC7047044A03EBC30302EB830330BC0D
:109F500018797047FE990408D499040810B50021B7
:109F600004460120FFF7D4FF207010BD38B500244F
:109F70000472451EE1B20220FFF7CAFF0134082C2B
:109F800005F8010FF6D138BD68B10A4A292100232E
:109F900001E012F8241C884202F1240204D00133AB
:109FA000082BF6D100207047034803EBC30300EBF6
:109FB00083007047FC990408D49904082DE9F04FF8
:109FC00085B0CDE902109B4DDFF878A2029B013BE2
:109FD0000293013300F02A8135F0A0FD964C974F93
:109FE000DFF864E2964E4FF4FA7301934FF01008D5
:109FF000DEF80430C3F30803002B40F0F680EFF3E3
:10A000001183002B40F0F1802068AA6823689842F1
:10A01000FAD133689A42F7D8D7F800C04FF47A7172
:10A0200001FB0CF39B1AB3FBFCF301FB00304FF474
:10A030007A7C4FF00109DEF80430C3F30803002BEB
:10A0400040F0B580EFF31183002B40F0B08023681F
:10A05000A96822689342FAD132689142F7D83A68E7
:10A060000CFB02FBABEB0101B1FBF2F10CFB0313A8
:10A070001B1AB3F57A7FDED3019B013B0193B7D165
:10A08000039B6F4E581CC0B235F09CFBDFF8B8E163
:10A090004FF47A730193DEF80430C3F308034FF0F2
:10A0A0001008002B44D1EFF31183002B40D120681E
:10A0B000AA6823689842FAD133689A42F7D8D7F849
:10A0C00000C04FF47A7101FB0CF39B1AB3FBFCF355
:10A0D00001FB00304FF47A7C4FF00109DEF80430C8
:10A0E000C3F30803002B44D1EFF31183002B40D1BD
:10A0F0002368A96822689342FAD132689142F7D85E
:10A100003A680CFB02FBABEB0101B1FBF2F10CFB7B
:10A1100003131B1AB3F57A7FE0D3019B013B019334
:10A120003FF454AFDEF80430C3F30803002BBAD079
:10A13000EFF3118388F31288D5F808C02A68D20398
:10A1400004D50122CAF80020D5F808C02068DAF842
:10A150000090DBB283F3118839684FF47A72484477
:10A1600002FB01F3A3EB0C03B3FBF1F302FB0030A2
:10A17000B0E7EFF3118188F31288D5F808B02B68A7
:10A18000DB0344BFCAF80090D5F808B02368DAF8BA
:10A190000020C9B281F31188396813440CFB01F225
:10A1A000A2EB0B02B2FBF1F20CFB0323B1E7EFF3DE
:10A1B000118188F31288D5F808B02B68DB0344BFFF
:10A1C000CAF80090D5F808B02368DAF80020C9B2C0
:10A1D00081F31188396813440CFB01F2A2EB0B02E6
:10A1E000B2FBF1F20CFB032342E7EFF3118388F398
:10A1F0001288D5F808C02A68D20304D50122CAF80B
:10A200000020D5F808C02068DAF80090DBB283F3AC
:10A21000118839684FF47A72484402FB01F3A3EBCA
:10A220000C03B3FBF1F302FB003000E705B0BDE81F
:10A23000F08F00BF10E000E0108A0020148A002098
:10A24000188A00200C8A002000ED00E0224B5B6899
:10A25000C3F3080330B4D3B9EFF31183BBB91F4A7A
:10A260001F4D20481368846811688B42FAD1296811
:10A270008C42F7D81C4A11684FF47A7202FB01F045
:10A28000001B30BCB0FBF1F002FB03007047EFF3A2
:10A290001182102383F3128803F1E023D2B29C6869
:10A2A000196811F4803F11491EBF012008609C68A5
:10A2B0000A4B18680B6882F311880B4A11684FF437
:10A2C0007A72034402FB01F0001B30BCB0FBF1F0DA
:10A2D00002FB0300704700BF00ED00E0108A002081
:10A2E000188A002010E000E0148A00200C8A002068
:10A2F0002DE9F84F8046274C274DDFF8A490274ED4
:10A30000FFF7A4FFDFF89CE0DFF89CC04FF0100AD5
:10A310004FF47A77DCF80430C3F30803CBB9EFF3DA
:10A320001183B3B92368A96822689342FAD13268CD
:10A330009142F7D8DEF8002007FB02FBABEB0101EE
:10A34000B1FBF2F107FB03131B1A4345E2D3BDE84F
:10A35000F88FEFF311818AF31288D5F808B02B68D3
:10A36000DB0304D50123C9F80030D5F808B0236811
:10A37000D9F80020C9B281F31188DEF80010134427
:10A3800007FB01F2A2EB0B02B2FBF1F207FB032386
:10A39000DAE700BF108A002010E000E0188A0020F1
:10A3A0000C8A0020148A002000ED00E070B59D4C5E
:10A3B0002368002B40F005819B4B1A78002A68D057
:10A3C0009A4B19789A4B002964D11868B3F82C512C
:10A3D00041628489012A44EA05048481A3F82C118E
:10A3E00057D0D3F83001B3F85C5241628489022A15
:10A3F00044EA05048481A3F85C124AD0D3F86002D1
:10A40000B3F88C5341628489032A44EA05048481A9
:10A41000A3F88C133DD0D3F89003B3F8BC54416239
:10A420008489042A44EA05048481A3F8BC1430D04A
:10A43000D3F8C004B3F8EC5541628489052A44EA94
:10A4400005048481A3F8EC1523D0D3F8F005B3F804
:10A450001C5741628489062A44EA05048481A3F8D2
:10A460001C1716D0D3F82007B3F84C5841628489E2
:10A47000072A44EA05048481A3F84C1809D0D3F8CC
:10A480005028B3F87C495162908920439081A3F809
:10A490007C1970BD5C68198961602568186845F091
:10A4A000010540F20D312560A0F848108489012A89
:10A4B00044F480748481ECD0D3F83441B3F838513B
:10A4C000D3F830016560256845F001052560A0F8E6
:10A4D00048108489022A44F480748481D9D0D3F846
:10A4E0006442B3F86852D3F860026560256845F0AD
:10A4F00001052560A0F848108489032A44F480747B
:10A500008481C6D0D3F89443B3F89853D3F890031A
:10A510006560256845F001052560A0F8481084892C
:10A52000042A44F480748481B3D0D3F8C444B3F8CB
:10A53000C854D3F8C0046560256845F0010525605E
:10A54000A0F848108489052A44F480748481A0D03E
:10A55000D3F8F445B3F8F855D3F8F00565602568ED
:10A5600045F001052560A0F848108489062A44F4C6
:10A57000807484818DD0D3F82447B3F82857D3F85A
:10A5800020076560256845F001052560A0F84810A2
:10A590008489072A44F4807484813FF47AAFD3F825
:10A5A0005428B3F85808D3F850385060106840F079
:10A5B00001001060A3F848109A8942F480729A81D1
:10A5C00070BD0546FFF742FE217AA9B16DB1194A67
:10A5D000002316890133002E18BF0021AB4202F17F
:10A5E0006002F6D100293FF4E7AE00F51C501030B0
:10A5F000002320602372DFE62368C31A002BFFF6D6
:10A6000048AF637A3BB1013BDBB263722BB100F51B
:10A610007A702060D0E62360CEE66368034423604E
:10A62000CAE600BF387C0020B4A80020B0A50020F6
:10A63000B8A80020B4A500202DE9F04FDFF834C100
:10A64000494CDFF834E1DFF83481484E824648480F
:10A650001AF1FF3AC0F08680DCF80430C3F3080337
:10A66000002B5ED1EFF31183002B5AD10568A2684D
:10A6700003689D42FAD133689A42F7D8DEF8007039
:10A680004FF47A7101FB07F39B1AB3FBF7F301FB5D
:10A690000535DCF80430C3F308034FF010094FF41C
:10A6A0007A77F3B9EFF31183DBB90368A168026825
:10A6B0009342FAD132689142F7D8DEF8002007FBC6
:10A6C00002FBABEB0101B1FBF2F107FB03135B1BD8
:10A6D000B3F57A7FBCD2DCF80430C3F30803002B57
:10A6E000E0D0EFF3118189F31288D4F808B0236821
:10A6F000DB0304D50123C8F80030D4F808B00368A0
:10A70000D8F80020C9B281F31188DEF80010134494
:10A7100007FB01F2A2EB0B02B2FBF1F207FB0323F2
:10A72000D5E7EFF31183102282F31288A168226823
:10A73000D20303D50122C8F80020A168D0F8009008
:10A74000D8F80050DBB283F31188DEF800704FF4C4
:10A750007A724D4402FB07F35B1AB3FBF7F302FB7B
:10A76000053596E7BDE8F08F10E000E0188A00207C
:10A77000108A002000ED00E0148A00200C8A0020DE
:10A7800030B4EFF31183102282F31288084809498C
:10A790000268094D094C013202608A682A60002271
:10A7A0002260DBB20A6883F3118830BC704700BFB7
:10A7B000108A002010E000E0188A00200C8A002097
:10A7C00038B5254B5C68A26BE36D62B1E26BC2B138
:10A7D000998A1A88C90792B204D5120744BF4FF666
:10A7E000F7721A8038BD99891A88890692B2EDD518
:10A7F0009206EBD5E26AFAB19888216B9047E36D37
:10A80000E4E799891A880D0692B2E1D51006DFD5E2
:10A81000D4E909128A420AD0A1692569885C988026
:10A820000132B2FBF5F105FB1122A262D0E7DA6832
:10A8300022F08002DA60CBE79B88E2696169DBB2D3
:10A840008B54E269E068E36D0132B2FBF0F100FB8A
:10A850001122E261BAE700BF0487002038B5254B1A
:10A860001C68A26BE36D62B1E26BC2B1998A1A886F
:10A87000C90792B204D5120744BF4FF6F7721A8087
:10A8800038BD99891A88890692B2EDD59206EBD522
:10A89000E26AFAB19888216B9047E36DE4E7998901
:10A8A0001A880D0692B2E1D51006DFD5D4E9091257
:10A8B0008A420AD0A1692569885C98800132B2FB7E
:10A8C000F5F105FB1122A262D0E7DA6822F08002DE
:10A8D000DA60CBE79B88E2696169DBB28B54E2699D
:10A8E000E068E36D0132B2FBF0F100FB1122E2619E
:10A8F000BAE700BF04870020002A12DD70B50446C5
:10A900000D468E18236820469B6898470028F9D08A
:10A91000236815F8011B1B6820469847B542F1D102
:10A9200070BD70470368DB6A03B11847704700BF0A
:10A9300003689B6A03B11847704700BF03682DE99D
:10A94000F0415D6A1DB12B46BDE8F0411847002A71
:10A95000174611DD04460E460F4400E023689B684D
:10A96000204698470028F9D0236816F8011B1B6879
:10A9700020469847BE42F1D1BDE8F08103689B694B
:10A98000184700BF03685B69184700BF0368DB68AE
:10A99000184700BF03689B68184700BF03685B68DF
:10A9A000184700BF03681B68184700BF014B986C2D
:10A9B000F8E700BFA826002038B50C46097849B151
:10A9C000054601342B6828461B68984714F8011B7C
:10A9D0000029F7D138BD00BF064B53F820302BB10A
:10A9E0001A689B8851690B4201D1138370475383C6
:10A9F000704700BFDC890020036803F13F4202F585
:10AA00007E022DE9F04F920A464DAA5C02F01F0526
:10AA100052090124032A04FA05F47ED0042A77D0CF
:10AA2000022A30D001F00306721E012AC1F3810E02
:10AA3000C1F300188588C1F341114FF000024FF0B7
:10AA4000010C25D94FF0030E0CFA02F0A84315D1E2
:10AA500050001F680EFA00F4E44327401F60D3F84B
:10AA6000008006FA00F747EA08071F60DF683C40ED
:10AA7000DC60DC6801FA00F02043D8600132102A63
:10AA8000E2D1BDE8F08F284A556C2C435464C9E7E5
:10AA90004FF003090CFA02F737EA050033D15000F2
:10AAA000D3F800A009FA00F4E4430AEA040AC3F860
:10AAB00000A0D3F800B006FA00FA4AEA0B0AC3F87D
:10AAC00000A0D3F808A004EA0A0AC3F808A0D3F843
:10AAD00008B00EFA00FA4AEA0B0AC3F808A0D3F845
:10AAE00004A02AEA07075F60D3F804A008FA02F777
:10AAF00047EA0A075F60DF683C40DC60DC6801FA17
:10AB000000F02043D8600132102AC3D1BDE8F08F95
:10AB1000054A156B2C43146384E7034A156C2C43D8
:10AB200014647FE78C990408003802402DE9F04F47
:10AB30004A484B494B4B4C4C4FF0010A4FF002092D
:10AB40004FF004084FF0080E4FF0100C202740265D
:10AB5000802530F8022B12F0010F03D01960A3F802
:10AB600004A0083312F0020F03D01960A3F8049078
:10AB7000083312F0040F03D01960A3F804800833DF
:10AB800012F0080F03D01960A3F804E0083312F0A4
:10AB9000100F03D01960A3F804C0083312F0200F7F
:10ABA00002D019609F80083312F0400F02D0196064
:10ABB0009E80083312F0800F02D019609D80083308
:10ABC00012F4807F05D04FF4807B1960A3F804B0A5
:10ABD000083312F4007F05D04FF4007B1960A3F80E
:10ABE00004B0083312F4806F05D04FF4806B196005
:10ABF000A3F804B0083312F4006F05D04FF4006BD3
:10AC00001960A3F804B0083312F4805F05D04FF444
:10AC1000805B1960A3F804B0083312F4005F05D01C
:10AC20004FF4005B1960A3F804B0083312F4804FAE
:10AC300005D04FF4804B1960A3F804B00833D20B51
:10AC400004D04FF4004219609A80083301F5806106
:10AC5000A1427FF47EAFBDE8F08F00BFF49A0408F4
:10AC600000000240248800200010024000B9704714
:10AC7000036803F13F4202F57E022DE9F04F920A8C
:10AC8000464DAA5C02F01F0552090124032A04FA6A
:10AC900005F47ED0042A77D0022A30D001F00306D2
:10ACA000721E012AC1F3810EC1F300188588C1F319
:10ACB00041114FF000024FF0010C25D94FF0030E67
:10ACC0000CFA02F0A84315D150001F680EFA00F4E8
:10ACD000E44327401F60D3F8008006FA00F747EAF4
:10ACE00008071F60DF683C40DC60DC6801FA00F0A8
:10ACF0002043D8600132102AE2D1BDE8F08F284A03
:10AD0000556C2C435464C9E74FF003090CFA02F761
:10AD100037EA050033D15000D3F800A009FA00F457
:10AD2000E4430AEA040AC3F800A0D3F800B006FA24
:10AD300000FA4AEA0B0AC3F800A0D3F808A004EA14
:10AD40000A0AC3F808A0D3F808B00EFA00FA4AEAD3
:10AD50000B0AC3F808A0D3F804A02AEA07075F602B
:10AD6000D3F804A008FA02F747EA0A075F60DF6831
:10AD70003C40DC60DC6801FA00F02043D86001321E
:10AD8000102AC3D1BDE8F08F054A156B2C4314631C
:10AD900084E7034A156C2C4314647FE78C990408FC
:10ADA0000038024010B1036882885A83704700BFA0
:10ADB00010B1036882881A83704700BF18B1036816
:10ADC000828809B95A8370471A83704710B40A4BB6
:10ADD0000A4A1C7801238340234052F8200029B9F5
:10ADE000B3FA83F149095DF8044BE7E7191C18BF72
:10ADF00001215DF8044BE1E7D8890020DC890020BF
:10AE000008B501210220FFF7E1FF0C4B1B7803F08E
:10AE10000503052B0ED000210120FFF7D7FF0021ED
:10AE20000846FFF7D3FF3220FFF706FC0220FFF7AA
:10AE3000D3FDF8E728F034FAEDE700BF00870020E3
:10AE40000E4B1B8801463BB90D4B0E4A1B78106810
:10AE50000BB981F00101B1E70B4B5A691AB11A68BD
:10AE600010B910605874704708480949008891FB70
:10AE7000F0F1012011605874704700BFE88900208C
:10AE8000EA890020EC890020F0890020088A00204F
:10AE900020A1070038B5074B03EBC0052C796A7970
:10AEA0004C40A24205D053F830002146FFF786FF00
:10AEB0006C7138BDDC9B002030B1036882881B694F
:10AEC0001A4214BF01200020704700BF2DE9F04155
:10AED0000B4E356873691D4010D0DFF828800127BC
:10AEE000B5FA85F4C4F11F0408EB840307FA04F4EF
:10AEF000D86C03689847A5437461F1D1BDE8F0812F
:10AF0000003C0140A82600202DE9F0410B4E356899
:10AF100073691D4010D0DFF828800127B5FA85F449
:10AF2000C4F11F0408EB840307FA04F4D86C036827
:10AF30009847A5437461F1D1BDE8F081003C014020
:10AF4000A82600202DE9F0410B4E356873691D409D
:10AF500010D0DFF828800127B5FA85F4C4F11F046A
:10AF600008EB840307FA04F4D86C03689847A543F8
:10AF70007461F1D1BDE8F081003C0140A8260020B9
:10AF80002DE9F0410B4E356873691D4010D0DFF894
:10AF900028800127B5FA85F4C4F11F0408EB840367
:10AFA00007FA04F4D86C03689847A5437461F1D19B
:10AFB000BDE8F081003C0140A82600202DE9F041C9
:10AFC0000B4E356873691D4010D0DFF828800127CB
:10AFD000B5FA85F4C4F11F0408EB840307FA04F4FE
:10AFE000D86C03689847A5437461F1D1BDE8F0813E
:10AFF000003C0140A82600202DE9F0410B4E3568A9
:10B0000073691D4010D0DFF828800127B5FA85F458
:10B01000C4F11F0408EB840307FA04F4D86C036836
:10B020009847A5437461F1D1BDE8F081003C01402F
:10B03000A82600202DE9F0410B4E356873691D40AC
:10B0400010D0DFF828800127B5FA85F4C4F11F0479
:10B0500008EB840307FA04F4D86C03689847A54307
:10B060007461F1D1BDE8F081003C0140A8260020C8
:10B07000094A10B5536C094C43F48043536404F1FE
:10B080004C00402200213BF0C9FB4FF0FF33C4F8D5
:10B090008C30C4F88F3010BD00380240A826002044
:10B0A00010B58B680160044698470022FF230121F8
:10B0B000A2736373217310BD03681B6A184700BF36
:10B0C00070B44E1C0568C2728672AC69A44670BC2E
:10B0D000604700BF2DE9F041044618460D4616466C
:10B0E0001F4639F07FF82844A0722068E67229468E
:10B0F00045693B4632462046AC46BDE8F0416047D4
:10B10000036810B504461B689847236820469B686F
:10B110009847A37B0133A37310BD00BF10B503682C
:10B1200004469B689847FF2301226373227310BD76
:10B130000B4B984211D0A3F57843984202D04FF0C0
:10B14000FF3070470122074B03EB02135A8901328B
:10B1500092B25A81588980B270470022F3E700BF4B
:10B1600000300140DC8700202DE9F0410546806871
:10B170001746984610B1036882885A8341F08001CF
:10B18000686840F2E93401E0002C43D00689013CB4
:10B1900016F0020FA4B2F7D089B2818140F2E931F2
:10B1A00001E0002936D00389013913F0010F89B27B
:10B1B000F7D08389838900264FF47A714FF6FF72A6
:10B1C0004FF0FF0C03E0013989B291421FD003898F
:10B1D0009C07F8D5A0F80CC04FF47A7102E0A1B238
:10B1E000914214D00389DB0701F1FF34F7D583893D
:10B1F0009BB20FB13B70013701364645E7D1AB68D2
:10B2000013B11A689B8813830120BDE8F081FFF712
:10B210008FFFF4E7FFF78CFF6868CBE7F0B587692D
:10B2200083B0064617B13B68BA885A837069DFF865
:10B23000A8E08389C3244FF47A734FF0060C6D465F
:10B240004FF6FF710EF1010E03E0013B9BB28B4202
:10B2500020D002899207F8D5A3B283814FF47A7384
:10B2600002E0A3B28B4215D00289D20703F1FF346A
:10B27000F7D5828992B20DB12A700135BCF1000F69
:10B280000BD00CF1FF3CFF24BEF1000FE1D09EF883
:10B290000040D7E7FFF74CFFB76917B13B68BA88A2
:10B2A0001A839DF805009DF801509DF802109DF845
:10B2B00003409DF804209DF8063041EA052143EA49
:10B2C000002342EA04220120A6F85010A6F85220DA
:10B2D000A6F8543003B0F0BD74690408037A022B59
:10B2E00001D000207047F0B5036983B013B11A682C
:10B2F0009B885383014640F2E933C06801E0002B8C
:10B300005DD00289013B12F0020F9BB2F7D0BB2344
:10B31000838140F2E93301E0002B50D00289013BE8
:10B3200012F0010F9BB2F7D08389838903899C07B0
:10B330004FF005076E464FF47A724FF0FF0C4FF650
:10B34000FF7506D4531E9BB2D2B11A4603899C07DF
:10B35000F8D5A0F80CC04FF47A7302E0A3B2AB4268
:10B360000ED00289D20703F1FF34F7D5828992B259
:10B370000EB1327001367A1E27B117461A46E5E73C
:10B38000FFF7D6FE0B6913B11A689B8813839DF8EB
:10B3900000609DF801009DF802509DF803209DF883
:10B3A00004409DF8053040EA062042EA052243EABF
:10B3B0000423C88201200A834B8303B0F0BDFFF74A
:10B3C000B7FEC868B1E700BF427A4AB110B504467B
:10B3D00004F10A01D0E9003098470023637210BDE0
:10B3E000704700BF437A5A1C0344D2B2427299722A
:10B3F000037A93420AD84AB110B5044604F10A010F
:10B40000D0E9003098470023637210BD704700BF39
:10B4100028B1302801D0312802D129B3002070474B
:10B420003228FAD03328F8D03428F6D03528F4D092
:10B430002028F2D02128F0D01028EED01128ECD00E
:10B440001228EAD01328E8D01428E6D01528E4D032
:10B45000162803D1B1FA81F0400970471728DDD1D1
:10B46000B1FA81F04009704701207047302829D097
:10B47000312829D0322829D0332829D0342829D07E
:10B48000352829D020282BD021282BD0102825D0B2
:10B49000112829D0122829D0132829D0142829D0DE
:10B4A000152829D0162805D0172808BF0F2302D049
:10B4B000002070470E23114A03EB4303134493F813
:10B4C000860070470023F6E70123F4E70223F2E742
:10B4D0000323F0E70423EEE70523ECE70823EAE77C
:10B4E0000623E8E70723E6E70923E4E70A23E2E780
:10B4F0000B23E0E70C23DEE70D23DCE7F868040804
:10B5000070B502221349144C144E4FF6FF70FCF72D
:10B51000D3FE22884AB1A518B54218D2052A16D9F9
:10B520002146FCF7C9FE2C46F3E721460222FCF730
:10B53000C3FE0222A118FCF7BFFE094BE41A094B17
:10B540001C8041F60F53C31A5842584170BD002069
:10B55000FCE700BF0040000802400008008000082F
:10B56000FA3F000840320020024A136823EA000034
:10B5700010607047A07000204F4B1B68B3F5FA7F36
:10B5800010B57FD84D4B9A89D989914224BF0022AA
:10B590009A81598A1A8A914224BF00221A82484904
:10B5A000DA7891F85C1072B1012A70D0454C012212
:10B5B00000200A2922709A70987179D00C2974D1D0
:10B5C0009FED417A06E00A2998792AD00C2963D1A7
:10B5D0009FED3E7ADFED3E7A002818BFB0EE677A25
:10B5E0003C4CA278062A97BF3B49DFED396A01EB54
:10B5F0008201D1ED2D6A2179C9B1013A032A0AD815
:10B60000B7EE000A80EE260A39F0F4FD238898424E
:10B6100028BF18462080314A9378013B012B03D97B
:10B6200010BD9FED2F7AD5E70023937010BD9B7856
:10B63000244907EE903A0A78F8EEE77A67EE877ABF
:10B6400007EE102AB8EEC77A27EE277AF4EEC76A1B
:10B65000F1EE10FADFDD86EEA77AFDEEC77A17EE7F
:10B66000903A102BA8BF1023012BB8BF0123DBB2E7
:10B670009A4238BF1A460A70184A9378013B012B48
:10B68000CED8D1E74FF00050FFF76EFF7AE70A29D6
:10B690009879C6D00C299BD0012A9FED127A99D9AE
:10B6A0000A298DD19FED107A94E79FED077A97E7ED
:10B6B0009FED0D7A94E700BFEC9C0020CC9C00200D
:10B6C000FC9C00202E3200206F12833A0AD7A33947
:10B6D0006F12033888A50020F8680408C0540020C1
:10B6E0005304E9386F1203390F506E3AF8B5B64972
:10B6F0000B78A3F11702022A0FD9B44A12F83300CB
:10B70000002840F03081D800024452782AB1B04A73
:10B7100012F83330002B00F0E8810024AD4EAE4F1C
:10B720002546315B4B0803F077334FEA910C0CF060
:10B73000333CCB1ACA08A3EB0C0302F011329B1A5C
:10B7400003EB231303F00F33A7FB03C2D209C2EBB1
:10B7500002229A1A11F001031CBF0135EDB2012A31
:10B7600006EB040004F108040BDD022A40F0EE8031
:10B7700013B111F42F7F04D11AF07AFA002800F0E7
:10B78000E580282CCDD1013D022D00F2DF80022082
:10B790002EF0B2FB002800F0E280904A5378052B8F
:10B7A00000F2D0808E4903EBC30301EB4301137811
:10B7B0008C488D4C0160022B00F2C08003EB4301EA
:10B7C00004EB411103EB430304EB4313874D9A88C9
:10B7D000D88829609042864924BF00229A808B78BD
:10B7E000042B00F0C98033B90B88B3F5F07F84BF18
:10B7F0004FF4F0730B807F4EFFF7BEFE35687E4B33
:10B800002B40002B00F07981EA0700F1C3806B0424
:10B8100000F1C7802F0700F1CB80A80400F1CF8092
:10B820002904764E40F182800023F37386F823309A
:10B8300028F03AF800285CD0737E032B59D05A1EAA
:10B84000012A6BD900232383A4F87830A4F8D830D8
:10B8500028F02AF8002860D10023EA0484F84F3049
:10B8600084F8AF3084F80F315DD5654BDA79022A60
:10B8700008BF01224FF00A0008BFDA7127F0BAFFB3
:10B88000002840F0D3804FF480602EF035FB002874
:10B8900000F02E814FF40070FFF766FE4FF4003089
:10B8A000FFF762FE4FF40010FFF75EFE554C4FF0BD
:10B8B0000070FFF759FE4FF08060FFF755FEA38838
:10B8C000002B40F0AB80504A1368DB0DDB050BB159
:10B8D00000231360936823F4007323F002030BB179
:10B8E000002393601379013B042B01D901231371C9
:10B8F000F8BD0023A3816382A4F86C30A4F87230F1
:10B90000A4F8CC30A4F8D23027F0CEFF002899D08C
:10B91000737E5A1E012A95D800E0737E023B022BEB
:10B920009AD8EA04A1D42B06ADD49EE7F37B002B72
:10B9300000F0CF80002386F8233079E700232146EA
:10B9400013703FE700232649537030E721482CF05D
:10B9500039FA02202EF0D0FA00287FF41EAF8020A2
:10B96000FFF702FE19E7D80014186468002C7FF472
:10B97000CBAE17240C70C7E64FF48050FFF7F4FDF0
:10B980008B8AB3F57A7F37BF4FF47A728B788B78D6
:10B990008A8228E71D48FFF7E7FD35686B047FF5CD
:10B9A00039AF1B48FFF7E0FD35682F077FF535AF4E
:10B9B0001848FFF7D9FD3568A8047FF531AF164860
:10B9C000FFF7D2FD35682BE7C4350020849B0408BF
:10B9D000D090040834BB002081808080BC9B002074
:10B9E0001E6D0020E8560020D46B0020E456002095
:10B9F00088A50020A0700020096000023CB2002051
:10BA0000847100201E870020A837002008600002F3
:10BA10000920000201600002094000022078FEF7C0
:10BA2000B3FA00287FF44FAFA0804CE7354F0022D7
:10BA300007F1060E1146944601EB4100430017F84A
:10BA400010000A2807EB030540D05B1B28464E1C5C
:10BA5000EABB7344142E1D443FF415AF10F8062FB3
:10BA60000A2A08D00136142E1D443FF40CAF10F8FA
:10BA7000062F0A2AF6D101229319132B15D803EBAE
:10BA8000430007EB400117F810000A2808BF0133F4
:10BA900005D012E011F8064F0A2C0ED10346132BE5
:10BAA00002F1010203F10100F4D9C5F800C0A5F8C4
:10BAB00004C0711C1429BFD1E5E603EB430307EB77
:10BAC0004303196829609B88AB80F2E752B10E46A8
:10BAD000D2E742F201031D423FF4AAAE002386F8EA
:10BAE0002330A5E60E460122C6E718230B7014E6A4
:10BAF0004FF00060FFF738FDCCE645F008053560F3
:10BB000082E600BFB83600202DE9F84F0CF048F966
:10BB10002B4B2C4A934250D22B4F03F114069B46D9
:10BB20004FF00108294C258862197DB1BA420DD227
:10BB3000052D0BD936F8143C6188C3F30B039942E9
:10BB40000AD0144625886219002DEFD156F8101C32
:10BB50005846FCF7F7FF0FE0637913F0030AF0D1C2
:10BB600056F8101C94F804905846FCF7EBFF36F892
:10BB7000141CB9EB113F11D04FF00008114B0BF121
:10BB8000140B9B4506F11406CCD3FFF7AFFDFDF770
:10BB900093F80CF0E5F84046BDE8F88F36F8123C13
:10BBA00056F8100CAA1FC3F30B039A4204F10601C6
:10BBB000A8BF1A4639F03EFAE0E74FF00108E4E783
:10BBC000A0010008C8060008008000080240000824
:10BBD000DFED2E7AB4EEE70AF1EE10FA4ADDDFED82
:10BBE0002C6A9FED2C7A01E0B0EE670AB4EEC70A2A
:10BBF000F1EE10FA70EE667AF6DC9FED277AF4EE3D
:10BC0000C77AF1EE10FA3ED5DFED216A9FED237A77
:10BC100001E0F0EE407AF4EEC77AF1EE10FA37EE7A
:10BC2000A60AF6D4DFED1E7AB4EEE70AF1EE10FABA
:10BC300014DDDFED167A37EEC00A60EE006A9FED84
:10BC4000196A9FED197ADFED197AA6EE867A20EE51
:10BC5000266AE6EE877AA6EE270A7047DFED147AA9
:10BC6000B4EEE70AF1EE10FA44BFDFED0B7A37EEDF
:10BC7000C00AE2E79FED087AF0EE407AF4EEC77A68
:10BC8000F1EE10FAC0D4B0EE670ACBE7DB0F494003
:10BC9000DB0FC940E4CB1641DB0F49C0E4CB16C132
:10BCA000DB0FC93F92E741B99730083C15A82ABE7F
:10BCB000DB0FC9BFF0EEC07AB0EEE07AB4EEE77AFF
:10BCC000F1EE10FAB4BFB0EE676AB0EE476AB5EEB7
:10BCD000406AF1EE10FA46D0B4EEE77AF1EE10FACF
:10BCE0008CBFF0EE675AF0EE475AC5EE866A9FEDBC
:10BCF0001F3A9FED1F6A9FED1F4A9FED1F5ADFED10
:10BD00001F3ADFED1F4ADFED1F5AA6EEC36AE6EECB
:10BD1000A34AA6EE864AB7EE006AA6EE845AA6EEBD
:10BD2000A46AE6EE855AC5EE866AB4EEE77AF1EECD
:10BD300010FA48BFDFED147AF5EEC00A48BF77EE7F
:10BD4000E66AF1EE10FA48BFDFED107AB5EEC00AF0
:10BD500048BF77EEE66AF1EE10FA48BFF1EE666A88
:10BD6000B0EE660A7047DFED076ADEE739094E3D3F
:10BD7000E3B59E3E88FA163E45FE7F3F99FB243F81
:10BD800069A2163EA7DFA834DB0FC93FDB0F49408D
:10BD9000DFED317A30EE277AFDEEC76A16EE903A83
:10BDA0002033402B02D99FED2D0A7047B4EEE70AED
:10BDB000F1EE10FA4DDD9FED2A6ADFED2A6A01E00F
:10BDC000B0EE677AB4EEE67AF1EE10FA77EE467AE4
:10BDD000F6DC9FED257AF4EEC77AF1EE10FA35D550
:10BDE000DFED1F6A9FED217A01E0F0EE407AF4EE7C
:10BDF000C77AF1EE10FA37EEA60AF6D4DFED167A1E
:10BE0000B4EEE70AF1EE10FA1BDCDFED197AB4EEBE
:10BE1000E70AF1EE10FA44BFDFED137A37EEC00AFD
:10BE200060EE006A9FED136A9FED137ADFED137ADF
:10BE3000A6EE867A20EE266AE6EE877AA6EE270A36
:10BE40007047DFED0F7A37EEC00AE9E7B0EE670A18
:10BE5000D4E7F0EE477ABCE7DB0FC93F00000000F3
:10BE6000DB0FC940E4CB1641DB0F49C0E4CB16C160
:10BE7000DB0FC9BF92E741B99730083C15A82ABE2D
:10BE8000DB0F494010B44C09012250F8243001F076
:10BE90001F0102FA01F10B4340F824305DF8044B16
:10BEA000704700BF4B0901F01F0150F82320012308
:10BEB00003FA01F1114214BF18460020704700BF79
:10BEC0002DE9F04FDE4D2DED068B2B7893B0044617
:10BED00043B1DFF8BCA3DAF80C305046984780F045
:10BEE00001002870D74B1A78002A00F00282D64948
:10BEF000D648D74E0D7804F5EC425F320260002040
:10BF000032681870002D00F0F981944201D9013D8A
:10BF10000D70204628F052FD002800F0EA81CD4D3A
:10BF2000CD4ED5F81C31C5F81C41E41A47F2305308
:10BF30009C42A8BF1C46C94A3778C94BDFF85483D6
:10BF4000B4F57A7FB8BF4FF47A7414800122174099
:10BF50001A7000F06782C34AB8F906301268D189B6
:10BF60008B4280F22482C04A4FF07E511160BF4A5A
:10BF7000DFF824C392F90410BCF81260B8F90090FD
:10BF8000107892F801E0BA4CA9EB0602002914BF20
:10BF900001214FF0FF31002AB8BF5242B2F5FA7FBB
:10BFA000A8BF4FF4FA728242C5BF121A07EE902A58
:10BFB000DFEDB07AF8EEE77A4E45B8F90290C4EDBD
:10BFC000007AA9EB0602C4BFF1EE677AC4ED007AED
:10BFD000002AB8BF5242B2F5FA7FA8BF4FF4FA72F6
:10BFE0009042BABF121A07EE902ADFEDA27AB8F992
:10BFF0000400B8BFF8EEE77A4E45A0EB0602C4EDA8
:10C00000017AC4BFF1EE677AC4ED017A002AB8BFA5
:10C010005242B2F5FA7FA8BF4FF4FA72964580F209
:10C02000DE81A2EB0E0E01FB0EFE07EE90EAF8EEAB
:10C03000E77A914AC4ED027A86421168C4BFF1EEF4
:10C04000677AC4ED027A11F4805100F09C81B3F557
:10C05000FA6FA8BF4FF4FA63B3F57A7FB8BF4FF415
:10C060007A73A3F57A70854B1A78002A40F095818F
:10C07000DFF82882DFF828C288FB0023C217C2EB52
:10C08000631303F1010E6FF063023CF91EE03CF90B
:10C0900013C002FB0303AEEB0C0003FB00F388FBB1
:10C0A0000302DB17C3EB621363441BB207EE903A43
:10C0B000F8EEE77AC4ED037A002940F08882704BED
:10C0C0001B885A0640F1118140F603026D49D4EDF8
:10C0D000011AD1ED010AD1ED033AD1ED028AD1ED79
:10C0E000005A94ED002A1340674A08BFD4ED022A93
:10C0F00092ED019A92ED026A92ED031A92ED004AD6
:10C1000018BFDFED5C2A614A30EEE35A79EE466AE9
:10C1100075EEE84A65EE266A74EE017A35EEA8AA55
:10C1200074EE419A24EEA70AB0EE663AAAEE293AD6
:10C13000B0EE405A30EEA37A79EE067AAAEE295A8A
:10C14000A7EE273AA7EE675AF0EE664AD7EE274ADF
:10C1500033EE003AB6EE008A75EEA0AA28EE433A16
:10C1600035EE665A74EE096AB0EE647AEAEE694A10
:10C17000AAEEA63A77EE407A76EE416A73EEE8AA26
:10C1800025EE085AEAEE297AAAEEA65A74EE804AFB
:10C1900063EE036A34EE494A73EEA83A64EE884AC5
:10C1A00075EEE05A36EE016A67EE887AB0EE667A8E
:10C1B000E3EE844A95EE057AE5EE056AE5EE867AC9
:10C1C000B1EE648AF0EE665AF0EE476AB1EE674A65
:10C1D000E8EE246A63EE270A67EEA43AE4EE275AF3
:10C1E000B1EE450AB0EE609AB0EE631AA4EE277A7B
:10C1F00023EE244AE7EEA76AA5EE249AA0EE031ADE
:10C20000E8EE245AB0EE448A31EEA16AE0EE240A48
:10C21000A5EE278A66EEA16A72EE028AE5EE033A7F
:10C2200061EE211A26EE096AA4EEA47AA0EE274A4E
:10C23000A2EE256AE8EEA06AE2EE081A32E000BF3C
:10C24000B92F0020B82F00206C360020B42F00201A
:10C2500068360020A8260020DE510020423200204F
:10C26000E87A0020E8560020F08200203472002096
:10C27000105200200000000084A300202C81002028
:10C280003C5200203C230020E822002024230020F0
:10C290009C2F0020C65400203CB200201F85EB518B
:10C2A000CC7A002073EEA33A27EE227A34EE044AC9
:10C2B000F0EE005AE2EEA36AA2EE846AA1EEA57A3D
:10C2C000C5ED496AC4ED016A85ED486A84ED006AEE
:10C2D00085ED4A7A82ED005A82ED013AC2ED027A8A
:10C2E000C2ED034A002B00F09A80002F7AD12AF089
:10C2F0001BFE13B0BDEC068BBDE8F08F94427FF6B9
:10C3000008AECC4B1E78002E00F0B881DFF85CA39D
:10C31000DFF85CB3DFF85C83DFF85C93574628E016
:10C3200018F805109847032D03462ADCC8B109EB1D
:10C33000850339F825105A88401A4FF47A7303FBA5
:10C3400000F0521A40F6CA0390FBF2F000F57A7042
:10C350009842A8BF184640F2EE239842B8BF18464C
:10C3600000B2B44B2BF8020B1E780135B54280F2B7
:10C370008581072D3846DAF80430D1DDE9B29847D7
:10C38000034618B2EDE7BCF81420934237DAAA4B03
:10C390001A780846002A3FF46BAE5B78A74A00FB88
:10C3A00003F382FB0320DB17C3EB601060E6B3F5F9
:10C3B000FA6F127B9FEDA27ABFBF581A4243C1F5B4
:10C3C000FA6192FBF1F2C2F1640207EE902AF8EEF4
:10C3D000E77A9C4A67EE877AC2ED007AC7E5DFED1F
:10C3E0009A7A26E6994A9A4B1178186801F0010169
:10C3F000FEF7E4FC13B0BDEC068BBDE8F08FB3F59F
:10C40000FA6FD4BFC2EB0303C2F5FA634FF47A703C
:10C41000C2F5FA6200FB03F3B3FBF2F023E684ED0E
:10C42000027A62E7B8F90090B8F902E0B8F90CC0F6
:10C43000B8F90440B8F90800B8F90610B8F90E20A8
:10C44000B8F90A30DFF820A2B9F5FA6FA8BF4FF4A7
:10C45000FA69BEF5FA6FA8BF4FF4FA6EBCF5FA6F31
:10C46000A8BF4FF4FA6CB4F5FA6FA8BF4FF4FA64A2
:10C47000B0F5FA6FA8BF4FF4FA60B9F57A7FB8BF8C
:10C480004FF47A79BEF57A7FB8BF4FF47A7EBCF567
:10C490007A7FB8BF4FF47A7CB4F57A7FB8BF4FF497
:10C4A0007A74B0F57A7FB8BF4FF47A70B1F5FA6F4D
:10C4B000A8BF4FF4FA61B1F57A7FB8BF4FF47A7133
:10C4C000B2F5FA6FA8BF4FF4FA62B2F57A7FB8BF3F
:10C4D0004FF47A72B3F5FA6FA8BF4FF4FA63B3F56D
:10C4E0007A7FA0F57A70B8BF4FF47A73C0EBC010B2
:10C4F000A9F57A79AEF57A7EACF57A7CA4F57A74F2
:10C50000A1F57A71A2F57A724000A3F57A73AAFBBD
:10C5100000B0C9EBC919CEEBCE1ECCEBCC1CC4EBE2
:10C52000C414C1EBC111C2EBC212C3EBC3135B0055
:10C5300080094FEA49094FEA4E0E4FEA4C0C64005D
:10C5400049005200AAFB09B9AAFB0EBEAAFB0CBC0B
:10C55000AAFB04B4AAFB01B1AAFB02B2AAFB033AEC
:10C56000A0F17F033B488DF8443090F812314FEA38
:10C5700099194FEA9E1E4FEA9C1CA4098909920949
:10C580004FEA9A1AA9F17F09CEF17F0EACF17F0C28
:10C590007F3C7F397F3AAAF17F0A032B8DF84090C8
:10C5A0008DF841E08DF842C08DF843408DF845107C
:10C5B0008DF846208DF847A07FF4CDAC082310AA53
:10C5C000832115F00DFD377807F00107C3E4224BF6
:10C5D000DB78002B7FF473AD204B214893F80C805F
:10C5E0001821FFF75FFCB8F1000F40F031810028FF
:10C5F0003FF465AD9FED1B7A1B4977EEC77AC6F510
:10C60000FA63FDEEE77A1AB217EE903A1BB21B03FB
:10C6100081FB0301DB17C3EBA11302FB03F343F31D
:10C620000F33334407EE903AF8EEE77AC4ED037A1D
:10C6300045E500BFA03700202C8100201F85EB516D
:10C640000AD7233CF082002000000000D889002097
:10C65000DC89002024930020E0510020D8790020BC
:10C66000FC33002000007A44D34D62109C2F002040
:10C670003C2700203CB20020083B0020B74B1A7832
:10C68000B74BD3F80090002A40F0DD801346B5493F
:10C6900009780491292904D1B348B4490078488025
:10C6A0000A80B34A01251570002E00F0A781B14A17
:10C6B000B14F10780390B148DFF8F8C2C18B0191F7
:10C6C000018C0291418A03980A91397B0D910746AA
:10C6D000ACFB07714908079201EB4101A84ADFF85A
:10C6E000D8A21268DFF8ACB20B95411AC8B206F1B5
:10C6F000FF380590CDE90864400042F20101069040
:10C70000B8F1030F02F480500C9002EA0102A8BFB6
:10C710004FF003080025002B00F0BF8099490198D5
:10C7200031F8151081424FEA4507C0F0B6800298F3
:10C73000814200F2B28009F596704AF8250009B2EC
:10C74000002A40F0CA802BF8071001354545E2DD8C
:10C75000DDE90864B54227DA8B4FDFF838B206947A
:10C7600005EB450107EB4107002B00F0DC80854914
:10C77000019831F8151088424FEA450800F2D3803D
:10C7800002988842C0F0CF8009F596704AF82500DB
:10C7900009B2002A40F012812BF808100135AE4290
:10C7A00007F10607E0D1069C714B1B78002B40F087
:10C7B00027816D4B012204201A7011F06BFD734A22
:10C7C000674BD2E901101B68D3601B1A8B4202D958
:10C7D000002382F821306E4B1E78624B1B78049345
:10C7E000002E00F02481644A654B117B1B68634A6C
:10C7F00003F48053B2F81E80578A002900F0448168
:10C800006449654D83B1AAE1022A40F0258142784E
:10C8100002EB820202EB820202F2EE2201339E421E
:10C8200021F8022B00F0038115F8132005EB4300DB
:10C83000002AE9D1DAB2022A40F25E81032A40F0EE
:10C840000B814246EAE7484B1B7883F001031EE761
:10C850009FED527A524A77EEC77AFDEEE77A17EEED
:10C86000903A1BB21B0382FB0312DB17C3EBA2132C
:10C87000002800F02B81C6F57A7212B203FB02F396
:10C8800043F30F33334407EE903A464BF8EEE77A22
:10C890000122C4ED037A1A7011E45AF82510A9EBAD
:10C8A00001010029FFF651AF3B4810F815106F0049
:10C8B0003844002900F0D280022940F0CA80417833
:10C8C00001EB810101EB810101F2EE21284C0020F6
:10C8D000207009B2002A3FF436AF2B48324C069E36
:10C8E00094F800E107EB050C00EB4C008153BEF11E
:10C8F000000F06D1039E022E7FF625AF0B9984F818
:10C9000000114188B0F804E01F4830F81C00714461
:10C91000014408B2254981FB0041254CA1EBE0719F
:10C92000E05309B20FE75AF82510A9EB01010029DD
:10C93000FFF634AF184810F815104FEA4508404488
:10C94000002900F09680022940F08080417801EBB8
:10C95000810101EB810101F2EE2119E75D5C00200C
:10C96000108A00200D88002022000020108800205E
:10C97000043400206D360020D87900203CB200201D
:10C9800084A300203C27002060270020E0510020E5
:10C99000A0370020C65400207F3B002000007A44CE
:10C9A000D34D6210087A0020A82600205655555510
:10C9B000AC270020ABAAAAAA703600208C48059CA0
:10C9C00090F8000127F8141038B9039C022C7FF668
:10C9D000E3AE8748012180F800117988B7F800C0DC
:10C9E000B8886144014408B2824981FB0041824C0D
:10C9F000A1EBE07124F8080009B2CDE67F4B079364
:10CA00007F480921FFF74EFA00287FF4D2AE7D4A15
:10CA10007D4BD1681B6893605B1AC82B07D97B4993
:10CA20000B68012023F004030B6082F82100049BB3
:10CA3000292B05D1DFF8DC81754BB8F80620DA80A8
:10CA4000079A137801331370FFF763BA3BF80810A5
:10CA50009EE63BF8071039E70A88DFE6E9B20229CB
:10CA600048D90329F5D10C99002940F09C800199FF
:10CA70002CE7E9B202293BD90329E7D10C99002917
:10CA800040F0A380019983E6002B39D16149624DC2
:10CA90000DE0022A18D1427802EB820202EB8202F8
:10CAA00002F2EE2201339E4221F8022BBFD015F88C
:10CAB000132005EB4300002AEBD1DAB2022A1DD97C
:10CAC000032A01D14246EDE70A88EBE7C6F5FA6290
:10CAD00012B203FB02F343F30F33334407EE903AF1
:10CAE0004E4BF8EEE77A1870C4ED037AFFF7E7BA19
:10CAF0000A994DE60A99E9E63A468FE63A46D1E7C1
:10CB0000DFF810A1444DDFF8F8B089460EE0022BA3
:10CB100022D1507800EB800000EB800000F2EE2084
:10CB200009F10109B1452AF8020B80D015F8193036
:10CB300005EB4902002BEAD15FFA89F3022B2ED9CB
:10CB4000032B4FF01801584606D1FFF7ABF9002828
:10CB50000CBF38464046E3E7BAF80000E0E70023A0
:10CB60000EE0022A19D1427802EB820202EB820225
:10CB700002F2EE2201339E4221F8022B3FF457AF1E
:10CB800015F8132005EB4300002AEAD1DAB2022A95
:10CB900007D9032A01D14246ECE70A88EAE738467A
:10CBA000BEE73A46E6E718211548CDE90E32FFF711
:10CBB00079F9DDE90E3200287FF459AF0D9901981B
:10CBC00000290A9918BF014680E618210C48CDE9D2
:10CBD0000832FFF767F9DDE9083200287FF452AF29
:10CBE0000D99019800290A9918BF0146D0E500BFA8
:10CBF000A826002056555555AC2700206D3600203C
:10CC0000FC330020E0510020108A002090540020C6
:10CC100010880020C65400207F3B0020087A0020A6
:10CC20002DE9F043002489B006460D461F46A04674
:10CC300005E025290CD030460134A847039A531C3F
:10CC4000039311780029F4D1204609B0BDE8F083A0
:10CC5000931CCDE903385078302842D0A0F130033E
:10CC6000DBB2092B4FF0000945D96C282AD0642883
:10CC700073D019D9732858D063D9752840F08280B1
:10CC800007F1040C386805AB00220A216746FBF760
:10CC900053FC05AB049A009329464B463046FBF7FC
:10CCA000CFFA039A0444CAE725283CD051D9582822
:10CCB0006BD06328C2D139783046A8470437013495
:10CCC000039ABCE7039B5A1C03921B78642B52D037
:10CCD00016D8252B27D064D9582B18D0632BEAD02F
:10CCE000ADE7D31C03939078A0F13003DBB2092B9E
:10CCF0004FF00109B9D804AA03A934F091F9B4E7B7
:10CD0000732B12D051D9752B2DD0782B97D1A3F13D
:10CD10005802B2FA82F23868520905AB1021043782
:10CD2000FBF70AFCB5E7252185E73B68049A0093E9
:10CD3000294600233046FBF783FA04370444039A5C
:10CD40007DE76E287FF47AAF039A3B6804371C6056
:10CD500075E700283FF478AF70E7386805A9FBF75E
:10CD6000B5FB043795E7386805AB00220A21FBF7CD
:10CD7000E3FB04378DE73B1D386805A91F46FBF729
:10CD8000A5FB86E778287FF459AFA0F15802B2FAE4
:10CD900082F23868520905AB1021FBF7CDFB04374E
:10CDA00077E7002B3FF450AF49E76E2BCDD046E735
:10CDB0000EB400B584B005AB019053F8042B0649BE
:10CDC000039301A8FFF72CFF019B00221A7004B007
:10CDD0005DF804EB03B070473582000870B4066854
:10CDE0008E4217D90139751E002311F8014F082210
:10CDF000634013F0800F4FEA430318BF83F0D5035D
:10CE0000013ADBB2F5D18D42EFD1721C0260337072
:10CE100070BC7047721C00230260337070BC704796
:10CE20000A44914215D010B40139541E11F8012F53
:10CE30000823504010F0800F4FEA400018BF80F0E8
:10CE4000D500013BC0B2F5D1A142EFD15DF8044B52
:10CE5000704770474840082310F0800F4FEA4000A9
:10CE600018BF80F0D500013BC0B2F5D1704700BFBC
:10CE70002DE90048FBF7F4FA054A064B1268B0EBBF
:10CE8000020B61F1000CC3E900BC0120BDE8008881
:10CE9000108A0020B86E00200F4B2DE93048D3E9EE
:10CEA000004554EA05020AD1034640F2011200206F
:10CEB0001880988098715A801881BDE83088074B97
:10CEC0001A6814EB020B45F1000C5A466346FBF757
:10CED0000DFA0120BDE83088B86E0020108A0020CD
:10CEE0002DE9F04707468CB01E469246002A5CD1D9
:10CEF000154614460A88B2F5FA6F36D38B78581E59
:10CF00000B2832D891F803C00CF1FF301E282CD822
:10CF100091F804E0BEF1170F27D891F80590B9F108
:10CF20003B0F22D888793B281FD8B1F80880B8F584
:10CF30007A7F1AD24FF001085EBB09890491002C58
:10CF4000B4BF2D212B21002CB8BF6442CDE9029043
:10CF5000CDE905140795CDE900CE38462A49FFF7FB
:10CF600027FF40460CB0BDE8F08700232749ADF805
:10CF700028304FF0010C18468DF82A30ADF82C30CF
:10CF800099469E461A4698460991634609A9002E7D
:10CF9000D3D0CDE90290CDE900CE38461C49FFF749
:10CFA00007FF40460CB0BDE8F0871A4C84FB023402
:10CFB000A318D417C4EB6314C4EB0415A2EB8505C6
:10CFC0002DB2002D0846B8BF6D42FBF749FA4FF469
:10CFD0007A7200238046894637F0F0FD3C230AFB35
:10CFE000030A4FF47A7200234046494637F0E6FDC3
:10CFF0004FF47A7192B20023C1FB0A2309A8FBF710
:10D0000075F924B209A975E7B0A10408000001016F
:10D0100090A10408898888880378202B024600F1B3
:10D020000100F9D0092BF7D02D2B00F0A4802B2B79
:10D0300003BF5378B7EE000A0246B7EE000AA3F129
:10D040003001C8B209289FED577A10D8F2EE046A71
:10D0500007EE901AF8EEE77A12F8013FE7EE267A2B
:10D06000A3F13001C8B20928B0EE677AF0D92E2BAF
:10D0700063D003F0DF03452B02D020EE070A704790
:10D0800010B451782D294FD02B2979D0A1F130033C
:10D09000092B02F101027AD80024002303EB830359
:10D0A00001EB430312F8011FA1F130000928A3F19D
:10D0B0003003F3D9B3F59A7F1A4628BF4FF49A721A
:10D0C000072B6CD9DFED386A1346F7EE007A083B80
:10D0D000072B67EEA67AFAD802F00702DAB1F2EE71
:10D0E000046A012A67EEA67A15D0022A67EEA67AAC
:10D0F00011D0032A67EEA67A0DD0042A67EEA67A2D
:10D1000009D0052A67EEA67A05D067EEA67A062A28
:10D1100018BF67EEA67A002C3BD087EE277A5DF821
:10D12000044B20EE070A70479178A1F13003092BD8
:10D1300002F1020230D80124AFE75378A3F13001A5
:10D14000C8B2092802F1010293D8F2EE046AF0EEA7
:10D15000665A07EE901AF8EEE77A12F8013F87EE6A
:10D16000A66AA3F13001C8B2092866EEA56A37EEB7
:10D17000067AEED97DE75378BFEE000A02465EE7F5
:10D180009178A1F13003092B02F1020284D9F7EE64
:10D19000007A27EE277AC2E7F7EE007ABDE7F7EECE
:10D1A000007A9BE70000000020BCBE4CF8B50646A4
:10D1B00015460846B6FBF2F434B905FB14640C4B73
:10D1C0001B5D00F8013BF8BDB4FBF2F75FB905FB4E
:10D1D0001747074B05FB1464DA5D00F8012B1B5D54
:10D1E00000F8013BF8BD3846FFF7E0FFEFE700BF6E
:10D1F000E0A10408B5EEC00ADFED677A674AF1EEF8
:10D2000010FACCBF30EE270A30EE670ADFED647A01
:10D2100020EE270A2DE9F047FDEEC07A88B017EE20
:10D22000904A84EAE4760023A6EBE476CDE9023363
:10D230000493A2FB06325FEAD208054641D105AF4E
:10D2400058483946554BA3FB0623DB0803EB830301
:10D25000A6EB4303002CC35C0B704FF00002ACBF85
:10D2600020232D234A7038468DF8083036F0BAFF57
:10D270000128394639D0022842D0032805BF30237F
:10D2800002A802A88DF8093039F0D0FA02A836F0C9
:10D29000A9FF0338C4B2224602A9284639F0FCFA95
:10D2A00000232B55284636F09DFF2E22431C02A951
:10D2B0002A542144E81839F0D5FA284608B0BDE8C8
:10D2C000F087394BA3FB06235B0922D105AF354814
:10D2D0003946324AA2FB0832D20802EB8202A8EB9E
:10D2E0004202835C01F8013BACE7302302A88DF8D1
:10D2F00009308DF80A308DF80B3039F097FAC5E710
:10D30000302302A88DF809308DF80A3039F08EFAF2
:10D31000BCE7264AA2FB06125FEA92190ED105AFBE
:10D32000204839461D4AA2FB03C2D20802EB820202
:10D33000A3EB4203C35C01F8013BCAE71C4AA2FB12
:10D3400006125FEA523A0ED105AF16483946134A23
:10D35000A2FB09C2D20802EB8202A9EB4202825C64
:10D3600001F8012BDEE71348B6FBF0F058B905AF22
:10D3700039460A20BAFBF0F200FB12A20948825C8F
:10D3800001F8012BE3E705AF39460A220193FFF7C5
:10D390000DFF019B0146ECE76F12033ACDCCCCCCDC
:10D3A00000007A44E0A104081F85EB51D34D6210C0
:10D3B0005917B7D1A086010002B370B48E1803E0EC
:10D3C000121B14D1B14215D010F8012BA2F1410368
:10D3D000192B11F8013BA3F1410598BF2032192DFB
:10D3E00003F12004ECD9D21A01D1002BEAD1104666
:10D3F00070BC70470022104670BC704710467047E2
:10D4000070B5044608460D4636F0ECFE064602E0CE
:10D4100014F8013F43B1324629462046FFF7CCFFBE
:10D420000028F5D1204670BD1C46204670BD00BFC7
:10D430004FF0FF32FFF7C0BFA0F16103192B98BF77
:10D4400020387047A0F14103192B98BF2030704756
:10D45000202805D0093804288CBF002001207047FF
:10D46000012070472DE9F0411F46064603461C780F
:10D470002046FFF7EDFF1D4601330028F7D12B2C86
:10D4800051D02D2C24D0102A804628D04FF0FF33C5
:10D49000B3FBF2F302FB03FC6FEA0C0C5FFA8CFCAB
:10D4A000013500200BE0303CE4B2944225DA98428A
:10D4B0002E461DD81AD002FB004015F8014B392C1E
:10D4C000F1D944F02004602C17D9573CE4B2ECE7C2
:10D4D0004FF00108102A6C7805F10105D6D1302CE7
:10D4E00023D06FF070434FF00F0CD9E76445E2D9B9
:10D4F00007EA08084FF0FF30DFE701B10E60B8F12E
:10D50000000F08D027B1B0F1004F28BF4FF0004006
:10D510004042BDE8F081002FFBD06FF000439842FD
:10D5200028BF1846F5E78046D4E76C782046FFF719
:10D5300089FF782805F1010605D035466FF0704364
:10D540004FF00F0CACE7AC786FF0704302354FF042
:10D550000F0CA5E701230A22002183E7613819286F
:10D560008CBF002001207047413819288CBF002053
:10D5700001207047303809288CBF002001207047F7
:10D58000A0F13003092B07D920F0200041381928D9
:10D590008CBF0020012070470120704707EE901AD1
:10D5A000F8EE677A9FED837A27EE800A20EE070A6D
:10D5B000FDEEC07A17EE903A2033402B00F28180C6
:10D5C000DFED7D7AB4EEE70AF1EE10FA40F3E68083
:10D5D000B0EE407A9FED796ADFED796A01E0B0EE56
:10D5E000677AB4EEE67AF1EE10FA77EE467AF6DC78
:10D5F0009FED747AF4EEC77AF1EE10FA40F1D18023
:10D600009FED6E6ADFED706A01E0F0EE477AF4EEAE
:10D61000E67AF1EE10FA37EE867AF6D4DFED6B7A21
:10D62000B4EEE77AF1EE10FA40F3A780DFED627A0C
:10D6300037EEC77A27EE076ADFED655ADFED657AC8
:10D64000DFED656A9FED655AE6EE257A67EE065ACC
:10D65000E6EE276AF7EE007AA5EEA67AF0EE675AB4
:10D66000E7EE055AE7EE457A87EEA55ADFED577AE1
:10D6700030EE277AFDEEC76A16EE903A2033402B43
:10D6800024D99FED577AF6EE006AB7EE006AF7EEFE
:10D69000004AC4EEA57A0023836143610362C3613B
:10D6A00080ED045A67EEA66A27EE866A27EE877A2F
:10D6B000C0ED006AC0ED026A80ED016A80ED037A78
:10D6C0007047B7EE005AF0EE455ACFE7B4EEE70ADE
:10D6D000F1EE10FA6BDD9FED396ADFED396A01E09A
:10D6E000B0EE677AB4EEE67AF1EE10FA77EE467AAB
:10D6F000F6DC9FED347AF4EEC77AF1EE10FA53D5EA
:10D700009FED2E6ADFED306A01E0F0EE477AF4EE2D
:10D71000E67AF1EE10FA37EE867AF6D4DFED2B7A60
:10D72000B4EEE77AF1EE10FA33DCDFED2E7AB4EEE8
:10D73000E77AF1EE10FA44BFDFED227A37EEC77ACE
:10D7400027EE076ADFED224ADFED226ADFED227A5B
:10D75000E6EE246A67EE064AE6EE267AB7EE006A3F
:10D76000A4EEA77AF6EE006A36EE476AF8EE007A83
:10D7700027EE277A66EE266A89E7DFED1A7AB4EE9D
:10D78000E77AF1EE10FA44BFDFED0E7A37EEC77A92
:10D7900050E7DFED097A37EEC77AD1E7F0EE407A4D
:10D7A00026E7B0EE677A39E7B0EE677AB6E7F0EED3
:10D7B000477A9EE727D4D236DB0F4940DB0FC940BA
:10D7C000E4CB1641DB0F49C0E4CB16C1DB0FC93FE8
:10D7D00092E741B99730083C15A82ABEF304353FBB
:10D7E00000000000DB0FC9BF30B402681146531CB3
:10D7F000036011F8024B0160D31C517803609378E9
:10D80000151D05601B0443EA0123D078234343EA36
:10D81000006030BC704700BF0368591C1A460160A5
:10D8200012F8021B0260587841EA0020704700BFDE
:10D8300003685A1C02601878704700BF70B5044630
:10D8400008460E4636F0CEFC3146054602462068B4
:10D8500037F0F0FB20682844206070BD38B50446DE
:10D860000068154637F0E6FB22682A44226038BD7E
:10D87000036810B40A0E5C1C04601A7003680A0C7A
:10D880005C1C04601A7003680A0A5C1C04601A704D
:10D8900003685A1C026019705DF8044B704700BFA2
:10D8A000036810B40A0A5C1C04601A7003685A1CEE
:10D8B000026019705DF8044B704700BF03685A1C82
:10D8C000026010B4197003680A0A5C1C04601A70C4
:10D8D00003680A0C5C1C04601A700368090E5A1C69
:10D8E000026019705DF8044B704700BF03685A1C52
:10D8F000026019700368090A5A1C026019707047A7
:10D9000038B5064C064DAC4206D261682046143448
:10D91000FBF718F9AC42F8D338BD00BFA0010008EE
:10D92000C8060008084B09498B4203D309E01433A9
:10D930008B4206D21A88C2F30B029042F7D11846E6
:10D940007047002318467047A0010008C806000869
:10D950002DE9F047A84F3B7803B1FEE7A74EB36827
:10D9600001223A7013B11A689B885383A44B012299
:10D970008A461A70014640F2E933706802E0002BD3
:10D9800000F07C810289013B12F0020F9BB2F6D0BD
:10D990000023838140F2E93302E0002B00F06E8126
:10D9A0000289013B12F0010F9BB2F6D0838940F24D
:10D9B000E93302E0002B00F075810289013B12F08F
:10D9C000020F9BB2F6D00023838140F2E93302E0DC
:10D9D000002B00F067810289013B12F0010F9BB21E
:10D9E000F6D0838940F2E93302E0002B00F0568143
:10D9F0000289013B12F0020F9BB2F6D0092383810A
:10DA000040F2E93302E0002B00F048810289013B3B
:10DA100012F0010F9BB2F6D0838940F2E93302E0A5
:10DA2000002B00F037810289013B12F0020F9BB2FC
:10DA3000F6D089B2818140F2E93302E0002B00F098
:10DA400029810289013B12F0010F9BB2F6D0838934
:10DA5000DFF8B0810AF1FF3A00244FF00A090B25E4
:10DA600040F2E93302E0002B00F0E6800289013B3E
:10DA700012F0020F9BB2F6D0A0F80C9040F2E933FE
:10DA800002E0002B00F0D8800289013B12F0010F68
:10DA90009BB2F6D0838940F2E93302E0002B00F01C
:10DAA000D7800289013B12F0020F9BB2F6D0A3B2DD
:10DAB000838140F2E93302E0002B00F0C980028943
:10DAC000013B12F0010F9BB2F6D083891AF8011FB7
:10DAD00040F2E93302E0002B00F0B2800289013B02
:10DAE00012F0020F9BB2F6D0858140F2E93302E0DA
:10DAF000002B00F0A5800289013B12F0010F9BB2C0
:10DB0000F6D0838940F2E93302E0002B00F09C80DC
:10DB10000289013B12F0020F9BB2F6D089B28181DB
:10DB200040F2E93302E0002B00F08E800289013BD5
:10DB300012F0010F9BB2F6D08389D8F8003033B1D0
:10DB40001A689B8851690B4214BF538313830134B5
:10DB5000362C85D140F2E93302E0002B00F09680AC
:10DB60000289013B12F0020F9BB2F6D00823838199
:10DB700040F2E93302E0002B00F088800289013B8B
:10DB800012F0010F9BB2F6D0838940F2E93301E035
:10DB9000002B77D00289013B12F0020F9BB2F7D025
:10DBA000A023838140F2E93301E0002B6AD002898F
:10DBB000013B12F0010F9BB2F7D08389A024002112
:10DBC00040F2E93301E0002B46D00289013B12F01C
:10DBD000020F9BB2F7D0848140F2E93301E0002BC1
:10DBE0003AD00289013B12F0010F9BB2F7D0838932
:10DBF00040F2E93309E000BF55700020CC870020D7
:10DC000056700020DC89002053B30289013B12F0DA
:10DC1000020F9BB2F8D0818140F2E93300E0FBB102
:10DC20000289013B12F0010F9BB2F8D08089C0B28B
:10DC300083061AD57068C3E7FDF77AFA70682AE799
:10DC4000FDF776FA70685DE7FDF772FA706874E7C1
:10DC5000FDF76EFA706839E7FDF76AFA7068C7E792
:10DC6000FDF766FAC0B28306E4D4B36813B11A684C
:10DC70009B88138300233B70BDE8F087FDF758FABB
:10DC8000706894E6FDF754FA706897E7FDF750FA6C
:10DC900070687AE7FDF74CFA7068D9E6FDF748FA44
:10DCA0007068BAE6FDF744FA70689BE638B51E4D19
:10DCB00040F2E9326B6800E05AB31C89013A14F073
:10DCC000020F92B2F8D080B2988140F2E93200E0BF
:10DCD000FAB11889013A10F0010F92B2F8D09A897E
:10DCE00040F2E93200E0CAB11889013A10F0020F9F
:10DCF00092B2F8D089B2998140F2E93200E06AB17B
:10DD00001989013A11F0010F92B2F8D09889C0B286
:10DD100038BD1846FDF70CFA6B68E1E71846FDF7C9
:10DD200007FAC0B238BD00BFCC8700202DE9F84FFC
:10DD3000DFF8B493D9F8083013B11A689B8853837D
:10DD4000D9F8040040F2E93302E0002B00F0F6813C
:10DD50000289013B12F0020F9BB2F6D005238381AA
:10DD600040F2E93302E0002B00F0E8810289013B38
:10DD700012F0010F9BB2F6D0838940F2E93302E042
:10DD8000002B00F0D6810289013B12F0020F9BB2FA
:10DD9000F6D00023838140F2E93302E0002B00F04B
:10DDA000C8810289013B12F0010F9BB2F6D0838932
:10DDB00040F2E93302E0002B00F0B6810289013B1A
:10DDC00012F0020F9BB2F6D00623838140F2E933B2
:10DDD00002E0002B00F0A8810289013B12F0010F44
:10DDE0009BB2F6D0838940F2E93302E0002B00F0C9
:10DDF00098810289013B12F0020F9BB2F6D00023FA
:10DE0000838140F2E93302E0002B00F08A8102892D
:10DE1000013B12F0010F9BB2F6D08389DFF8CC8270
:10DE2000AE4F98F82C41042044F00101FFF73EFF6B
:10DE30003B88002B4BD008F5987BA94E5D464FF0F0
:10DE4000200A072416F8011FD9F80400FF2940F220
:10DE5000E93303D108E1002B00F032810289013B54
:10DE600012F0020F9BB2F6D0848140F2E93302E057
:10DE7000002B00F025810289013B12F0010F9BB2BB
:10DE8000F6D0838940F2E93302E0002B00F01581DF
:10DE90000289013B12F0020F9BB2F6D089B2818158
:10DEA00040F2E93302E0002B00F007810289013BD8
:10DEB00012F0010F9BB2F6D08389337805F8013B4D
:10DEC0003A88A5EB0B039A42BCDC98F82C41FF2161
:10DED0000720FFF7EBFE21460420FFF7E7FE3B8813
:10DEE000002B00F0B8807F4C0021FF26072503E0BF
:10DEF00001318B4240F3AF8014F8012BFF2AF7D198
:10DF00004FEA2128D9F8040040F2E93302E0002B5F
:10DF100000F002810289013B12F0020F9BB2F6D0A1
:10DF20000523838140F2E93302E0002B00F0F48006
:10DF30000289013B12F0010F9BB2F6D0838940F2B7
:10DF4000E93302E0002B00F0E2800289013B12F08D
:10DF5000020F9BB2F6D01FFA88F8A0F80C8040F2AE
:10DF6000E93302E0002B00F0D2800289013B12F07D
:10DF7000010F9BB2F6D083895FFA81F840F2E93352
:10DF800002E0002B00F0BE800289013B12F0020F7C
:10DF90009BB2F6D00623838140F2E93302E0002BE6
:10DFA00000F0B0800289013B12F0010F9BB2F6D065
:10DFB000838940F2E93302E0002B00F09E80028961
:10DFC000013B12F0020F9BB2F6D01FFA88F8A0F8BE
:10DFD0000C8040F2E93302E0002B00F08E800289D1
:10DFE000013B12F0010F9BB2F6D0838940F2E93376
:10DFF00001E0002B7CD00289013B12F0020F9BB2A2
:10E00000F7D0858140F2E93301E0002B70D002891E
:10E01000013B12F0010F9BB2F7D0838940F2E93344
:10E0200001E0002B56D00289013B12F0020F9BB297
:10E03000F7D0868140F2E93301E0002B4AD0028913
:10E04000013B12F0010F9BB2F7D083893B8801316D
:10E050008B423FF751AFD9F8083013B11A689B884B
:10E060001383BDE8F88F83B30289013B12F0020FDE
:10E070009BB2F8D0848140F2E93300E02BB30289EF
:10E08000013B12F0010F9BB2F8D0838940F2E933D3
:10E0900000E093B10289013B12F0020F9BB2F8D06D
:10E0A000A0F80CA040F2E93300E033B10289013B53
:10E0B00012F0010F9BB2F8D0FEE6FDF739F8FCE64E
:10E0C000FDF736F8D9F80400DCE6FDF731F8D9F8A9
:10E0D0000400DBE7FDF72CF83B8809E7EC0600209D
:10E0E000675C0020685C0020CC870020A826002008
:10E0F000FDF71EF8D9F8040090E7FDF719F8D9F8F4
:10E10000040073E7FDF714F8D9F8040051E7FDF7B0
:10E110000FF8D9F804002FE7FDF70AF8D9F8040042
:10E120000DE7FDF705F879E6FDF702F8D9F80400E8
:10E1300059E6FCF7FDFFD9F8040039E6FCF7F8FFD3
:10E14000D9F8040019E600BFF8B5724EB36813B1F0
:10E150001A6899885183704A70681278012A00F011
:10E16000CA80C0F08480022A44D06C4D2A7812F014
:10E17000400F0CBF4FF4C3724FF4F072684C228012
:10E1800013B11A689B8853831021012740F2E933A9
:10E1900001E0002B62D00289013B12F0020F9BB21A
:10E1A000F7D08BB2838140F2E93301E0002B55D0E8
:10E1B0000289013B12F0010F9BB2F7D0838940F234
:10E1C000E93300E0E3B10289013B12F0020F9BB298
:10E1D000F8D0878140F2E93300E08BB10289013B3E
:10E1E00012F0010F9BB2F8D00131202983890CD0A5
:10E1F0007068CBE7494D08222A704FF4C372BDE71F
:10E20000FCF796FF01312029F2D1B3681BB11A68DF
:10E210009B881383538329780020FFF747FD414BE8
:10E2200002201978FFF742FD3F4B03201978FFF7D2
:10E230003DFD3E4B93F82C1104200143FFF736FDC2
:10E24000B36813B11A689B881383394D2288394803
:10E25000002138F0E3FA2B7823B9F8BDFCF768FF0A
:10E260007068ACE7FFF762FD00232B70F8BD40F249
:10E27000E93301E0002B48D00289013B12F0020F84
:10E280009BB2F7D0A023838140F2E93301E0002B59
:10E290003BD00289013B12F0010F9BB2F7D083897A
:10E2A00040F2E93300E063B30289013B12F0020F50
:10E2B0009BB2F8D00023838140F2E93300E003B33E
:10E2C0000289013B12F0010F9BB2F8D08389D8B2CA
:10E2D00000F00603022B114D08D000F00503012BBE
:10E2E00004D14822D6E901032A7007E00822D6E9C2
:10E2F00001032A7081E7094D48222A704FF4F07219
:10E300003CE7FCF715FFC0B2E2E7FCF711FF7068CD
:10E31000C6E700BFCC87002018880020E008002056
:10E32000EC0600201F88002020880020A82600205E
:10E3300000000020D827002073498B682DE9F041A8
:10E3400013B11A689B885383486840F2E93301E0AF
:10E35000002B4AD00289013B12F0020F9BB2F7D08A
:10E360008023838140F2E93301E0002B3DD0028914
:10E37000013B12F0010F9BB2F7D0838940F2E933E1
:10E3800001E0002B2DD00289013B12F0020F9BB25D
:10E39000F7D00023838140F2E93300E00BB3028918
:10E3A000013B12F0010F9BB2F8D08089C0B28B689C
:10E3B00013B11A689C881483544C554D22782E68EA
:10E3C00082420BD1534A127832B9534FD7F81023F7
:10E3D000B21AB2F57A7F0CD8BDE8F081BDE8F04101
:10E3E000B2E6FCF7A5FEC0B2E1E7FCF7A1FE486883
:10E3F000C4E713B11A689B885383486840F2E93335
:10E4000001E0002B78D00289013B12F0020F9BB291
:10E41000F7D0A023838140F2E93301E0002B6BD0D9
:10E420000289013B12F0010F9BB2F7D0838940F2C1
:10E43000E93301E0002B5BD00289013B12F0020FAF
:10E440009BB2F7D00023838140F2E93301E0002B37
:10E450004ED00289013B12F0010F9BB2F7D08089A8
:10E46000C0B28B6813B11A689B881383DFF8B08041
:10E4700098F80030182B0FD12378284A03F0400376
:10E48000002B00F007010CBF4FF00D0C4FF0100CEB
:10E4900013805180A2F806C0410706D50023C7F8B3
:10E4A0001433C7F81063BDE8F08100F005000128BF
:10E4B0001AD00028F5D123785B06F2D5D7F81423BB
:10E4C0002B68EAB19B1A642BEBD9FFF73DFE98F855
:10E4D0000030182BE5D1B7F81833104A01339BB23E
:10E4E000A7F818339380DCE723785A06E6D5D8E7F7
:10E4F000FCF71EFEC0B2B4E7FCF71AFE486896E7C8
:10E50000C7F81433CDE700BFCC870020E008002017
:10E51000108A002018880020A826002010880020DB
:10E520000D8800202DE9F84F424A434E0123137015
:10E53000FFF702FFB6F87435404ADFF808E1B2F899
:10E54000008003F1640C1FFA8CFC00214FF0050BD6
:10E550004FF0060A4FF0070901E0634567D0F41851
:10E560001EF8030094F83021824203F1010501F105
:10E57000050211D0B718721884F830011C0A82F80D
:10E580001CB382F81EA382F81F3382F8209382F80E
:10E590001D43063187F81C03ABB24345DDD300238E
:10E5A000A6F8743521B9234A00231370BDE8F88F0B
:10E5B000234EB76817B13B68BA885A837068DFF892
:10E5C00088C0838901394FF47A734FF6FF74BCF128
:10E5D000000F2AD09CF800500CF1010C01E0A3427E
:10E5E0001FD00289013B92079BB2F8D5ABB2838161
:10E5F0004FF47A7302E0ABB2A34212D00289D20781
:10E6000003F1FF35F7D5013982894A1CDFD1002F8C
:10E61000C9D03B68BA881A83064A00231370BDE844
:10E62000F88FFCF785FDB768F1E7FF25D9E7A6F875
:10E630007435B7E755700020A8260020EC060020AE
:10E64000CC870020685C0020C42900200F4B10B448
:10E650001C889CB10E4B0F4A187892F830118842F2
:10E6600010D11C4402F59872013305E013F8011B28
:10E6700012F8010F884205D1A342F7D101205DF8BD
:10E68000044B704700205DF8044B7047EC060020F7
:10E69000685C0020A82600201378C3B130B41E2483
:10E6A0000B4D14FB01012944801A84181D2C07DC32
:10E6B00001F8013B12F8013F002BF6D130BC704746
:10E6C00012F8013F0131002BEFD130BC7047704789
:10E6D000685C002038B5264CC1F10301A36841EA0B
:10E6E0008005EDB213B11A689B885383ADB2102137
:10E6F000606840F2E93301E0002B31D00289013B30
:10E7000012F0020F9BB2F7D08BB2838140F2E93353
:10E7100000E02BB30289013B12F0010F9BB2F8D04D
:10E72000838940F2E93300E0F3B10289013B12F042
:10E73000020F9BB2F8D0858140F2E93300E09BB133
:10E740000289013B12F0010F9BB2F8D0838901319D
:10E750002029CDD1A36813B11A689B88138338BDD3
:10E76000FCF7E6FC6068DCE7FCF7E2FCEFE700BFE3
:10E77000CC87002010B5274B93F82C4100283FD1BF
:10E7800004F0F704244983F82C418B6813B11A680C
:10E790009B885383486840F2E93301E0002B35D071
:10E7A0000289013B12F0020F9BB2F7D00423838150
:10E7B00040F2E93300E04BB30289013B12F0010F54
:10E7C0009BB2F8D0838940F2E93300E0DBB10289E3
:10E7D000013B12F0020F9BB2F8D0A4B2848140F248
:10E7E000E93300E07BB10289013B12F0010F9BB2DB
:10E7F000F8D083898B6813B11A689B88138310BD86
:10E8000044F00804BEE7FCF793FCF3E7FCF790FC48
:10E810004868D8E7A8260020CC870020144B9842EF
:10E8200023D003F5806398421FD0038823F0400370
:10E830001B041B0C0380038823F038031B041B0CF0
:10E8400059B141F48071002991FAA1F1B1FA81F135
:10E8500008BF4FF0FF310139C900194389B2018067
:10E86000038843F04003038070474908DDE700BF99
:10E8700000380040F0B587B00023604A0093019350
:10E88000136843F48033136003E0009BB3F5A04F9B
:10E8900009D0136803F400330193009B0133009304
:10E8A000019B002BF1D0554B1B6813F4003318BFAC
:10E8B00001230193019B012B63D0514D4F4B514AD2
:10E8C000EA605149586F514A0860AA605E6B504C2B
:10E8D000504F514A514826F080065E635E6F46F005
:10E8E00080765E67196B0C431C63596B5963196C16
:10E8F00039431964596C06AC0A4348F2FF715A64F3
:10E9000044F8101D0123002621468DF80F304FF6E4
:10E91000FF778DF80C608DF80D608DF80E6014F0A7
:10E92000E9F821463E48029714F0E4F821463D48B4
:10E93000029714F0DFF821463B4814F0DBF821463B
:10E940003A4814F0D7F8204614F0D8F9384B394C2F
:10E950001B68029A38483949A4FB03439B09A0FB72
:10E960000202013B920CB3F1807F0A6007D2344A65
:10E97000F0200721536085F823009660116007B0EE
:10E98000F0BD1E4B2F4C1A6C2F4942F080521A6476
:10E99000206840F44040D1E90152C968206098687D
:10E9A000986098689860120642EA8512986842F466
:10E9B0008002490842F00802013942EA014240F46B
:10E9C000805098605A601A6842F080721A601A6823
:10E9D0009201FCD51D49094A40F20270086099680D
:10E9E00021F003019960996841F0020199609368F0
:10E9F00003F00C03082BFAD15FE700BF0038024098
:10EA000000ED00E00005FA0568B2002000000008F3
:10EA10001F906700FFC9FE36335F07000000024009
:10EA20000004024000080240000C024000100240B6
:10EA300084A50020D34D621083DE1B43148A00207E
:10EA400010E000E00070004000000020003C0240A8
:10EA5000074A08B51168074B994208D1064B0020B8
:10EA60001968106081F308885B689847FEE708BD65
:10EA7000DCBF0020EFBEADDE0000FF1F08B5054B78
:10EA80001B6803B19847044B044A1A6072B636F00B
:10EA9000A3FA00BF68310020DCBF0020EFBEADDE6E
:10EAA0002DE9F04FA84B1B78232B8DB000F0AE81E1
:10EAB000A64B1D78002D52D1A54BA64C93F800B063
:10EAC000DFF8C892DFF8C8A20BF0010B04F5257738
:10EAD00054F80B0C38B1FBF761FF002840F00581BA
:10EAE00014F8033C3BB9DC34BC4205F10105EFD11D
:10EAF0000DB0BDE8F08FDAF8002054F8071C521A68
:10EB0000632AF0D9012B00F03A83022BEBD1924B10
:10EB100089F881059148DA78914E0660914854F859
:10EB20000B3C91490360003218BF012287480A70EC
:10EB3000C9F8483001218D4AC9F87C35402301705D
:10EB4000C9F8782589F88035894821F0F3F9894892
:10EB500020F028F94FF480500FF09CFBC3E77F4B67
:10EB600018680028C4D0FCF72FFCDFF8F8A1824F0A
:10EB7000DAF80000FBF712FF0028B9D0DAF800003D
:10EB8000DFF81092FBF702FF0928D9F8006019D0CE
:10EB90003F2817D0002E6BD1042800F0EC820C28FF
:10EBA00000F09C807F28E3D0A0F12003DBB25E2B35
:10EBB000DED82028DCD0731CB855C9F8003020F00E
:10EBC000E9F8D5E7002E67D16C4B354603F5387868
:10EBD000002D46D010334345FAD1DFF8BCB1286888
:10EBE000DBF80020845D935D9C42304402EB06011B
:10EBF00040F06E82741E3C44324613B9FD2A40F246
:10EC0000FD8004F8013F0132C9F8002010F8013FEF
:10EC100011F801CF9C45F0D00AB1AB4513D058484C
:10EC200020F0C0F8AB4508D355F8100B20F0BAF827
:10EC3000092020F0AFF85D45F6D94E4820F0B2F833
:10EC4000D9F800200026964292D2741E3C4414F853
:10EC5000010F20F09FF8D9F8003001369E42F6D31C
:10EC600086E703F1100242451D46B6D01346AFE7D2
:10EC70000C2833D00A2800F091800D2800F08E80F7
:10EC80007F2800F0FD81FF2E3FF672AFA0F1200338
:10EC9000DBB25E2B8FD96BE7384C4FF0000B04F5DD
:10ECA00038785D4602E0103444450DD03246216884
:10ECB0003846FEF781FB0028F5D1A346002DF2D19E
:10ECC000254610344445F1D1002D88D1BBF1000F09
:10ECD0003FF44EAF2A4820F065F8A5E7294820F018
:10ECE00061F8244820F05EF842E7DAF8003044F892
:10ECF000073C254B4FF0DC08002608FB0538A4F143
:10ED00000B0304F8036C009354F80B0CFBF746FE5E
:10ED100000283FF4E8AE54F80B0CFBF737FE14F86C
:10ED2000021C4B1E02460B2B00F29781DFE813F00A
:10ED300088017B016D01450132011601E900CC001B
:10ED4000BF009800800078000D880020DC53002070
:10ED5000DE51002023990020BC9B00202832002097
:10ED6000202C00206832002068820020DD8100080D
:10ED700044A2040810A204086E320020146D040896
:10ED800008A2040818A2040818990020A826002048
:10ED9000108A002070330020E46F040820F09BF8F4
:10EDA0002321CF4837F051FD002800F05381C31BC9
:10EDB000C9F800309BB15A1EB95C202940F00B8283
:10EDC000023B3B444AB113F80119202902F1FF30FC
:10EDD00040F063810246002AF5D1C9F800204FF4C3
:10EDE00080720021384637F019FDBE4B1B78002B8E
:10EDF0003FF47EAEBC481FF0D5FFB9E6511C202081
:10EE0000B854C9F800107B540A4606E7B74BB84A15
:10EE10001B6800215B1A18BF01235380118047E64D
:10EE200094F8CE30934200F09E8004F8026C6BE7B9
:10EE3000114694F8CE00FEF70DF8D4F8C53084F8EA
:10EE4000CE0008EB03010133C4F8C530CA72D4F810
:10EE5000C92093427FF458AF0C2304F8023C53E7D7
:10EE6000D4F8C53008EB03010133C4F8C530CA72C9
:10EE700094F8CE0001931146FDF7ECFF019B84F856
:10EE8000CE00052B7FF440AFB4F80330B4F8011086
:10EE90002278C4F8C560C4F8C930A4F8C11084F859
:10EEA000C320002BD8D00B2304F8023C2CE794F8A5
:10EEB000CD3094F8CE105340914284F8CD30B4D187
:10EEC000062304F8023C1FE7114694F8CE00FDF734
:10EED000C1FFD4F8C53094F8CD1084F8CE0008EB0B
:10EEE000030051400133C4F8C53084F8CD10C2721C
:10EEF000D4F8C92093427FF407AF092304F8023CF9
:10EF000002E7D4F8C53008EB03010133C4F8C5307B
:10EF1000CA7294F8CDC094F8CE00019382EA0C0C2A
:10EF2000114684F8CDC0FDF795FF019B84F8CE0013
:10EF3000072B7FF4E9AEB4F80530B4F80310A278DB
:10EF4000C4F8C560C4F8C930A4F8C11084F8C3205F
:10EF5000002BD2D0082304F8023CD5E694F8CD303B
:10EF600093427FF462AF0D2304F8023C14F801CC05
:10EF7000BCF1000F00F0C480BCF1010F00F00C8167
:10EF8000002304F8023CDC34BC4205F101057FF4A7
:10EF90009FADADE5D4F8C53008EB03010133C4F8EB
:10EFA000C530CA7294F8CD00D4F8C91042408B42E3
:10EFB00084F8CD207FF4A8AE82E7D4F8C53008EB02
:10EFC00003010133C4F8C530CA7294F8CD10022B86
:10EFD00082EA010284F8CD207FF496AE2378C02B1C
:10EFE0003FF623AF6278FF2A00F0F780C4F8C930FB
:10EFF000A4F8C12084F8C360C4F8C560002B3FF4B6
:10F000005FAF052304F8023C7EE63C2A7FF40DAF97
:10F0100002220A23C4F8C56084F8CE6084F8C420B4
:10F0200004F8023C70E63C2A7FF4FFAE0423C4F8E7
:10F03000C56084F8CD6084F8CE6004F8023C63E6D5
:10F040004D2A00F09480582A7FF4EFAE032304F891
:10F05000023C59E6D9F80030ACE6242A3AD0BBF19C
:10F06000000F02D00D2981D04EE6232A11D0214B6A
:10F0700093F82A30934204BF012304F8033CF1E7DC
:10F08000013E00231C48C9F80060BB551FF08AFEF2
:10F090006EE5022304F8033CE4E7C9F80020174CAE
:10F0A000002304F53878BB5403E01034444500F0E5
:10F0B0009E80216838460AF051FE0028F5D044456C
:10F0C00080F09580E36898470023C9F8003086E611
:10F0D0003246A1E5012384F8C46004F8023C13E63B
:10F0E0006E320020DC53002010A2040814480020D7
:10F0F0001088002034BB002040A20408146D0408CE
:10F100003D4BB4F8C180ADF82CC00FCB0DF1300EE3
:10F1100004AE86E80F00D4F8C9104EF824CD60186C
:10F1200094F8C33009904FF0010C7246314608A89C
:10F130000894ADF828808DF82A308DF82EC00FF095
:10F14000B1F8F0B9039E002304F8023C002E3FF40E
:10F15000CAAC54F80B0C2AF01DFDDC3454F8E70C53
:10F16000B047BC4205F101057FF4B2ACC0E4022314
:10F1700004F8023CC8E5214806F0FAFCB8E4FFF7C1
:10F180007DFC049A1E4B05923146009894F8C420E9
:10F1900004932AF005FCD5E7D4F8C930B4F8C120AF
:10F1A0000894234409936E2A4FF00003ADF82E30E3
:10F1B000CDF82A30ADF828207FF4E2AE08A8FEF79B
:10F1C00037FB08A8FEF728FB08A8FEF725FB08A8D0
:10F1D000FEF722FBD4E61A4661E7052B7FF625AE43
:10F1E0000122072384F8C42004F8023C8CE505487A
:10F1F0001FF0D8FD68E700BFC86904086E32002020
:10F20000DCBE002024A204082DE9F04F90F8653000
:10F2100085B00546002B40F0FF83AB4E96F8C43511
:10F220006869002B00F09680A84B984200F0E583B7
:10F2300003F58063984200F0E083038823F04003E5
:10F240001B041B0C0380038823F038031B041B0CD6
:10F25000382213430380038843F04003038095F86A
:10F260005F30032B74D895F86210012900F04786AF
:10F27000A1F10201B1FA81F14909AB6913B11A6830
:10F280009B88538340F2E93304E0013B9BB2002B9F
:10F2900000F0CB8702899207F7D51A23838140F2C9
:10F2A000E93304E0013B9BB2002B00F0BE870289EA
:10F2B000D707F7D5838940F2E93304E0013B9BB2DD
:10F2C000002B00F0AE8702899607F7D5818140F2C6
:10F2D000E93304E0013B9BB2002B00F0A2870289D6
:10F2E000D407F7D58389AB6913B11A689B88138358
:10F2F000FAF7ACFF0446FAF7A9FF8442FBD068692D
:10F30000724B984200F0148503F58063984200F038
:10F310000F85038823F040031B041B0C0380038824
:10F3200023F038031B041B0C0822134303800388BB
:10F3300043F0400303802B7C022B00F0A384B5F93B
:10F3400052305BB2013300F0258505B0BDE8F08F87
:10F35000002192E75D4B984200F06C8703F58063D3
:10F36000984200F06787038823F040031B041B0CBE
:10F370000380038823F038031B041B0C4FF48072B6
:10F3800042F48072002A92FAA2F2B2FA82F208BF24
:10F390004FF0FF32013A43EAC2039BB20380028876
:10F3A000AB6942F04002028013B11A689B88538314
:10F3B00040F2E93304E0013B9BB2002B00F04887A8
:10F3C00002899707F7D56B23838140F2E93304E084
:10F3D000013B9BB2002B00F03B870289D407F7D595
:10F3E000838940F2E93304E0013B9BB2002B00F03B
:10F3F0003D8702899107F7D58023838140F2E93365
:10F4000004E0013B9BB2002B00F030870289D20759
:10F41000F7D58389AB6913B11A689B8813832C4C89
:10F42000DFF8B8A02B4FDFF8B890DFF8B8804FF0C6
:10F43000960BFAF70BFF4FF47A7C274B5B68C3F30C
:10F440000803002B40F06186EFF31183002B40F09E
:10F450005C862368B96822689342FAD1D8F8002004
:10F460009142F6D8DAF800E00CFB0EF2521AB2FB29
:10F47000FEF20CFB03231B1AB3F57A7FDDD3BBF13D
:10F48000010BD6D1AB6913B11A689B8853836869A5
:10F4900040F2E93304E0013B9BB2002B00F0DD8633
:10F4A00002899207F7D56823838140F2E93304E0AB
:10F4B000013B9BB2002B00F0D0860289D707F7D51D
:10F4C000838940F2E93314E0A82600200038004088
:10F4D000108A002010E000E000ED00E0148A002017
:10F4E0000C8A0020188A0020013B9BB2002B00F000
:10F4F000B98602899107F7D50323838140F2E93366
:10F5000004E0013B9BB2002B00F0AC860289D207DD
:10F51000F7D58389AB6913B11A689B881383904F21
:10F52000DFF84492DFF844824FF0960BFAF78EFE34
:10F530004FF47A7C8B4B5B68C3F30803002B40F0DD
:10F540000686EFF31183002B40F001862368B9682B
:10F5500022689342FAD1D8F800209142F6D8DAF81E
:10F5600000E00CFB0EF2521AB2FBFEF20CFB03237E
:10F570001B1AB3F57A7FDDD3BBF1010BD6D1AB6992
:10F5800013B11A689B885383686940F2E93304E039
:10F59000013B9BB2002B00F0248602899207F7D52D
:10F5A0006B23838140F2E93304E0013B9BB2002BE3
:10F5B00000F017860289D707F7D5838940F2E9332F
:10F5C00004E0013B9BB2002B00F0108602899407F7
:10F5D000F7D50323838140F2E93304E0013B9BB27A
:10F5E000002B00F003860289D107F7D58389AB6928
:10F5F00013B11A689B8813830F20FAF779FEAB6961
:10F6000013B11A689B885383686940F2E93304E0B8
:10F61000013B9BB2002B00F0ED8502899207F7D5E4
:10F620006A23838140F2E93304E0013B9BB2002B63
:10F6300000F0E0850289D707F7D5838940F2E933E6
:10F6400004E0013B9BB2002B00F0D98502899407AE
:10F65000F7D51023838140F2E93304E0013B9BB2EC
:10F66000002B00F0CC850289D107F7D58389AB69DF
:10F6700013B11A689B8813830F20FAF739FEAB6920
:10F6800013B11A689B885383686940F2E93304E038
:10F69000013B9BB2002B00F0B68502899207F7D59B
:10F6A0006C23838140F2E93304E0013B9BB2002BE1
:10F6B00000F0A9850289D707F7D5838940F2E9339D
:10F6C00004E0013B9BB2002B00F0A2850289940765
:10F6D000F7D50023838140F2E93304E0013B9BB27C
:10F6E000002B00F095850289D107F7D58389AB6996
:10F6F00013B11A689B8813830F20FAF7F9FDAB69E1
:10F7000095F8641013B11A689B885383686940F2B6
:10F71000E93304E0013B9BB2002B00F07D850289B8
:10F720009207F7D51923838140F2E93304E0013BC6
:10F730009BB2002B00F070850289D707F7D583892B
:10F7400040F2E93304E0013B9BB2002B00F021853D
:10F7500002899407F7D589B2818140F2E9330CE040
:10F7600010E000E000ED00E00C8A0020188A002084
:10F77000013B9BB2002B00F00C850289D107F7D525
:10F780008389AB6913B11A689B8813830F20FAF73A
:10F79000AFFDAB6913B11A689B885383686940F267
:10F7A000E93304E0013B9BB2002B00F0F6840289B0
:10F7B0009207F7D51B23838140F2E93304E0013B34
:10F7C0009BB2002B00F0E9840289D707F7D5838923
:10F7D00040F2E93304E0013B9BB2002B00F0E284ED
:10F7E00002899407F7D51823838140F2E93304E0B6
:10F7F000013B9BB2002B00F0D5840289D107F7D5DD
:10F800008389AB6913B11A689B8813830F20FAF7B9
:10F810006FFDAB6913B11A689B885383686940F226
:10F82000E93304E0013B9BB2002B00F0BF84028966
:10F830009207F7D51C23838140F2E93304E0013BB2
:10F840009BB2002B00F0B2840289D707F7D58389D9
:10F8500040F2E93304E0013B9BB2002B00F0AB84A3
:10F8600002899407F7D51823838140F2E93304E035
:10F87000013B9BB2002B00F09E840289D107F7D593
:10F880008389AB6913B11A689B8813830F20FAF739
:10F890002FFDAB6913B11A689B885383686940F2E6
:10F8A000E93304E0013B9BB2002B00F0888402891D
:10F8B0009207F7D53723838140F2E93304E0013B17
:10F8C0009BB2002B00F07B840289D707F7D5838990
:10F8D00040F2E93304E0013B9BB2002B00F074845A
:10F8E00002899407F7D51023838140F2E93304E0BD
:10F8F000013B9BB2002B00F067840289D107F7D54A
:10F900008389AB6913B11A689B8813830F20FAF7B8
:10F91000EFFCAB6913B11A689B885383686940F2A6
:10F92000E93304E0013B9BB2002B00F051840289D3
:10F930009207F7D53823838140F2E93304E0013B95
:10F940009BB2002B00F044840289D707F7D5838946
:10F9500040F2E93304E0013B9BB2002B00F03D8410
:10F9600002899407F7D50123838140F2E93304E04B
:10F97000013B9BB2002B00F030840289D107F7D500
:10F980008389AB6913B11A689B8813830F20FAF738
:10F99000AFFC69691F4B994200F06C8403F58063EA
:10F9A000994200F067840B8823F040031B041B0C72
:10F9B0000B800B8823F038031B041B0C042242F439
:10F9C0008072002A92FAA2F2B2FA82F208BF4FF0D5
:10F9D000FF32013A43EAC2039BB20B800B8843F02B
:10F9E00040030B800120FAF783FC0123686986F845
:10F9F000C435084B98427FF41BAC038823F04003C6
:10FA00001B041B0C0380038823F038031B041B0C0E
:10FA100030221EE4003800401E09013E032E03F090
:10FA20000F0300F268829B4A32F8160040FA03F294
:10FA3000D40740F16082012404FA03F3013B18402B
:10FA400035F00CF9944B954A9B5D184412EBC007B6
:10FA500000F0518220210023B971FB7152F830303F
:10FA60008F4A03F13F4101F57E01890A505C00F0A5
:10FA70001F024009032804FA02F200F0CE82042893
:10FA800000F0C682022803D18648446C22434264B7
:10FA9000BA88D0070BD5186820F0030018601868E2
:10FAA0001860D86820F00300D860D868D86096073E
:10FAB0000BD5186820F00C00186018681860D8681A
:10FAC00020F00C00D860D868D86054070BD51868AF
:10FAD00020F03000186018681860D86820F03000F6
:10FAE000D860D868D86010070BD5186820F0C0001F
:10FAF000186018681860D86820F0C000D860D8680E
:10FB0000D860D6060BD5186820F4407018601868C5
:10FB10001860D86820F44070D860D868D86094061F
:10FB20000BD5186820F44060186018681860D86811
:10FB300020F44060D860D868D86050060BD51868AB
:10FB400020F44050186018681860D86820F44050BD
:10FB5000D860D868D86016060BD5186820F44040E5
:10FB6000186018681860D86820F44040D860D868D9
:10FB7000D860D4050BD5186820F440301860186898
:10FB80001860D86820F44030D860D868D8609005F4
:10FB90000BD5186820F44020186018681860D868E1
:10FBA00020F44020D860D868D86056050BD5186876
:10FBB00020F44010186018681860D86820F44010CD
:10FBC000D860D868D86014050BD5186820F44000B8
:10FBD000186018681860D86820F44000D860D868A9
:10FBE000D860D0040BD5186820F0407018601868F1
:10FBF0001860D86820F04070D860D868D860960443
:10FC00000BD5186820F04060186018681860D86834
:10FC100020F04060D860D868D86054040BD51868CC
:10FC200020F04050186018681860D86820F04050E4
:10FC3000D860D868D86010040BD5186820F0404010
:10FC4000186018681860D86820F04040D860D868FC
:10FC5000D860B2FA82F0144BEB60C0F11F00431C75
:10FC600040F0F081114EB2FA82F3C3F11F0301227A
:10FC700012FA03F33FF4D2AA0D490A6813430B604A
:10FC8000FFF7CCBAAB6913B11A689B88538340F273
:10FC9000E93314E0F49A0408FC9A0408248800204C
:10FCA0008C99040800380240E9860008A826002044
:10FCB000003C0140013B9BB2002B00F0A581028972
:10FCC0009107F7D5C323838140F2E93304E0013B78
:10FCD0009BB2002B00F098810289D207F7D5838967
:10FCE000838903899B074FF0050402AA4FF47A71B8
:10FCF0004FF0FF074FF6FF7606D44B1E9BB229B399
:10FD0000194603899B07F8D587814FF47A7303E07E
:10FD1000013B9BB2B34219D00189C907F8D581894B
:10FD200089B20AB11170013294B1013C1946E8E779
:10FD3000038823F040031B041B0C0380038823F07B
:10FD400038031B041B0C0022FFF7EFBAFBF7F0F996
:10FD5000AB6913B11A689B8813839DF80A609DF8FC
:10FD60000B309DF808409DF809109DF80C009DF897
:10FD70000D2043EA06231BB2A5F852305BB241EADC
:10FD8000042142EA00220133A5F85010A5F85420BE
:10FD90007FF4DBAA95F9503001337FF4D6AA0A2309
:10FDA000A04CDFF898A2A04FA04DA14E01932FF0D8
:10FDB000B5FE4FF4FA73DFF888E200934FF01008B5
:10FDC0007B68C3F30803002B40F0DA80EFF3118364
:10FDD000002B40F0D5802068AA6823689842FAD1A9
:10FDE00033689A42F7D8DAF800C04FF47A7101FB11
:10FDF0000CF39B1AB3FBFCF301FB00304FF47A7C4D
:10FE00004FF001097B68C3F30803002B40F0998091
:10FE1000EFF31183002B40F094802368A9682268D7
:10FE20009342FAD132689142F7D8DAF800200CFBFD
:10FE300002FBABEB0101B1FBF2F10CFB03131B1A4C
:10FE4000B3F57A7FDED3009B013B0093B8D1072046
:10FE50002FF0B8FC4FF47A73DFF8E4E100934FF031
:10FE600010087B68C3F30803002B40F0AB80EFF36E
:10FE70001183002B40F0A6802068AA68236898426E
:10FE8000FAD133689A42F7D8DAF800C04FF47A71A1
:10FE900001FB0CF39B1AB3FBFCF301FB00304FF4A6
:10FEA0007A7C4FF001097B68C3F3080353BBEFF37F
:10FEB00011833BBB2368A96822689342FAD1326858
:10FEC0009142F7D8DAF800200CFB02FBABEB010102
:10FED000B1FBF2F10CFB03131B1AB3F57A7FE2D3EB
:10FEE000009B013B0093BCD1019B013B01937FF43C
:10FEF0005EAFFEF7C3FD4F4BEB60FFF78EB90721F6
:10FF0000FFF7BBB9EFF3118188F31288D5F808B079
:10FF10002B68DB0344BFCEF80090D5F808B0236807
:10FF2000DEF80020C9B281F31188DAF8001013441A
:10FF30000CFB01F2A2EB0B02B2FBF1F20CFB032370
:10FF4000CAE7EFF3118188F31288D5F808B02B685F
:10FF5000DB0344BFCEF80090D5F808B02368DEF884
:10FF60000020C9B281F31188DAF8001013440CFBA9
:10FF700001F2A2EB0B02B2FBF1F20CFB03235EE7F2
:10FF8000EFF3118388F31288D5F808C02A68D203EA
:10FF900004D50122CEF80020D5F808C02068DEF88C
:10FFA0000090DBB283F31188DAF800104FF47A7214
:10FFB000484402FB01F3A3EB0C03B3FBF1F302FB98
:10FFC00000301BE7EFF3118388F31288D5F808C0DF
:10FFD0002A68D20304D50122CEF80020D5F808C043
:10FFE0002068DEF80090DBB283F31188DAF80010A5
:10FFF0004FF47A72484402FB01F3A3EB0C03B3FB0A
:020000040801F1
:10000000F1F302FB00304AE7FBF792F8686967E614
:100010000948046B224302633AE50748046C224313
:10002000026435E5108A002000ED00E010E000E0F9
:10003000188A0020E986000800380240148A00204F
:100040000C8A0020C3B203F0FC0404F1804404F5E0
:100050009C3403F0030CD4F808E08D4E8D4B4FEA2E
:100060008C0C4FF00F0808FA0CF82EEA080E06EB7D
:10007000800805F10C09C8F84C90C4F808E0D4F8E1
:100080000880DFF818E2C9B201FA0CF14FF0010C58
:1000900041EA08010CFA00F8A160C3F814801C685A
:1000A0006FEA08010C401C605C680C405C601C68D6
:1000B00044EA08041C609C680C409C60DC68704446
:1000C0002140754CD960236890F8E00043EA0803AA
:1000D0003118236091F88C30F02B7FF6C4AD0EEB15
:1000E0000003032293F8F0308DF80830F024002349
:1000F00002A88DF809208DF80BC081F88C408DF88E
:100100000A302FF033F9BA88ADE5EFF311811023EF
:1001100083F31288D7F808E03B68DB0304D501239A
:10012000C9F80030D7F808E02368D9F80020C9B230
:1001300081F31188DAF8001013440CFB01F2A2EBF2
:100140000E02B2FBF1F20CFB0323FFF794B9EFF3BD
:100150001181102383F31288D7F808E03B68DB0392
:1001600004D50123C9F80030D7F808E02368D9F88E
:100170000020C9B281F31188DAF8001013440CFB97
:1001800001F2A2EB0E02B2FBF1F20CFB0323FFF72C
:10019000EFB9FAF7CDFFFFF7F4BAFAF7C9FF6869CC
:1001A000FFF716BBFAF7C4FFFFF72BBBFAF7C0FF48
:1001B0006869FFF74DBBFAF7BBFFFFF762BBFAF7C1
:1001C000B7FF6869FFF784BBFAF7B2FFFFF799BB87
:1001D000FAF7AEFF6869FFF7BBBBFAF7A9FFFFF7B5
:1001E000D0BBFAF7A5FF6869FFF7E8B9FAF7A0FFF7
:1001F000FFF7FDB9FAF79CFF6869FFF71FBAFAF736
:1002000097FFFFF734BAFAF793FF6869FFF756BA1A
:10021000FAF78EFFFFF76BBAFAF78AFF6869FFF704
:100220008FBAFAF785FFFFF75EB8FAF781FF6869C2
:10023000FFF741B8038823F040031B041B0C038025
:10024000038823F038031B041B0C8022FFF798B8A7
:10025000FAF76EFF6869FFF7C4B8FAF769FF6869D3
:10026000FFF72FB9FAF764FFFFF754B9FAF760FF09
:10027000FFF7D0B80B8823F040031B041B0C0B8046
:100280000B8823F038031B041B0C0222FFF797BBDB
:10029000A8260020003C0140083C0140F868040802
:1002A000F8B50468C4F30D0405460E4604B32F6880
:1002B00012F00EFC092840F08980464C236923F493
:1002C00040732361236943F400732361236943F07E
:1002D000010323613E6012F0FBFB2369092823F030
:1002E0000103236172D12B6804332B60002036E0B8
:1002F000394B3A4A93422CD902F58042934227D98E
:1003000002F5804293422BD902F58042934229D9CB
:1003100002F58032934227D902F50032934225D963
:1003200002F50032934223D902F50032934221D9DB
:1003300002F5003293421FD902F5802293421DD963
:10034000B3F1016F1CD305202FF088FDFEF796FB5B
:10035000082412F0BDFB092814D04FF0FF30F8BD7F
:100360001024F6E71824F4E72024F2E72824F0E725
:100370003024EEE73824ECE74024EAE74824E8E7B5
:100380005824E6E7134F3B6923F440733B613B6914
:1003900043F400733B613B6923F0F8033B613B6925
:1003A00043F002031C433C613B6943F480333B61EF
:1003B00012F08EFB3B6923F002033B613B69092885
:1003C00023F0F8033B613FF472AFC6E76FF0010022
:1003D000C5E700BF003C024000400008FF3F0008A6
:1003E000F8B504460D468E180027B542206900D1A5
:1003F000F8BDE368591CE160234415F8012B1A721B
:100400000429F2D118B9A1682046FFF749FFC4E9D1
:100410000370EAE72DE9F04F8DB0FBF767F9DFF8DD
:1004200084915B4FDFF8808107F0BAFC594A5A4B40
:10043000B2F8F820ADF80620A3EB090300934FF0C3
:10044000030A0026CDE90866CDE90A66009BCDF8CF
:1004500018900793D8F81030002BC0F29080012339
:100460008DF82C30F323C8F80C300222BDF806308A
:10047000ADF8083002A906A8FFF7B2FF022202A9D0
:100480004FF6FF70F7F718FF444BBB42834629D263
:100490001C46658823888DF81560C5F30B05C3F3EA
:1004A0000B00A91D1B0B0622ADF81010ADF81200B1
:1004B00004A906A88DF81430FFF792FF58460622CB
:1004C00004A9F7F7F9FE616883462A4606A8FFF7F4
:1004D00087FF616858462A46F7F7EEFE1434BC429F
:1004E0008346D6D3022203A906A8ADF80C60FFF715
:1004F00077FF022203A95846F7F7DEFE40BAC3434E
:10050000022204A906A8ADF81030FFF769FF099888
:1005100028BB0A989DF82C3043B978B1BAF1010A8A
:1005200090D105202FF09AFCFEF7A8FAD8F81030E9
:1005300043F00043C8F810300028EFD199F800309C
:10054000AB2BEED199F80130BE2BEAD1FAF7D8FFE8
:100550000028E6D007F004FC0DB0BDE8F08F08AB32
:10056000C0F104020021184436F058F90A9818B96D
:10057000089906A8FFF794FECDE90960CAE7084B81
:10058000C8F8043003F18833C8F8043067E700BFC7
:10059000C8060008F868040800800008A0010008E8
:1005A0002301674500400008003C024008B5FFF702
:1005B00031FFFBF7A9FA0120BDE808402DF052BF3A
:1005C0002DE9F047D64C2DED028B63682046984705
:1005D000002800F0CF80D34B1B780122042B84F835
:1005E000342000F0CB80B4F9163006EE903AB4F91E
:1005F000183007EE103AB4F91A3007EE903AF8EED8
:10060000E66AB8EEC77AF8EEE77AC4ED0A6A84EDD6
:100610000B7AC4ED0C7AC44B1B88002B60D0C34B03
:1006200094ED0A2AD4ED0B2A94ED0C3A93ED008A4E
:10063000D3ED054A93ED090AD3ED0E3AD3ED120A34
:1006400093ED174A93ED011A93ED065AD3ED0A1A6A
:1006500093ED0F6AD3ED137A93ED187AD3ED045A24
:10066000D3ED0D6AE8EE024AE0EE223AA3EE204A0C
:10067000A1EE025AA1EEA26AA3EE277A93ED038AB5
:10068000D3ED167A93ED020AD3ED0C0A93ED0B1A13
:10069000D3ED151AC4ED0A4A65EEE45AA8EE645A81
:1006A00066EEE36AD3ED144A83ED055A67EEC47A29
:1006B000E0EE025AA0EEE36AE1EE226AA4EE617A6D
:1006C000E3EE247AC3ED065AC4ED0B3A83ED0E6ACD
:1006D000C3ED0F6A83ED177AC3ED187A84ED0C4AE7
:1006E000934EA17F9348944D06F02CFD32886B68A1
:1006F000002A40F09780914A126852075BD4B3F900
:10070000002094ED0B6A94ED0C7A94ED0A5A8C4912
:1007100005EE902AB3F90220B3F9043006EE902AD0
:1007200007EE903AF8EEE55A864B0A68D3ED003AA8
:1007300093ED014AD3ED024AF8EEE66AF8EEE77A65
:1007400075EE655A76EE666A77EE677AC4ED0A5AF8
:1007500034EE266A73EEA55A34EEA77A0132C3ED61
:10076000005AC4ED0B6A83ED016AC4ED0C7A83ED87
:10077000027A0A60BDEC028BBDE8F087B4F916007E
:10078000B4F91810B4F91A206F4B07EE900AF8EE7E
:10079000E76A07EE901AB8EEE77A07EE902AF8EECD
:1007A000E77AC4ED0A6A188059809A8084ED0B7A42
:1007B000C4ED0C7A2FE7654E3288322A00F0D080E3
:1007C000002A40F02781624E3278002A97D0614F8C
:1007D000D5F8E825D5F8E015D5F8E40587FB02EC57
:1007E000D217C2EB2C12B4F814C0A2EB0C029A8000
:1007F00087FB01C287FB00C7C017C0EB2710C917D2
:10080000554F5880C1EB2211002232701980BA81F5
:10081000FA81FFF7FFFDFBF777F901202DF022FEAB
:100820006B686CE7B2F5C87F18BFD5F8C825D4ED62
:100830000A6A0EBF9FED497A07EE902AB8EEE77A72
:10084000DFED467A37EE267A0022C4ED0A7ABDEE55
:10085000C77A1A80328817EE101AB2F5C87FC5F829
:10086000C81505D0D5F8CC2507EE902AF8EEE77A22
:1008700094ED0B7A378877EE877A0020FDEEE77AE1
:100880004FF0000C17EE902AB7F5C87FE062C5F86C
:10089000CC25A3F802C000F0B18094ED0C7A20635F
:1008A000D5F8D005A3F804C007EE900AF8EEE77A71
:1008B000012F77EE877AFDEEE77A17EE900AC5F8FA
:1008C000D00529D1DFF88CE0B4F81480C8308EFB55
:1008D00000A9C831C832C017C0EBE9108EFB01A9CE
:1008E0008EFB02AED217C2EBEE12C917DFF868E03A
:1008F0005A80C1EBE911A0EB080098801980AEF88E
:100900000CC0AEF80EC0FFF785FDFBF7FDF83846CA
:100910002DF0A8FD37886B68013F3780EBE600BFFC
:10092000405200200D880020F4300020F8300020D4
:10093000A87B002068520020A826002084A3002065
:10094000107600201476002010880020AA7B00205A
:10095000A67B00201F85EB51E43000200000000042
:100960003F4A1968D268C5F8DC259FED3E7AB3F995
:100970000420C5F8D415A5F8D825D4ED0A6ADFED12
:10098000397A37EE267A0022C4ED0A7ABDEEC77AAC
:100990001A80328817EE101A322AC5F8E01505D0F1
:1009A000D5F8E42507EE902AF8EEE77A94ED0B7A75
:1009B000328877EE877A0020FDEEE77A002117EE85
:1009C000907A322AE062C5F8E47559803DD094ED02
:1009D0000C7A2063D5F8E805998007EE900AF8EEC6
:1009E000E77A012A77EE877AFDEEE77A17EE900A2A
:1009F000C5F8E80515D0013A3280E4E6D4ED0C7A6A
:100A00002063FDEEE77AA3F804C017EE902AC5F83C
:100A1000D02581E7D5F8E02507EE902AB8EEE77AF1
:100A2000ABE71148114B01700B201A7029F012FB33
:100A30006B68D5F8D4251A600949B5F9D875D5F889
:100A4000DC059F803288C860D5E7D4ED0C7A20633E
:100A5000FDEEE77A998017EE901AC5F8E815CAE717
:100A6000E430002000000000AC7B0020A57B0020CB
:100A700008B5FCF745FFFFF7CDFCBDE80840F8F7E7
:100A80001BB900BF08B5034B1B6803B1984772B68A
:100A900034F0A2FA68310020074B10B51B681844E7
:100AA0000C46007EF8F7C0FD20B12146BDE810409D
:100AB000FAF784B910BD00BF2487002030B5044682
:100AC000C06D21718389A26823F400531B041B0CA1
:100AD000838185B06379009213F0040F4FEA0332EB
:100AE0004FEA03230CBF00254FF4805503F48063C5
:100AF00002F40052ADF80450ADF80830002511F0B2
:100B00000103ADF80620ADF80C501ED1ADF80A3047
:100B100008238D07694648BFADF80A3012F056FC2D
:100B20006279E36DD10715D412F0080F9A8A05BFD8
:100B300022F00802120442F00802120C9A829A89EA
:100B400042F400529A8105B030BD0423ADF80A305A
:100B50000C23DEE707498B4205D0A1F54C418B42BF
:100B6000E2D1012000E000200121FFF795FF62792A
:100B7000E36DD9E70010014030B50446C06DA160B7
:100B8000838923F400531B041B0C838185B0637994
:100B9000009113F0040F21794FEA03324FEA032347
:100BA00003F48063ADF808300CBF00254FF4805586
:100BB000CB0748BF0423ADF804504FF00005ADF853
:100BC0000A5002F400524ABFADF80A3008230C2341
:100BD000ADF80C508D07694648BFADF80A30ADF846
:100BE000062012F0F3FB6279E36DD10710D412F006
:100BF000080F9A8A05BF22F00802120442F0080288
:100C0000120C9A829A8942F400529A8105B030BD42
:100C100007498B4205D0A1F54C418B42E7D1012019
:100C200000E000200121FFF737FF6279E36DDEE786
:100C3000001001400A4B10B51B6803440446187E9F
:100C4000F8F7F2FC50B128228271621CC2712EF0BA
:100C50002FFB20460021BDE810401DE710BD00BF5E
:100C600024870020074A002302E00133102B07D01D
:100C70005168814202F12002F7D1581CC0B270477E
:100C800000207047402400200138F0B540013C4C62
:100C9000DFF820C125583B4FDCF83060BD420CBF67
:100CA0004FF400154FF4800527182E437D68CCF8CB
:100CB0003060354EF960B54283B07B6151D0334B23
:100CC0009D424ED0A3F57A739D4236D003F58063E2
:100CD0009D4232D0A3F57A739D4246D003F58063DE
:100CE0009D4242D0A3F57A739D4240D003F58063C4
:100CF0009D423CD0A3F57A739D4234D003F58063C6
:100D00009D4230D0A3F57A739D4232D003F58063C3
:100D10009D422ED0A3F57A739D422CD003F58063BB
:100D20009D4228D0A3F57A739D4226D01849194BCD
:100D30008D420CBF1D46002500E0174D044492096A
:100D4000667CE5610021012301A88DF804608DF81F
:100D500005208DF806108DF807302EF007FB03B044
:100D6000F0BD0E4DEAE70E4DE8E70E4DE6E70E4DFD
:100D7000E4E70E4DE2E70E4DE0E7064DDEE700BF8B
:100D800040240020006002401060024010640240D5
:100D9000B864024000800028008800102080001005
:100DA0002080002000802010008000180088002093
:100DB00000802020003802400138F0B44401094886
:100DC000094D0359094F2E6B2044BB420CBF4FF411
:100DD00000134FF4800333432B6301764276F0BC5B
:100DE000704700BF402400200038024000600240ED
:100DF0002DE9F04F534C54F8204083B0002C00F004
:100E00009C80656E002D00F09A809846174604F18C
:100E10006A034D4A064628692260636104F1EA02CA
:100E20008023A261E3604FF480726B68A16022614D
:100E3000E365A24668B1FFF715FF721CD2B20C2120
:100E4000FFF7BAFFE36DA9682A69A263043321643E
:100E5000A365E868A0B1FFF705FF721C8146D2B216
:100E60000B21FFF7A9FF2346EA7F38494846FFF7E1
:100E70000BFFD5E90212E36D616404336365E2633D
:100E800094F86900F8F7D0FB814694F86800F8F709
:100E9000CBFB8346287F00284CD118F0080F36D1B1
:100EA000BA070DD5B9F1000F0AD00B22731C89F8CF
:100EB000062089F8073048466A7F2221F8F74EFA63
:100EC000FB0715D4236C7BB995F82020A97F8DF8FA
:100ED000063001A8930901228DF805308DF8041021
:100EE0008DF807202EF042FA504603B0BDE8F08F8F
:100EF000BBF1000FE6D0701C0C238BF807008BF8B9
:100F0000063058466A7F2221F8F728FADAE7B9F165
:100F1000000F05D0701C0B2389F8070089F80630F4
:100F200018F0100F484614BF022112216A7FF8F70B
:100F300015FAC7E72EF09EF9AFE7A246D4E7AA4616
:100F4000D2E700BF04870020F4690408F186000896
:100F50000348D0F8EC3113B100F5F0701847704732
:100F6000402400200348D0F8CC3113B100F5E070E4
:100F700018477047402400200348D0F8AC3113B123
:100F800000F5D07018477047402400200348D0F87F
:100F90008C3113B100F5C070184770474024002011
:100FA0000348D0F86C3113B100F5B07018477047A2
:100FB000402400200348D0F84C3113B100F5A07054
:100FC00018477047402400200348D0F82C3113B153
:100FD00000F5907018477047402400200348D0F86F
:100FE0000C3113B100F58070184770474024002081
:100FF0000348D0F8EC300BB1E0301847704700BF21
:10100000402400200348D0F8CC300BB1C030184742
:10101000704700BF402400200348D0F8AC300BB12B
:10102000A0301847704700BF402400200348D0F884
:101030008C300BB180301847704700BF402400202F
:101040000248C36E0BB1603018477047402400203F
:101050000248C36C0BB14030184770474024002051
:101060000248C36A0BB12030184770474024002063
:101070000248C36803B11847704700BF40240020EE
:10108000F8B5624D04012F190646387A2EF0F2F8B1
:101090003B7A03F01F015B090122032B02FA01F2E4
:1010A0006DD0042B66D0022B5CD02B190136187939
:1010B000F8F7BAFAF6B2074610B11223C671837177
:1010C0002B195879F8F7B0FA10B11323C671837150
:1010D0002B199879F8F7A8FA10B11423C671837107
:1010E0002E190A21F2793846F8F738F97079F8F7AD
:1010F0009BFAF2790A21F8F731F9B079F8F794FA06
:10110000F2790A21F8F72AF92B59414A934246D03D
:10111000404A93424ED0404A934256D03F4A93426F
:101120005ED03F4A93422FD03E4A934263D02B1960
:101130001B7BE3B9012002222B59198801F441518C
:1011400041F445710A4302431A809A8B22F40062EB
:101150001204120C07219A8319821A8842F0400265
:101160001A80F8BD304B596A0A435A629DE7002045
:101170000246E1E72C4B19690A431A6195E72A4BAD
:10118000196A0A431A6290E702F568424FF4801028
:10119000536A43F48013536211F0F2FCC7E702F57F
:1011A00084324FF48050536A43F48053536211F0F9
:1011B000E7FCBCE702F500324FF48040136A43F4C9
:1011C0008043136211F0E4FCB1E702F5FE324FF404
:1011D0000040136A43F40043136211F0D9FCA6E700
:1011E00002F582324FF40050536A43F400535362C5
:1011F00011F0C6FC9BE702F564424FF40010536AFD
:1012000043F40013536211F0BBFC90E7DC8700202D
:101210000030014000380040003C004000340140F4
:10122000005001400054014000380240044B18783F
:1012300028B1044A1268520744BF00201870704752
:10124000F28100200020014043680B4A23F04073E4
:1012500023F4807343F48073436083681A4042F040
:1012600002028260C36A0139C9B223F4700343EAFF
:101270000153C362704700BFFDF7FFC01D4B1B68E1
:10128000022B30B432D81C4A1C4903EB43035B00E9
:1012900098189B5A428880884B60C1E90202B3FBD0
:1012A000F2F21748174D1849184B194C00FB02F27F
:1012B0002A60D1F8882042F47002C1F888201A68A8
:1012C000002042F001021A6098601A6822F08472CD
:1012D00022F480321A605C601A684FF0006422F4D5
:1012E00080221A60D8608C6030BC7047034A536813
:1012F000D268D4E7E0BF002048980408000000202E
:1013000040420F0084A5002000ED00E000380240BC
:101310001030002400230122C27083700380037107
:1013200043718371C37103724372704700230A22B1
:1013300003604360C381C0F80630C0F80A30028001
:10134000704700BF2DE9F843704CE279237A9A4246
:101350007FD0E279E379C2EBC20204EB8202C3EBF5
:10136000C30304EB830392F82B101E7C8B1E9E425A
:101370002CD0674AB4F864301278E16801339BB22C
:101380001B2AA4F8643067D00025E379614A013351
:10139000A2FB0302520802EB42029B1ADBB2E3718A
:1013A00000293BD0F8F752FFD4F89830C01AB0F5B6
:1013B000FA7F04DB002345F0040584F89630D4F866
:1013C0009030002B32D12846BDE8F883E37904F150
:1013D0001007C3EBC30307EB830361B11944002279
:1013E00013F8015B2A44994292B2F9D1D3B203EBCC
:1013F0001222FF2A38D0464AB4F864301278E168E5
:1014000001339BB21B2AA4F86430BDD1424BB4F81F
:1014100064205A8004229A800025B6E794F896301A
:10142000002BBFD1D4F89030002BCCD03B4A1268AF
:10143000D31AB3F5FA7FC6D994F86630032B04BFEC
:101440000023A4F88C300023C4F890302846BDE86F
:10145000F883E1680025A3E72F4BB4F864205A8095
:1014600003229A80002590E7E37901221C2101FBE9
:101470000323FA18FD5C5DB3012D15D1082E3CD075
:10148000234AB4F864301278E16801339BB21B2A16
:10149000A4F864307FF478AF1F4BB4F864205A800E
:1014A00006229A80002570E7194AB4F86430127851
:1014B000E16801339BB21B2AA4F864307FF464AF67
:1014C000154BB4F864205A8005229A8000255CE709
:1014D000192EE16824D00E4AB4F864301278013332
:1014E0009BB21B2AA4F864307FF44FAF0A4BB4F8C8
:1014F00064205A8006229A8047E794F89430002BA3
:1015000040F0E9801D46E1683FE700BFDC2C002089
:101510000D880020ABAAAAAA10880020108A0020FB
:1015200092F802C05578036992F8038092F804900B
:101530009679D77992F808E00CF0070C45EA0C256B
:1015400008F03F0892F80AC01D8095784FEA4818C5
:1015500048EAD508957BA3F8028092F803804FEA09
:10156000890040EA981092F8058008F0010840EAE6
:101570008820988006F00F06507992F80780F601CF
:1015800046EA5000567AD8804FEA4E0E4EEAD81EF0
:1015900006F0030692F80680D07A07F07F074EEA3D
:1015A000462E3F01567BA3F80AE047EA18171F8131
:1015B00006F00707967A92F809E0C00040EA561054
:1015C000167B0CF01F0C46EA072605F03F05577BFB
:1015D000D8816D014FEA8C1C45EAD7004CEA9E0C7D
:1015E000A3F80CC01E825882D07B92F80EE0D77C04
:1015F00092F8128092F811C0967C557D800040EAE6
:101600009E1092F810E07F000EF0010E47EAD81706
:101610000CF00F0C92F8108040EA8E204FEACC1CA0
:1016200092F814E098824CEA580C907DA3F816C00A
:1016300006F07F0692F811C00EF0030E47EA4E271F
:10164000360146EA1C165F8392F814C0577D1E834C
:1016500005F01F05AD01C00045EA9C0540EA5710A2
:10166000D8839D83D57D40F2147015F0010F14BF0F
:101670000646AD2615F0020F08BFAD201E84588423
:101680002B0759D415F0040F0CBF0125092594F838
:101690006630032B1AD194F86700137E2B4FA26E8D
:1016A00004EB4006C3EB8323A7FB0373B6F86C700F
:1016B0005B09D21B01301A4400F00F0084F8670068
:1016C0001009A6F86C30A266A4F88C00204B1B68A9
:1016D000C4F8903059E65378102B14D01ED8D3B9E3
:1016E00094F89530E168002B7FF44EAE94F8973073
:1016F000012B23D919B10A78303A012A1ED90025C5
:1017000084F8975041E694F895300BB984F89550D9
:10171000012384F89630E168002536E6303B012B42
:10172000F9D852F8010FE46091889379A180206084
:10173000A3710849002528E60325A8E70133012203
:1017400084F8973084F8962000251EE61F85EB511B
:10175000108A0020DC2C002010B50446F8F776FD36
:10176000514B002283F89C2093F89D20012A19D91F
:10177000D3F8A02040F6AC51821A8A4212DD4B49C0
:10178000B3F864200978013292B21B29A3F86420CF
:1017900005D1474AB3F8641051800121918000229D
:1017A00083F89D20E2B27E2A27D093F89D1019B3CA
:1017B00093F89D101B2956D893F8AC1000296CD0D3
:1017C000002182F0200283F8AC1093F89D100229CA
:1017D00003D1012A08BF83F8A420197A93F89D4009
:1017E00093F89D00C1EBC10103EB8101214401305D
:1017F000C0B2CA7383F89D0010BD93F89D20012AE2
:101800002BD91A7A2B49DC790132A1FB02C1490894
:1018100001EB4101521AD2B294420AD093F89D4092
:10182000197A1A72C1EBC10103EB8101621E81F8C2
:101830002B2093F8A4203AB10121002283F89C10B8
:1018400083F8A420C3F89800184A12781B2A1ED0E7
:101850000022C3F8A80083F8AC20012283F89D2061
:10186000C3F8A00010BD002283F89D200F49B3F8F3
:1018700064200978013292B21B29A3F86420BBD1FD
:101880000B4AB3F8643053800223938010BDD3F821
:10189000A8200749821A0A80DAE77D2A95D1012219
:1018A00083F8AC2010BD00BFDC2C00200D88002088
:1018B00010880020ABAAAAAA03788B4283BF034BEF
:1018C00003EB4101B1F8B00000207047DC2C002090
:1018D000044B93F8C80018B1002283F8C8200120F7
:1018E000704700BFDC2C0020F0B4C24D95F8EF60CB
:1018F00005F1CC020244B41E1444A24200F07881E7
:10190000013A013C002341F2210112F8017F83EAF0
:1019100007231FB2BBB2002FACBF5B0081EA4303B9
:101920009BB21F0454BF5B0081EA43039BB21F04B8
:1019300054BF5B0081EA43039BB21F0454BF5B00AA
:1019400081EA43039BB21F0454BF5B0081EA430357
:101950009BB21F0454BF5B0081EA43039BB21F0488
:1019600054BF5B0081EA43039BB21F0454BF5B007A
:1019700081EA4303A2429BB2C7D10644B21E013E94
:101980002A442E4492F8CC1096F8CC2002EB012287
:1019900092B29A4201D0F0BC704795F8F020002A2C
:1019A00000F02181431CDBB25C1C2C442B444FF41F
:1019B000AF6193F8CC6094F8CC3003EB06239BB274
:1019C00001FB03F31B1303F54873012AA5F8B0309C
:1019D00000F00981C31CDBB25C1C2C442B44022A9E
:1019E00093F8CC6094F8CC3003EB06239BB201FB58
:1019F00003F34FEA233303F54873A5F8B23000F040
:101A0000F280431DDBB25C1C2C442B44032A93F868
:101A1000CC6094F8CC3003EB06239BB201FB03F3BC
:101A20004FEA233303F54873A5F8B43000F0DB80A8
:101A3000C31DDBB25C1C2C442B44042A93F8CC60FD
:101A400094F8CC3003EB06239BB201FB03F34FEA7F
:101A5000233303F54873A5F8B63000F0C48000F1D5
:101A60000903DBB25C1C2C442B44052A93F8CC60A0
:101A700094F8CC3003EB06239BB201FB03F34FEA4F
:101A8000233303F54873A5F8B83000F0AC8000F1BB
:101A90000B03DBB25C1C2C442B44062A93F8CC606D
:101AA00094F8CC3003EB06239BB201FB03F34FEA1F
:101AB000233303F54873A5F8BA3000F0948000F1A1
:101AC0000D03DBB25C1C2C442B44072A93F8CC603A
:101AD00094F8CC3003EB06239BB201FB03F34FEAEF
:101AE000233303F54873A5F8BC307CD000F10F0315
:101AF000DBB25C1C2C442B44082A93F8CC6094F88D
:101B0000CC3003EB06239BB201FB03F34FEA2333F4
:101B100003F54873A5F8BE3065D000F11103DBB2C0
:101B20005C1C2C442B44092A93F8CC6094F8CC30EC
:101B300003EB06239BB201FB03F34FEA233303F5C8
:101B40004873A5F8C0304ED000F11303DBB25C1C23
:101B50002C442B440A2A93F8CC6094F8CC3003EB45
:101B600006239BB201FB03F34FEA233303F54873CB
:101B7000A5F8C23037D000F11503DBB25C1C2C4451
:101B80002B440B2A93F8CC6094F8CC3003EB06235B
:101B90009BB201FB03F34FEA233303F54873A5F827
:101BA000C43020D000F11703DBB25C1C2C442B4462
:101BB0000C2A93F8CC6094F8CC3003EB06239BB24C
:101BC00001FB03F34FEA233303F54873A5F8C6304E
:101BD00009D000F11903DBB25A1C2A442B4493F8B4
:101BE000CC3092F8CC30012385F8C830F0BC704777
:101BF0000023C2E6DC2C002070B55C4C0646F8F7EA
:101C000025FBD4F8F430C4F8F400C01AB0F5FA5F3C
:101C10001AD9002384F8F83084F8F930A12E2FD097
:101C2000A22E00F09C8094F8F92094F8EF30002563
:101C3000A2B16A1C6119D5B2F6B29D4281F8CC609E
:101C400084F8F8500CD070BD94F8F850002DE5D011
:101C500094F8F92094F8EF30002AEAD19D42F2D1AD
:101C600094F8FA30052B72D0062B03D194F8CD30BE
:101C70001E2B0DD0002384F8F93084F8F83070BDA5
:101C800001221B2384F8F92084F8EF300025D0E7E7
:101C90006A1E002A4FF0000150DD08460B4623441F
:101CA000013093F8CC30DBB283EA0105ED074FEA4F
:101CB000530348BF83F08C0383EA5105EE074FEAD4
:101CC000530348BF83F08C0383EA9105ED074FEA85
:101CD000530344BF83F08C03DBB283EAD105EE07E4
:101CE0004FEA530344BF83F08C03DBB283EA111540
:101CF000ED074FEA530344BF83F08C03DBB283EA62
:101D00005115EE074FEA530344BF83F08C03DBB257
:101D100083EA9115ED074FEA530344BF83F08C0328
:101D2000DBB283EAD1155908EB0748BF81F08C017B
:101D3000C0B248BFC9B282420346B0DC224492F826
:101D4000CC308B4296D10320FFF7CEFD92E70020E6
:101D5000FFF7CAFD94F8CD301E2B8BD198E70122F6
:101D6000232384F8F92084F8EF308FE7DC2C00205F
:101D700007299DBF034B03EB8101B1F8FC00002054
:101D8000704700BFDC2C00201A4B93F81C2132B1A5
:101D900093F820210021A82A83F81C1101D00020EB
:101DA000704793F83321002AF9D110B4DFED126A9D
:101DB00003F5907103F1F80003F59872B4EE047A1C
:101DC000CC780B7903EB042307EE903AF8EEE77A30
:101DD000B0EE666AA7EE876A02318A42FCEEC67AE6
:101DE00017EE903A40F8043FEAD101205DF8044B29
:101DF000704700BFDC2C00200080BBC310B5044638
:101E0000F8F724FA0F4BD3F83821C3F83801801AB9
:101E100041F288329042E4B205D983F82041012290
:101E200083F83C2110BD93F83C219918142A81F8BD
:101E3000204103D1012283F81C2110BD0132D2B20E
:101E4000EEE700BFDC2C0020034B03EB4101B1F8AF
:101E50004001C008704700BFDC2C0020724B93F893
:101E60006021002A00F0C28070B493F86141B3F899
:101E7000625103EB4401002091F8676191F86821F9
:101E800083F8600142EA0622954202D0002070BC2D
:101E9000704793F86521012A00F0AA80812AF6D1C3
:101EA0000320102C40F2A68093F8694193F8675103
:101EB00093F8681193F86A2141EA052142EA042265
:101EC0001024A3F84011A3F8422183F8614193F84C
:101ED0006B1193F86C21032C42EA0122A3F84421F0
:101EE000D5D093F86D1193F86E21042C42EA0122AB
:101EF000A3F84621CBD093F86F1193F87021052CED
:101F000042EA0122A3F84821C1D093F8711193F855
:101F10007221062C42EA0122A3F84A21B7D093F895
:101F2000731193F87421072C42EA0122A3F84C2183
:101F3000ADD093F8751193F87621082C42EA01226E
:101F4000A3F84E21A3D093F8771193F87821092CA8
:101F500042EA0122A3F8502199D093F8791193F81D
:101F60007A210A2C42EA0122A3F852218FD093F859
:101F70007B1193F87C210B2C42EA0122A3F8542117
:101F800085D093F87D1193F87E210C2C42EA012232
:101F9000A3F856213FF47BAF93F87F1193F880218B
:101FA0000D2C42EA0122A3F858213FF470AF93F8B8
:101FB000811193F882210E2C42EA0122A3F85A21C2
:101FC0003FF465AF93F8831193F88421102C42EA13
:101FD0000122A3F85C217FF45AAF93F8851193F89E
:101FE000862142EA0122A3F85E2150E700207047D3
:101FF000104656E7002C3FF44AAF93F8671193F868
:102000006821012C42EA0122A3F840213FF43FAFAE
:1020100093F8691193F86A21022C42EA0122A3F88D
:1020200042217FF454AF32E7DC2C002038B504465F
:10203000F8F70CF9444AD2F88C31C31AB3F57A6F29
:1020400016D892F89031C2F88C01B3B1022B1FD090
:10205000242B92F8611175D901330231DBB24900AA
:102060008B4282F890311BDB01318B4263D038BD4B
:102070000023C2F88C0182F89031A82CF7D10023FC
:1020800082F86031A2F8623192F86111204603E0D3
:10209000E0B282F861010146D51885F86401DBE7FA
:1020A000B2F86231E4B283EA042424B2002CB8BF4F
:1020B00041F22101A3B2B4BF81EA43035B009BB2AA
:1020C0001C0446BF41F2210181EA43035B009BB23D
:1020D000180446BF41F2210181EA43035B009BB231
:1020E000190446BF41F2210181EA43035B009BB220
:1020F0001D0446BF41F2210181EA43035B009BB20C
:102100001C0446BF41F2210181EA43035B009BB2FC
:10211000180446BF41F2210181EA43035B009BB2F0
:10212000190446BF41F2210181EA43035B009BB2DF
:10213000A2F8623138BD0021012382F8901182F8A3
:10214000603138BDE0B2A7E7DC2C0020F8B5134DB4
:1021500095F8A9210AB90120F8BD114B1C68236824
:102160005E6A46B1204605F5CA71B047002385F87E
:10217000A9310120F8BD05F5CA77BE1800E0236833
:102180009B68204698470028F9D0236817F8011B60
:102190001B6820469847B742F1D1E7E7DC2C0020C6
:1021A000D059002003788B4210D9094B03EB8101F1
:1021B00093F8DC31D1F8AC011BB900F5777080B22F
:1021C0007047400800F5777080B270470020704774
:1021D000DC2C00202DE9F843F8F738F8CD4C054603
:1021E00094F8DD0180B9042294F8A93153B1D4F8F0
:1021F00000323BB1ED1AB5F57A7F03DB00231046C0
:10220000C4F80032BDE8F88394F8DE11002384F8A6
:10221000DD31002900F0308194F8E031BE4F94F8B0
:10222000F0215BB213F1630FB8BF97F90030002AB9
:1022300041D013F1310F80F2B18113F1380F80F2E8
:10224000B18113F13D0F80F2B18113F1420F80F2A1
:10225000B18113F1450F80F2B18113F1470F80F284
:10226000B18113F1490F80F2B18113F14A0F00F0EF
:10227000B18113F14B0F00F0B08113F14C0F00F05E
:10228000B08113F14D0F00F0AF8113F15C0FB8BFB7
:10229000642680F24981D4F8F401DFF888C200FB9B
:1022A00006F08CFB00C6C017C0EB661004EB82067C
:1022B00080B2C6F8AC013B7094F8EC7194F8ED3143
:1022C00094F8EE0194F8EF611B0443EA076333438B
:1022D00043EA002303F0F020B0F1E02F00F0C380C8
:1022E000102794F8040294F8E231D4F8086294F8C4
:1022F0000CC23678034103F00F039E4210D90B2B1A
:102300000ED8002A40F0F38094F8E28194F8E3E1DB
:1023100004EB83030CEA08080EEB082EC3F8ACE1CB
:1023200094F8E431034103F00F039E4210D90B2BC4
:102330000ED8002A40F0DF8094F8E48194F8E5E1BB
:1023400004EB83030CEA08080EEB082EC3F8ACE19B
:1023500094F8E631034103F00F039E4210D90B2B92
:102360000ED8002A40F0CB8094F8E68194F8E7E19B
:1023700004EB83030CEA08080EEB082EC3F8ACE16B
:1023800094F8E831034103F00F039E4210D90B2B60
:102390000ED8002A40F0B78094F8E88194F8E9E17B
:1023A00004EB83030CEA08080EEB082EC3F8ACE13B
:1023B00094F8EA31034103F00F039E423ED80D2FFB
:1023C00032DD94F8EC31034103F00F039E4210D943
:1023D0000B2B0ED80AB19A420BD094F8EC8194F8EA
:1023E000EDE104EB83030CEA08080EEB082EC3F8BA
:1023F000ACE1102F18D194F8EE3143FA00F000F060
:102400000F00864210D90B280ED80AB190420BD08B
:1024100094F8EE2194F8EF3104EB800002EA0C0C02
:1024200003EB0C23C0F8AC31D1B194F8E2311B06B8
:1024300016D4C4F8005205220120D5E60B2BBED8D5
:102440000AB19A42BBD094F8EA8194F8EBE104EB2C
:1024500083030CEA08080EEB082EC3F8ACE1AEE7E4
:1024600005220120C0E694F8E20100063FF538AFEE
:102470002A480C27036034E7F7F7E8FE2649284B83
:102480004A78A3FB00035B0C12B394F8E00194F8C4
:10249000E121D2B2122A18BF012A08D002F0EF02BD
:1024A000A2F1A202B2FA82F2520902B94A70D4F839
:1024B000F81194F8F02199B18B4228D0591A0129CA
:1024C00056D094F8DE11A4F8FC01C4F8F831F3E614
:1024D00094F8E02194F8E10100EB022080B2E6E7F5
:1024E000A4F8FC01C4F8F83194F8DE11E4E6934254
:1024F0007FF40AAF14E793427FF41EAF28E79342BC
:102500007FF432AF3CE793427FF446AF50E794F854
:10251000DE11D1E6DC2C002020000020E8010020A4
:1025200083DE1B431F85EB516FF05B080C263048A0
:1025300006F1FF3900EB490E00EB46069EF801E07C
:1025400096F801C010F91960ACEB0E0C981B00FB5B
:102550000CF0A8EB060690FBF6F0704440B20028A1
:1025600001DA002697E66428A8BF6420064692E6B2
:10257000002AA6D0B4F8FC61D4F8F4111D4F861BD4
:10258000143E01FB06F187FB0176C917A1EBE601BA
:1025900004EB820689B2C6F8AC1192E76FF03008FE
:1025A0000126C4E76FF037080226C0E76FF03C0849
:1025B0000326BCE76FF041080426B8E76FF0440833
:1025C0000526B4E76FF046080626B0E76FF0480826
:1025D0000726ACE798460826A9E76FF04A080926BF
:1025E000A5E798460A26A2E798460B269FE700BF74
:1025F000246A040867666666344B5B68C3F30803A5
:1026000070B4CBB9EFF31183B3B9314A314E324DC7
:102610001368AC6811688B42FAD131688C42F7D8E4
:102620002E4A15684FF47A7101FB05F2141BB4FBB6
:10263000F5F401FB034321E0EFF31181102383F351
:10264000128803F1E023C9B29D681A6812F4803F32
:10265000234A1EBF012414609D681D4B1E68136829
:1026600081F311881D4A14684FF47A71334401FBD9
:1026700004F2521BB2FBF4F201FB0323194AD2F815
:102680001012C2F810325B1A41F288318B420AD91B
:10269000C0B2012382F8E00182F81432002382F8EC
:1026A000DD3170BC704792F814320F2BF9D8D11875
:1026B0000133DBB2C0B2102B81F8E00182F8143292
:1026C000ECD1012382F8DD3170BC704700ED00E0F1
:1026D000108A0020188A002010E000E0148A0020F0
:1026E0000C8A0020DC2C0020036933F8110000EB79
:1026F0008000C01000F55C7080B27047436993F8A9
:102700002320002A00F0CF802DE9F0477B4ADE7DB0
:10271000127800211A2A06F0040506F0080483F84E
:10272000231000F0C280002D40F0CC80002C40F03F
:10273000D980254693F802A093F8068093F801E02B
:102740000269DF7893F8049093F807C00AF0070055
:1027500008F00F014FEAC1184EEA002107F03F07C9
:10276000187A1180997893F805A093F80AE07F0110
:1027700047EAD107D97857804FEA890949EA911980
:10278000997B0AF0010A01F03F014F0149EA8A21D1
:102790009180597948EA5101D1800CF07F0C9979E8
:1027A00093F807804FEA0C1C4CEA111C597AA2F8E6
:1027B00008C0400040EAD81001F0030140EA41207F
:1027C00093F80DC0D97A50810EF01F0E587A4FEA57
:1027D0008E1E4EEA90009081187B93F80AE00CF070
:1027E000070C40EA0C20C90093F80DC0108241EAA2
:1027F0005E11D18147EADC01518293F80FE093F832
:102800000E80597CDF7C93F812C0587D4FEA8E0E03
:102810004EEA981E93F8108008F001084EEA882EC0
:1028200001F00F0193F81280A2F814E093F810E081
:102830007F00C90141EA5E0147EAD81793F814E026
:1028400093F81180D1820CF07F0C4FEA0C1C997D1B
:102850000EF0030E4CEA181C47EA4E2716F0010F43
:1028600093F814E0A2F818C000F01F0093F815C008
:10287000578340F2147314BF1F46AD278001C9006F
:1028800016F0020F40EA9E0041EA5C1108BFAD233A
:102890009083D183178453840CBB002D0CBF01207F
:1028A0000920BDE8F0871046704715491F8C0E803F
:1028B00075B147F002021A8412B274B147F00302F4
:1028C0001A8409E01A8C94B942F002021A8431E7A2
:1028D0008CB147F001021A8412B24A802AE7032021
:1028E000BDE8F0871A8C42F001021A8422E742F018
:1028F00003021A841EE73AB22546EEE70D8800204F
:10290000108800203B4B5B68C3F30803F0B42BBB7B
:10291000EFF3118313BB384A384F394E1368B5684B
:102920001468A342FAD13C68A542F7D8354A166824
:102930004FF47A7404FB06F2551BCA69B5FBF6F531
:1029400004FB03539A1A40F6AC54A2422EDC91F8D1
:10295000224074B3182C38D9F0BC7047EFF31184BF
:10296000102383F3128803F1E023E4B29E681A680F
:1029700012F4803F244A1EBF012515609E681E4B3D
:102980001F68136884F311881E4A15684FF47A741F
:1029900004FB05F23B44921BB2FBF5F204FB03235C
:1029A000CA6940F6AC549A1AA242D0DD002281F8DE
:1029B00022200F28D0D10122CB61087081F822207B
:1029C000002381F82330F0BC7047631CDBB2192B65
:1029D00081F822300855F3D10C4B1B781A2B08BF15
:1029E0000B4B4FF0010081F8230008BF9A80F0BC28
:1029F000704700BF00ED00E0108A0020188A002018
:102A000010E000E0148A00200C8A00200D880020CD
:102A100010880020094BDFED0A6ADFED0A7A03EB2C
:102A2000810191ED867AB8EE477AE7EE267AFCEEE0
:102A3000E77A17EE903A98B2704700BFDC2C00207E
:102A400001F11F3F00405C44714A92F8583233B1A3
:102A500092F85E320021162B82F8581201D0002025
:102A6000704792F85D32022BF0B440F2CE8002F54E
:102A70001770184402F25E21D32311F8014F63400E
:102A800013F0800F4FEA430318BF83F0D503DBB286
:102A900013F0800F4FEA430318BF83F0D503DBB276
:102AA00013F0800F4FEA430318BF83F0D503DBB266
:102AB00013F0800F4FEA430318BF83F0D503DBB256
:102AC00013F0800F4FEA430318BF83F0D503DBB246
:102AD00013F0800F4FEA430318BF83F0D503DBB236
:102AE00013F0800F4FEA430318BF83F0D503DBB226
:102AF00013F0800F4FEA430318BF83F0D5038842D9
:102B0000DBB2BAD192F87512994202D00020F0BC23
:102B1000704792F8640292F8636292F8681292F831
:102B20006C3292F8704292F86052B2F860C2D2F8F9
:102B3000607200F00F00C00140EA560001F01F0172
:102B400092F86762C2F82402890141EA960103F013
:102B50003F0392F86B6292F86F02C2F830125B0189
:102B600043EAD60392F85F12C2F83C3204F07F04C5
:102B7000B2F86432D2F86462240105F0070544EA31
:102B8000101041EA0521C3F30A13C2F84802B2F853
:102B90006852C2F81812B2F86A42D2F86C02B2F85F
:102BA0006E12C2F82832D2F87032C0F38A10C1F324
:102BB0004A01C3F3CA13CCF3CA0CC7F38A37C6F36E
:102BC000CA366D09C4F30A04C2F84002C2F84412BE
:102BD000C2F81CC2C2F82072C2F82C62C2F8345289
:102BE000C2F83842C2F84C3292F8743292F873024A
:102BF000B2F87212DB0043EA5013C1F38A01C2F843
:102C00005432C2F85012012081E7D3237AE700BF83
:102C1000DC2C0020F8B5634B634C1D68EB070646BF
:102C200015D594F89C3294F89D229A4235D1D4F867
:102C3000A032B34202D85D4B00221A70D4F8D802F9
:102C4000301A002822DD012084F8DC02F8BD15F4DA
:102C5000005543D1D4F8C83204F530709847C707FF
:102C60000AD5534A94F86630C0F3400110F00A0FB9
:102C7000917023D0052B62D04307D8D5012384F867
:102C8000DD32D4F8A032B342D8D8D4E794F8DC02CD
:102C90000028DBD194F8DD02F8BDD4F8A402444941
:102CA000424A84F89D32304400250123C4F8A00232
:102CB00001208D70137084F8DC02C7E7D4F8A422D9
:102CC000052B1644C4F8A0624FD0420765D4374B99
:102CD000012201201A7084F8DC02B7E7B4F8A832A8
:102CE0000BBBB4F8AA32F3B9B4F8AC32DBB9B4F820
:102CF000AE32C3B9B4F8B032ABB9B4F8B23293B9AA
:102D0000B4F8B4327BB9B4F8B63263B9B4F8B832B7
:102D10004BB9B4F8BA3233B9B4F8BC321BB9B4F811
:102D2000BE32002B83D0D4F8A43221491F4A334449
:102D30000020C4F8A0320123887013707EE794F855
:102D40006730A26E04EB43010133B1F86C70A1F857
:102D50006C50D21B110903F00F03A4F88C1041072B
:102D600084F86730A26689D461E794F86720A36E7F
:102D700004EB420103F2FF33B1F86C5001325B1BEC
:102D800002F00F0240F2FF3584F867201A09A1F81B
:102D90006C50A366A4F88C2097E7012384F8DD32F9
:102DA00095E700BF84A30020DC2C00205D5C0020A0
:102DB000200000200020704700207047012070474D
:102DC000024B03EB4101B1F8E0027047DC2C00201C
:102DD000044B93F8040318B1002283F80423012064
:102DE000704700BFDC2C0020024B03EB8101B1F8DF
:102DF00008037047DC2C002038B50446F7F726FAA4
:102E00002E4BD3F84023821AB2F5FA7F14D9002250
:102E1000C3F8400383F8442383F84523E1B204292F
:102E200024D0202922D093F848230AB9552C35D034
:102E3000A24216D1002209E093F8452392B993F8F3
:102E40004423C3F84003E1B2002AE8D093F84603D4
:102E50009C180138824284F850131BD0013283F849
:102E6000442338BD013A83F8452338BD00220224AB
:102E70004FF6FF7083F84C43A3F84A039C18481E92
:102E8000824283F8481383F8461383F8472384F873
:102E90005013E3D1012283F8702338BD01201F2590
:102EA00083F84843A3F84A2383F8501383F8470371
:102EB00083F84C0383F84653D0E700BFDC2C002096
:102EC00003788B4283BF034B03EB4101B1F87403DA
:102ED00000207047DC2C002038B5394C0546F7F748
:102EE000B5F9D4F8C833C4F8C803C01AB0F57A7F6E
:102EF0001CDD0023282284F8CC3384F8CE3384F8F8
:102F0000CF3384F8CD233D2D42D03E2D0DD12D4A17
:102F1000C4F8D023012384F8CE330123157084F83C
:102F2000CC3394F8CD239A4220D038BD94F8CC23EA
:102F3000002AE8D0531CDBB2D4F8D01384F8CC3389
:102F4000062B8D54EDD194F8CE33012B27D094F875
:102F5000CF33012B27D00023282284F8CC3384F8E8
:102F6000CE3384F8CF3384F8CD2338BD94F8CE33F4
:102F7000012B04BF022384F8CE3394F8CF33012B06
:102F800015D00022282384F8CC2384F8CD3338BD13
:102F90000D4AC4F8D023012384F8CF33BDE78B78E2
:102FA000282BD4D8F1E78B78092BD4D8EDE702236E
:102FB00084F8CF33F7F74AF9C4F8D403E1E700BF48
:102FC000DC2C00207C3000207030002030B4024621
:102FD000002305251E2400E00232032BD4BF00216C
:102FE000012100F813100133042B04D0122B54706C
:102FF000F2D130BC70475570EEE700BF024B036062
:1030000043608360C3607047E803D007024B03EB63
:103010004101B1F8A8027047DC2C0020024B03EB01
:103020004101B1F8A8027047DC2C002030B4264CD6
:1030300094F8CE33022B02D0002030BC704794F8B5
:10304000A253EDB1013D04F2A13353FA85F504F525
:103050006870002210F8013B534083EA0313DBB28F
:10306000120AD90042EA0322854281EA131382EA56
:103070000302EFD122B1002084F8CE0330BC7047A8
:10308000B4F8A0335BBA9BB243F60162934209D015
:1030900043F60362934205D0002384F8CE33012027
:1030A00030BC7047094AA2F12E0102F12005D07907
:1030B0009379023203EB0023C3F3CC03AA4221F835
:1030C000023FF4D1E8E700BFDC2C00207C30002078
:1030D00070B540F2014444EA8004F7F7B7F80C4EAB
:1030E000054696F8F83306EB8303D3F8D803E307D5
:1030F0000AD5F7F75DFE640805F1340507D0F7F748
:10310000A5F88542FBD8ECE7F7F74CFEF3E770BD76
:10311000DC2C00200D49B1F8F93330B508224AF211
:10312000010580EA030414F0010F4FEA530318BFAE
:103130006B4002F1FF3218BF9BB212F0FF024FEA60
:103140005000EED1A1F8F93330BD00BFDC2C0020D7
:10315000084619F063BA00BF0FB400B583B004ABE2
:10316000054953F8042B01930020F9F759FD03B0EA
:103170005DF804EB04B07047513101080EB470B52E
:1031800083B007AC0646482054F8045B19F046FAB1
:10319000202019F043FA304619F02CFA3A2019F0A1
:1031A0003DFA2A462346094901940020F9F738FDE3
:1031B00004460A2019F032FA054A136803341B1B2F
:1031C000136003B0BDE8704003B07047513101088F
:1031D000C0720020F8B50F4BD3F8FC53D3F800446D
:1031E000D3F80464A9B1831E00EB410727441E44B1
:1031F00004441D4434F9022B36F9023F35F9020F1D
:10320000134403EBD373A0EB630019F0C2FAA74297
:10321000F0D1F8BDDC2C0020F8B52A4C2A4D38221C
:103220000021204633F0FAFA284B95F80B64B3F8E6
:103230005C20A283103393E8070095F80C7484F89F
:10324000207004F1080383E807001EB1072E01D0A7
:10325000012E02D0237F032B01D00020F8BD1C4A91
:103260001C4913681C4E216043F0020313601B4984
:103270001448616003224FF480730727A277A3826A
:103280007771F5F72DFAB5F818344FF47A72626257
:103290007BB1134E06F16C07B5F81834616A00EE85
:1032A000103A3046B8EE400A2436FAF777F9B742BA
:1032B000F2D195F80A3413B1A3770120F8BD0120AB
:1032C000F8BD00BF40520020DC2C0020FC9C0020F8
:1032D00080520020E186000820000020DDB20008B6
:1032E000F83000202DE9F04F2DED068BAB4B9B7D88
:1032F000012B87B000F09E85022BA94B02931A4642
:103300000CBF0723002382F88834A64B1B78132BAD
:1033100000F292840122A4499A400A4208BF002385
:103320009E49029C4A79DFF898A284F88934131CDC
:1033300018BF0123C9798AF8613020220023232095
:103340008AF85E3084F88A348AF8652084F88B1411
:10335000F7F772F9954BDAF81800CAF8143002231F
:103360008AF81030002800F05B851C22002382714F
:10337000C3710921F7F77AFCDAF81800F7F718FD9E
:103380004FF48071DAF81400FBF748FADAF81830D5
:1033900013B11A689B885383DAF8140040F2E933BA
:1033A00002E0002B00F057850289013B12F0020F6A
:1033B0009BB2F6D06B23838140F2E93302E0002B0D
:1033C00000F049850289013B12F0010F9BB2F6D053
:1033D000838940F2E93302E0002B00F0388502894E
:1033E000013B12F0020F9BB2F6D08023838140F2A2
:1033F000E93302E0002B00F02A850289013B12F03C
:10340000010F9BB2F6D08389DAF8183013B11A682D
:103410009B8813830623664CDFF8A881DFF8A89108
:10342000644D654E04939623DFF8A0C101934FF0DD
:10343000100ED9F80430C3F30803002B40F0E880E5
:10344000EFF31183002B40F0E3802068AA68236823
:103450009842FAD133689A42F7D8D8F800704FF4FE
:103460007A7101FB07F39B1AB3FBF7F301FB003002
:103470004FF47A77D9F80430C3F30803002B40F0F7
:10348000A780EFF31183002B40F0A2802368A96886
:1034900022689342FAD132689142F7D8D8F80020D6
:1034A00007FB02FBABEB0101B1FBF2F107FB0313DE
:1034B0001B1AB3F57A7FDDD3019B013B0193B8D191
:1034C000DAF8183013B11A689B885383DAF81400BD
:1034D00040F2E93302E0002B00F0BC800289013B9E
:1034E00012F0020F9BB2F6D0F523838140F2E9334C
:1034F00002E0002B00F0AE800289013B12F0010FC8
:103500009BB2F6D08389838940F2E93302E0002B35
:1035100000F09D800289013B12F0020F9BB2F6D0B1
:10352000FF23838140F2E93302E0002B00F08F801B
:103530000289013B12F0010F9BB2F6D08389DBB206
:103540000393DAF8180010B1036882881A83039B8A
:10355000682B00F08480049B013B13F0FF0304936D
:103560007FF461AF9AF85C300299DAF85820C1F81C
:103570008C24032B00F0B6800020104E8AF86700E0
:10358000737A23B19AF86630003318BF012373723F
:1035900007B0BDEC068BBDE8F08F00BFCC9C0020CF
:1035A000DC2C00200D88002048800A0000300140FB
:1035B000108A002010E000E0188A0020200000207F
:1035C000FC9C0020148A002000ED00E00C8A002002
:1035D000EFF311818EF31288D5F808B02B68DB0366
:1035E00004D50123CCF80030D5F808B02368DCF806
:1035F0000020C9B281F31188D8F80010134407FBEA
:1036000001F2A2EB0B02B2FBF1F207FB03234FE73F
:10361000EFF311828EF31288AF682B68D90303D5BC
:103620000123CCF80030AF682368DCF80000D2B288
:1036300082F31188D8F800104FF47A72184402FB14
:1036400001F3DB1BB3FBF1F302FB003010E7F7F7EC
:103650006FFD76E7F7F76CFDDAF8140053E7F7F73C
:10366000A1FBDAF8140040F2E93302E0002B00F08D
:10367000E9830289013B12F0020F9BB2F6D08C2342
:10368000838140F2E93302E0002B00F0DB83028902
:10369000013B12F0010F9BB2F6D08389838940F27F
:1036A000E9330289013B12F0020F9BB240F09C8388
:1036B000002BF6D1F7F73CFDDAF81800F7F778FBA6
:1036C000059B142BFFF44EAF182B03D9543B062B4C
:1036D0003FF648AF03228AF85C20029ADAF85830A5
:1036E000C2F88C34D249D34C0B68D34AD34EE0781D
:1036F000CAF81C2043F0010306220B60D04BD149CD
:1037000032718AF86720CAF80030032200230128AA
:10371000CAF804108AF85E20A37140F290829FEDEF
:10372000CA7A8AF85F30012307EE903AF8EEE77A1A
:10373000C04DC64C8AF8620067EE877A013BFCEE0A
:10374000E77A8AF86430C2482B798AF86330C4ED8E
:10375000007AFBF759FD2B780BB18AF85E30012314
:103760008AF866302DF018FE25689FEDBA0ABA4C2B
:10377000DFF8348307EE905AF8EE677A80EE270A76
:1037800031F038FDA4FB0034640840F235539C420C
:10379000A8BF1C46A7B2029A7B08A2F89C3407EE89
:1037A000907A9FEDAE7ADFEDAE6AA2F89474F8EEEF
:1037B000677A4FEA970987EE270AA2F8969467EE90
:1037C000A67AB7EE087A17EE903A30EE470A48F834
:1037D000083B31F00FFD029A9FEDA25ADFEDA25A8D
:1037E000DFEDA24A9FEDA22ADFEDA22A9FEDB23AB9
:1037F0009FEDA11ADFEDA11ADFEDAD6A0128B8BF78
:10380000012082F89E04002306E00133F6EE007AE0
:10381000202BE8EC017A55D007EE903AB8EEE77A23
:1038200027EE057A77EE257ABDEEE76A16EE102AC6
:103830002032402AE9D8B4EEE57AF1EE10FA40F3EE
:1038400010829FED9A6A01E0F0EE477AF4EEC67AB4
:10385000F1EE10FA37EEE67AF6DCB4EEE47AF1EE49
:1038600010FA40F1FB819FED936A01E0B0EE677AB8
:10387000B4EEC67AF1EE10FA77EE267AF6D4F4EECC
:10388000E57AF1EE10FA40F3E18171EEE77A27EE86
:10389000A76AF0EE623AE6EE023A0133202BF0EE30
:1038A000430AE3EE860AB7EE007A26EE674A77EE21
:1038B000677AB6EE007AE4EE207A67EE877AE8EC73
:1038C000017AA9D15B496E4A887FB2FBF4F107EE19
:1038D000100AB2FBF5F080B2B0FBF7F0C0B207EE11
:1038E000900A92FBF4F2F8EEE77AB7EE005A85EE12
:1038F000270A05EB4505AD00A9420F4638BF2F4604
:103900004C498AF8F502AAF80C355E4C04EE907A20
:10391000F8EE644A06EE102AFCEEE44ACA7F9FEDF8
:103920005A3ADFED5A0ADFED5A6ADFED4F5A8AED57
:10393000BE0AB8EEC66AF8EE644AB8EEC77A64EE1C
:10394000A04A07EE902A26EE036A03EE109AC6EE0E
:10395000872A504ACAF8042502F12803A8324E49A2
:10396000CAF80035CAF810251023AAF8FC3414232D
:10397000AAF80835A1F54377A1F55E739FED477A64
:10398000DFED476A9FED474A9FED3C2ADFED373A6E
:103990009FED371ADFED371AB8EE433AF8EEE77AC3
:1039A00034EEA50A26EE036A77EE677ABDEEC07A9A
:1039B00076EE250A17EE10CABDEEE47A67EEA67A17
:1039C00017EE105ABDEEE07A0CF1200C17EE100A3B
:1039D000BDEEC67A203517EE102A20302032C4ED15
:1039E000007AC824402A21F8024B00F28E81B4EEFE
:1039F000C26AF1EE10FA40F34982F0EE467A9FED8A
:103A00002C3ADFED2A6A01E0F0EE477AF4EEE67A2E
:103A1000F1EE10FA37EEC37AF6DCB4EEE37AF1EEAB
:103A200010FA40F130829FED223ADFED226A49E040
:103A300080520020CC9C002090C1793D20000020C5
:103A400009F200081DB2000800007A44EC9C002036
:103A5000FC9C002000247449ABAAAAAA00003445AB
:103A60000000003D3C8C4F3EDB0FC93FDB0F49C0DF
:103A700092E741B99730083CDB0FC9BFDB0F4940E3
:103A800040420F006C31002027D4D236E5A6C5395C
:103A900000004842406A04087CA300200000C8429D
:103AA0000AD7233C0000000074310020E4CB16410B
:103AB000DB0FC940E4CB16C115A82ABEF304353F7D
:103AC000B0EE677AB4EEE67AF1EE10FA77EE037AAA
:103AD000F6D4F4EEE57AF1EE10FA40F3678172EE77
:103AE000677A67EEA76AB0EE618AA6EE818A4028FF
:103AF0001FED0F7AA8EE267A27EEA63AE3EE077AB4
:103B000067EEA26A76EE858A35EE663AC5EE287AC9
:103B100066EEA76A23EE273AB1EE669A40F200817C
:103B2000B0EE447A402DC3ED006A83ED014A83ED87
:103B3000029A83ED037A83ED043A83ED064A83ED1E
:103B4000054A83ED084A83ED074A00F28D80F4EEC2
:103B5000C24AF1EE10FA40F39381F0EE647A1FED61
:103B60002C3A5FED2E6A01E0F0EE477AF4EEE67A49
:103B7000F1EE10FA37EEC37AF6DCB4EEE37AF1EE4A
:103B800010FA40F17A811FED363A5FED366A01E0B6
:103B9000B0EE677AB4EEE67AF1EE10FA77EE037AD9
:103BA000F6D4F4EEE57AF1EE10FA40F3098172EE04
:103BB000677A27EEA77AB0EE618AA7EE018ABCF198
:103BC000400F5FED436A1FED433AE8EE076A27EEC8
:103BD000877AF0EE458AE7EE267AB0EE457AE7EE90
:103BE000838AA7EEC37A87EE288A44D9B0EE447A56
:103BF000F6EE006AB7EE003AC5EE287A243383ED7C
:103C0000BE8A66EEA76A23EE273A67EE277AC3EDEF
:103C1000BA6AC3EDBC6A83EDBB3AC3EDBD7A83EDEE
:103C2000C04A83EDBF4A83EDC24A83EDC14ABB421D
:103C30007FF4D7AE0120A3E40023FFF771BB954BBF
:103C40008AF85F209B789FED947A6DE5F4EEC17A57
:103C5000F1EE10FA48BF74EEE77A18E6F0EE477A14
:103C60000DE6B0EE677AF8E5B7EE008ABCF1400FDA
:103C7000F0EE488ABAD8F4EEE54AF1EE10FA40F3D5
:103C8000F380F0EE407A9FED853ADFED856A01E042
:103C9000F0EE477AF4EEE67AF1EE10FA37EEC37AF8
:103CA000F6DCB4EEE37AF1EE10FA40F1DA809FED43
:103CB0007B3ADFED7C6A01E0B0EE677AB4EEE67A3B
:103CC000F1EE10FA77EE037AF6D4F4EEE57AF1EE3F
:103CD00010FA7FDD72EE677A27EEA77AB0EE619A6E
:103CE000A7EE019ADFED706AE7EE096A27EE273A40
:103CF000B8EE007AE3EE267AF6EE006A35EE673A21
:103D000027EE877A63EE266A76E7B7EE003A402818
:103D1000F0EE438AB0EE449AF0EE446A3FF600AF0C
:103D2000B4EEE56AF1EE10FA40F3A480F0EE607AAA
:103D3000DFED5A9A9FED5A8A01E0F0EE477AF4EEF1
:103D4000C87AF1EE10FA37EEE97AF6DCB4EEE37AEF
:103D5000F1EE10FA40F18B80DFED509A9FED518A21
:103D600001E0B0EE677AB4EEC87AF1EE10FA77EEC1
:103D7000297AF6D4F4EEE57AF1EE10FA46DD72EE29
:103D8000677A27EEA77AB0EE61AAA7EE01AA9FEDA7
:103D9000468AAAEE078A67EE879AB8EE007AE9EEBD
:103DA000887A67EE877A87EEA87ABBE69FED3F7A3E
:103DB000F4EEC77AF1EE10FA48BF73EEE77A90E6B8
:103DC0009FED3A7AF4EEC77AF1EE10FA48BF73EE3F
:103DD000E77AEEE69FED357AF4EEC77AF1EE10FA67
:103DE00048BF73EEE77A77E7FF23838140F2E93338
:103DF00002E0002B3FF45EAC0289013B12F0010FA0
:103E00009BB2F6D08389DBB2059355E49FED277A08
:103E1000F4EEC77AF1EE10FA48BF73EEE77AB0E736
:103E20001420F5F701FCCAF8180000283FF4A1AAF5
:103E3000FFF79BBA1E4B02931A46042382F888347C
:103E4000FFF763BAF7F774F9DAF8140026E4F7F726
:103E50006FF9FFF7D9BAF7F76BF9DAF81400FFF743
:103E6000B8BAF0EE477A30E7B0EE407A19E7F0EEF4
:103E7000477A7FE7B0EE607A68E7F0EE477A90E63F
:103E8000B0EE647A79E6F0EE477A22E6B0EE467A52
:103E9000C3E500BFCC9C00200000FA42DB0FC94004
:103EA000E4CB1641E4CB16C115A82ABEDB0FC9BF6F
:103EB000DC2C0020F0B5184E002383B00446082106
:103EC000D6F8200586F89D3002ADF6F76BFDD6F8E2
:103ED00020058121F6F766FD8923D6F8206525F8AF
:103EE000023DE71D14F8010B3246294611F072FD20
:103EF000BC42F7D1BDF806301A0A52FA83F3C3F177
:103F0000FF039BB23246D8B20021ADF8063011F063
:103F100061FD03B0F0BD00BFDC2C002038B5384B8C
:103F20005B68C3F30803CBB9EFF31183B3B9354A28
:103F3000354D364C1368A06811688B42FAD1296858
:103F40008842F7D8324A11684FF47A7202FB01F4C2
:103F5000241AB4FBF1F402FB034421E0EFF31181D6
:103F6000102383F3128803F1E023C9B298681A681A
:103F700012F4803F274A1EBF012010609868214B31
:103F80001D68136881F31188214A11684FF47A740F
:103F900004FB01F22B44121AB2FBF1F204FB0324DE
:103FA0001D4DD5F89830E31AB3F5FA6FC4BF00235E
:103FB00085F89C3095F89C301BB90023EB600120FC
:103FC00038BD00221549E86811F058F895F89C3082
:103FD00073B9134B1B781B2B04D1D5F82435114A28
:103FE000E31AD3800023C5F82445EB60012038BDD7
:103FF0000D48FFF75FFF002385F89C30E9E700BF1D
:1040000000ED00E0108A0020188A002010E000E097
:10401000148A00200C8A0020DC2C0020782D00203F
:104020000D88002010880020686B040838B50D4CFE
:1040300005460146D4F82805F6F7B4FCB4F82C057B
:10404000082380EA052041F2210210F4004F4FEAD4
:10405000400018BF5040013B80B2F6D1A4F82C05B7
:1040600038BD00BFDC2C002070B582B00446F6F7E6
:10407000EDF8964AD2F8303503F24C4383420CD324
:1040800092F834354BB1022B8ABF92F85D020520BD
:10409000023098420DDC02B070BD01210023C2F84D
:1040A000300582F85C4282F8341582F8583202B04A
:1040B00070BD591CC9B288421344D4BF01250025E4
:1040C00082F8341583F85C4282F85852E3DC92F8A7
:1040D0005E520023162D82F83435DCD06B002906A1
:1040E00048BF83F0D503DBB213F0800F4FEA4303E0
:1040F00018BF83F0D503DBB213F0800F4FEA430300
:1041000018BF83F0D503DBB213F0800F4FEA4303EF
:1041100018BF83F0D503DBB213F0800F4FEA4303DF
:1041200018BF83F0D503DBB213F0800F4FEA4303CF
:1041300018BF83F0D503DBB213F0800F4FEA4303BF
:1041400018BF83F0D503DBB292F85D4213F0800F05
:104150004FEA430318BF83F0D503022CDBB247D9E3
:104160005B490C44023111F8016F734013F0800F6A
:104170004FEA430318BF83F0D503DBB213F0800F7F
:104180004FEA430318BF83F0D503DBB213F0800F6F
:104190004FEA430318BF83F0D503DBB213F0800F5F
:1041A0004FEA430318BF83F0D503DBB213F0800F4F
:1041B0004FEA430318BF83F0D503DBB213F0800F3F
:1041C0004FEA430318BF83F0D503DBB213F0800F2F
:1041D0004FEA430318BF83F0D503DBB213F0800F1F
:1041E0004FEA430318BF83F0D5038C42DBB2BAD148
:1041F000104490F85B1299427FF44DAF7A2D2AD08B
:1042000022D97C2D27D07D2D7FF445AF92F86132E5
:10421000042B4AD0052B34D0032B7FF43CAF92F80B
:10422000633292F862222B482B49202BA8BF20230F
:10423000092AA8BF092280F8292180F82A310A72A8
:104240004B7217F031FD26E7282D7FF424AF234B66
:1042500001221A701FE7224A136E572B3FF71BAF3C
:10426000204921480D684C680821995413440121C4
:10427000C3F80150C3F80540136E0170093313668B
:1042800009E71A4B1B78EBB1124C012194F8292154
:1042900004F5907032F0C2FA154B164A1B680121E2
:1042A0002D3384F82B111360F5E6104B1B78002B8F
:1042B0003FF4F1AE02A9002301F8013D064815F0D4
:1042C0005DF8E8E617F0F0FCE5E600BFDC2C002026
:1042D000382F002024580020505900202158002059
:1042E000685900203D2F002022580020A470002093
:1042F000108A0020EC6D00202DE9F04FDE4C94F880
:1043000070338BB023B9002318460BB0BDE8F08F93
:1043100094F8473394F846030022012B84F8702365
:1043200045D094F85053023D15F0FF0500F09F81F1
:1043300004F554710D444FF6FF7311F8012B9B1ACD
:10434000A9429BB2F9D11A0A204490F84F13914226
:10435000D9D190F84E23DBB29A42D4D194F84833A5
:10436000202B40F07D8194F84C138B1C09938B1DFE
:10437000019301F10803029301F10A03039301F190
:104380000C03049301F10E03059301F1100306934E
:1043900001F11603079301F1180301F1040A01F179
:1043A000120801F11407089301F11A0BAFE094F819
:1043B0004C13B4F84AE38B1C671854FA83F609933C
:1043C00001F1040A97F8503397F851C396F8505307
:1043D00096F8517354FA8AF673448A1D96F851E39D
:1043E00001921D4496F8503354FA82F605EB0C25E1
:1043F00001F1080296F851C302922B4496F85053EB
:1044000054FA82F603EB072301F10A0254FA82F709
:104410002B4496F85053039203EB0E2301F10C0248
:1044200097F851E396F8516304921D4497F850337E
:1044300054FA82F705EB0C2501F10E0254FA82FCC6
:104440001D4497F85033059205EB062501F1100243
:104450009CF8506397F851739CF851C306922B4413
:1044600054FA82F503EB0E2301F1120895F851E39B
:10447000334495F8506354FA88F503EB072301F1B0
:10448000140795F85193334495F8506354FA87F51F
:1044900001F1160203EB0C23334495F850C3079245
:1044A00054FA82F603EB0E2301F1180295F85153EA
:1044B0000892634496F850E396F851C303EB09233E
:1044C00054FA82F6734401F11A0B96F850E396F809
:1044D000516303EB052354FA8BF52044734495F89C
:1044E00050E390F84F9395F8515390F84E0303EB37
:1044F0000C239E440EEB062E0EEB052E00EB092935
:104500001FFA8EFE1FFA89F9F1457FF4FCAE099B74
:1045100054FA83F2019B54FA83FC029B9CF851935A
:104520009CF850C354FA83F30193039B54FA83F627
:10453000049B54FA83F5059B54FA83F0069B54FAC6
:1045400083F3029354FA88F30393079B92F8518301
:1045500092F8502354FA83F321440593089B54FAAC
:104560008AFE54FA87F791F851A391F850130497F3
:1045700054FA83F39EF8517306939EF850E3019B1F
:1045800001EB0A2102EB08220EEB072E93F8518370
:1045900093F85073C4F8081396F8513301930CEB59
:1045A0000921C4F8141395F851C396F8506395F88F
:1045B0005053019BC4F80C2306EB0326049B029A7C
:1045C000C4F810E393F851E393F8503392F8519301
:1045D00092F85013039A019603EB0E23C4F830337C
:1045E000059B90F851A3019E90F85003C4F81C63FA
:1045F00007EB082701EB092192F8518392F8502329
:1046000093F85163C4F8281354FA8BFB93F85013B2
:10461000069BC4F8187305EB0C2500EB0A2002EB8F
:104620000822C4F82053C4F8240393F851539BF88C
:104630005103C4F82C2393F850239BF8503301EB1B
:10464000062103EB0023C4F83413C4F83C330123E0
:1046500002EB05221846C4F838230BB0BDE8F08FF2
:10466000064810F041FA002384F845034CE6FF2287
:104670004FF6FF7368E600BFDC2C00202C300020D2
:10468000F8B5F5F7E3FD274E054600F1FA07344685
:1046900096F8F83306EB8303D3F8D803F6F70CFC4F
:1046A00038BB94F8F83304EB8303D3F8D803F6F758
:1046B00003FC28B3F5F7CAFDD4F83C35401B9842FB
:1046C000C4F838052BD805F5FA7594F8F83304EBDF
:1046D0008303D3F8D803F6F7EFFBB0B994F8F833B7
:1046E00004EB8303D3F8D803F6F7E6FB90B1002080
:1046F00005E0F5F7ABFDB842CAD94FF0FF30F8BD81
:10470000F5F7A4FDB842CCD9F7E7F5F79FFDA8422D
:10471000DBD9F2E7F5F79AFDA842DFD9EDE70120F2
:10472000EDE700BFDC2C002038B5002405460470FE
:10473000FFF7A6FF431C11D0012803D12B78A0401E
:10474000184328700134082CF2D1054A2B7892F8CE
:1047500040154B4082F84035012038BD0020FCE771
:10476000DC2C00202DE9F843204C214D266807461B
:104770000236A84695F8F83305EB8303D3F8D8033F
:10478000F6F79AFB10BBF5F761FD00F12706F5F788
:104790005DFD8642FBD800252C464FF0010998F8B4
:1047A000F83308EB8303D3F8D803F6F785FB18B189
:1047B00009FA05F31C43A4B2092D06F134060BD007
:1047C000F5F744FD8642FBD80135E8E723689E42B1
:1047D000D0D80020BDE8F88340F201232340B3F590
:1047E000007FF6D164083C700120F3E7108A0020B6
:1047F000DC2C002037B502ADFF2305F8013D04464F
:104800002846FFF7AFFF00B91CB99DF8070003B0B9
:1048100030BD013CF4E773B5204C002284F8F92345
:1048200084F8FA2384F8412584F842250144FF22C4
:104830008DF807200546CEB22846FFF793FFF8B162
:1048400015F8010BFEF766FCEBB2B342F4D194F815
:104850004335EBB11248FFF785FF88B11148FFF7E8
:1048600081FF68B10DF10700FFF77CFF40B1B4F89C
:10487000F923B4F841359A4202D0C2238DF80730AB
:104880009DF80700A0F130035842584102B070BDB6
:104890000DF10700FFF766FFF2E700BFDC2C0020F8
:1048A0001D3200201E32002070B5194C94F8F833E8
:1048B0000D4604EB8303013D0646EDB2D3F8D80361
:1048C0002AF0F6FC0135002384F8F93384F8FA3332
:1048D00035443078FEF7FCFB16F8010BFEF71AFCA6
:1048E000AE42F6D194F843353BB194F8F903FEF7A4
:1048F000EFFB94F8FA03FEF7EBFB94F8F83304EBC4
:1049000083042021D4F8D803BDE87040F6F7AEB98F
:10491000DC2C002013B5FE23ADF8043000238DF805
:10492000063003788DF80730044613B901238DF85B
:10493000063004210DEB0100FFF7B6FF0220FFF760
:1049400059FFFF280CD121786068FFF7ADFF2820C0
:10495000FFF750FFA0F130035842584102B010BD9C
:104960000020FBE737B5054608461446FFF7D2FF9F
:1049700078B10123022101A88DF805308DF804508B
:10498000FFF792FF2046FFF735FFA0F130035842B2
:10499000584103B030BD07B50E4B0268934317D0A2
:1049A000FF230421ADF8043043788DF80630837876
:1049B0008DF807300DEB0100FFF776FF0220FFF7BF
:1049C00019FFA0F130035842584103B05DF804FBD1
:1049D0000120FAE700FFFF0037B5054608460C4600
:1049E000FFF7D9FF60B123788DF80450022101A8A8
:1049F0008DF80530FFF758FF21786068FFF70BFF4F
:104A000003B030BD10B5064CD4F82805F5F7C6FF45
:104A10000028F9D0D4F82805BDE81040F5F7B6BF56
:104A2000DC2C002010B5FFF7EDFF0A4AB2F847353D
:104A300083EA00239BB2082141F2210413F4004FC2
:104A40004FEA430318BF634001399BB2F6D1A2F885
:104A5000473510BDDC2C002038B50B4B03EBC004F0
:104A60000D4694F82822094803EB8203D3F84C1131
:104A70001AF083F994F82E322BB1691C0448BDE872
:104A800038401AF07AB938BD246A040883A20408B1
:104A9000A4ED0408F8B50C4C0C4E0D4F04F5387518
:104AA00020681AF07FF9616811B130461AF065F993
:104AB000A16811B138461AF060F910341AF00BFAF7
:104AC000AC42EDD1F8BD00BF146D04087AA2040811
:104AD00080A204082DE9F04F002489B08346924655
:104AE0000D4626464FF019094FF46178BAF1000FD0
:104AF00022D004EB84030AEB03070522394628463B
:104B0000079331F063FE3A79079B19FB0282049206
:104B1000FA781AF8033019FB02820392BA780292EB
:104B2000B0FA80F67A78019276090093104A23460B
:104B3000314658461AF0B2FA2B790D4A19FB038315
:104B40000493EB7819FB03830393AB7802936B78A0
:104B5000019315F8053B009331462346584601342E
:104B60001AF0B4FA0A2CC1D109B0BDE8F08F00BF29
:104B700086A204087FB5094B0493094B0393094BA4
:104B80000293094B0193094B0093094A094B0A49C7
:104B90000A481AF023FA07B05DF804FBDCA2040807
:104BA000E1A20408EBA20408F4A2040800A304088C
:104BB0009CA20408C39B0020A6A20408B1A204087A
:104BC000044B054A05491B681268096804481AF035
:104BD00005BA00BF187AFF1F147AFF1F107AFF1F53
:104BE00006A3040870B5374C37481AF0DBF894F880
:104BF0002530012B60D13548354E1BF09BF994F8D8
:104C00002A3013B194F8273013B194F8263043B901
:104C1000B6F898502F481AF0C5F88DBB2E481BF0F7
:104C200089F92E482E4D1AF0BDF894F8293005EB7D
:104C30008303D3F8D0051AF0D1F9B6F894102948B7
:104C40001AF09BF894F826302BBB27481BF072F91A
:104C500026481AF0A7F894F82A3005EB8305D5F812
:104C6000D8051AF0BBF9B6F8961021481AF085F865
:104C700094F82A309BB91F48BDE870401BF05AB920
:104C80004FF47A72B5FBF2F102FB115292B21A485C
:104C90001AF0A4F9C5E719481BF04CF9D8E794F8C5
:104CA000273023B91648BDE870401BF043B91548BA
:104CB000BDE870401BF03EB91348BDE870401BF0E2
:104CC00039B900BF3CB200201AA3040830A304087D
:104CD0008CBB002037A3040852A3040864A3040873
:104CE000246A04087AA3040897A30408A7A3040865
:104CF000C2A30408E5A304085CA304089EA3040857
:104D000098A304089FA30408EAA304082DE9F84324
:104D10001AF0E1F81748184D1BF00CF914242D2156
:104D2000D5F84C05F6F75EFB013CF8D11AF0D3F844
:104D3000124D134E134FDFF854802B7EE11006EB1B
:104D4000830304F0070201313846D3F84C911AF07E
:104D500014F86A7E49464AB10B481AF03FF901340B
:104D6000102C05F12005E8D1BDE8F88340461AF083
:104D700035F9F4E7F8A30408DC2C002040240020D7
:104D8000246A04080EA404081FA404089FAA0408A7
:104D900038B50D46F8F7DEFB0C4B1978884204460F
:104DA00005D201460A481AF019F9204638BD2DB13E
:104DB000FF2803D107481AF011F9F6E70139064830
:104DC0001AF0EAF84FF0FF34EFE700BFAD480020DB
:104DD00026A4040837A404084AA404082DE9F04FC7
:104DE000354C87B08046354A2378608802EB8303D0
:104DF000D3F84C91F8F796FDD0E901A30493304B1A
:104E000093F8503513B9CDF810A09A4608F0400336
:104E1000DFF8B8B005930026A379002B08BF012363
:104E20009E4206DB274B08349C42DCD107B0BDE82C
:104E3000F08F6279237906FB0323049A0136D55C4F
:104E4000BAF1000F11D1B5FA85F77F090DB305F05E
:104E50000F032D0940350293CDE900654B465A46B4
:104E6000394640461AF032F9D6E71AF80330EA1A02
:104E700057425741C3B103F00F021B09403302925E
:104E8000CDE900635A464B46394640461AF006F9CA
:104E9000DCE7059B002BBFD100964B460A4A3946FA
:104EA00040461AF013F9B7E700964B46064A3946D2
:104EB00040461AF0F3F8C9E74C6C0408246A040869
:104EC000DC2C0020146D040885A404086FA40408D9
:104ED0002DE9F04F6B4BDA7891B09846002A00F03C
:104EE000A68069481BF026F80025DFF8B0A1DFF89E
:104EF000C4B10795A94608A9E8B224F099FC9DF829
:104F00002830002B6CD0022D0C9C40F09D80002C92
:104F100000F0918007EE904ADFED5C6AF8EEE77AE8
:104F200086EEA77AFDEEC77A17EE906A9AF8524598
:104F3000089B012C40F2818096FBF4F41A46022172
:104F4000534819F01AFF0D9A002A00F0918041F29F
:104F5000883002FB04004FF47A73B0FBF3F00F9B30
:104F6000002B00F0878041F2883103FB04114FF4DD
:104F70007A7CB1FBFCF1062D03D0079F0F448144DE
:104F8000079798F803C0BCF1000F75D04FF47A7CF6
:104F90000E9FB7FBFCFCCDF810C04FF00A0C91FB44
:104FA000FCFE0CFB1E11CDE902E190FBFCF10CFBB9
:104FB0001100CDE90010214636481AF00FF8022DF5
:104FC00008D19AF85235012B04D93246099958462E
:104FD0001AF004F8304A342303FB05230022DA6276
:104FE0000135182D87D198F80330EBB12B49D1F852
:104FF0005C25D1F85805D1F8601552094FF47A7341
:10500000B0FBF3F3264819F0E9FF0798079B0A2243
:1050100093FBF2F302FB130799FBF2F1009702FBFB
:105020001192204819F0DAFF11B0BDE8F08F1E4848
:105030001AF080FF58E7264678E7099A1B480221B4
:1050400019F09BFE34467EE75CB107EE904ADFED37
:105050000F6AF8EEE77A86EEA77AFDEEC77A17EECA
:10506000904A089A0A48294619F087FE00266AE7FE
:10507000104674E719467EE721460D4819F0AEFF49
:105080009DE700BFBC9B002099A40408002474493C
:10509000EEA4040810A5040800020020DC2C002067
:1050A00044A5040864A50408E4A40408FDA40408B5
:1050B00040A5040834A504082DE9F0476A4B6B4865
:1050C000196890B04FF47A73B1FBF3F119F086FFD1
:1050D00005A8F7F7E1FE58B1654A05A90023B2F922
:1050E000002008A8F7F7FCFE08A9624819F076FF2F
:1050F000614B624D1B78624A6249127809886248A6
:10510000DFF8E4A105EB830305F5BF69D3F8E435C7
:1051100019F064FF5D4B5E4819685E4BB1FBF3F11B
:1051200019F02BFE24F08AF84FF47A725A4BB0FB38
:10513000F2F102FB1102B3F900300A2092B289B2F7
:10514000B2FBF0F2554819F018FE554BD3F8008029
:10515000002405F5C36559F82470A300D7B10126D2
:10516000A64016EA080F13D0F20611D01AF8042050
:105170005B594C4853F82220394619F0FEFD022EA7
:1051800006D1494B93F8211011B1484819F0F5FDAB
:105190000134E0E719F09FFE454A46494648474C2E
:1051A00019F01CFF464A474B4748D31A3946B4F812
:1051B000642519F013FF4549D1F88420002A42D014
:1051C00007EE902ADFED426AB8EEE77AC6EE877AFC
:1051D000FDEEE77ACDED037AB4F866355BB107EE04
:1051E000903ADFED3B6AF8EE677A86EEA77AFDEE3D
:1051F000C77A17EE903AC96959B107EE901ADFEDF8
:10520000346AF8EEE77A86EEA77AFDEEC77A17EEF3
:10521000901AB4F868052F4E2F4F6428CDE900315D
:105220000146039B2D48A8BF642119F0D7FE2C48E6
:1052300019F0B8FD2B4B1C68012534B919F04BFE51
:1052400010B0BDE8F0870392C6E794FAA4F3B3FA6E
:1052500083F305FA03F256F82310384624EA0204D1
:1052600019F08BFDE9E700BF108A002092A5040821
:105270001C710020ACA50408F8540020246A04081E
:105280000A52002004520020BDA5040884A5002075
:10529000E3A5040840420F00F2720020F3A50408C1
:1052A0008052002014A60408405200201CA60408C6
:1052B000F0FF01200008000020A60408DC2C0020DC
:1052C000008000080040000844A6040800020020F6
:1052D00000247449188E04089FAA04087EA60408B6
:1052E000C4A60408905400202400002038B5114DB5
:1052F0000446204619F012FC60B10F4B0F4893F999
:105300000A104B1C0ABF0E4BC9B25978BDE8384091
:1053100019F064BE2046F8F71DF9052804D8C0B27C
:1053200023F08CFE2C46E4E705210648BDE8384012
:1053300019F032BE36EF040820000020DAA6040877
:10534000BC9B0020E9A60408052838B50D460FD8F7
:10535000084CA07208481AF06DFF0848FFF7C6FF16
:1053600019F0B9FD2946102019F0BAFDFF23A372E8
:1053700038BD00BF2000002009A7040836EF04084C
:1053800038B5114D0446204619F0C8FB60B10F4BEB
:105390000F4893F90B104B1C0ABF0E4BC9B219787A
:1053A000BDE8384019F01ABE2046F8F7D3F80228B5
:1053B00004D8C0B2F3F764FC2C46E4E702210648A7
:1053C000BDE8384019F0E8BD36EF040820000020A1
:1053D000DEA60408BC9B0020EEA604082DE9F74FCA
:1053E0003B4B3C4C1A785B780090E272A3721AF047
:1053F00043FFF8F785FA0025DFF8DCB0A8460D2753
:10540000354B00996F43DE19D6F800904846F7F700
:10541000F7FF00283DD0B8F1000F01D019F05BFD77
:1054200049462E485F4419F0A8FC0021304619F087
:1054300047FD19F050FD3B7903F01803082B3BD0D2
:10544000102B3DD0304619F0D8FD0D2303FB05B3DA
:10545000B3F80900F8F766FA0746C0B1304619F00C
:10546000AAFBD7E90121824602440144304619F0E3
:105470002AFC60B901904946194819F07EFC796808
:10548000019A5144304619F09DFC19F024FD08F1B1
:105490000108013540F267139D42B0D11AF0D6FEE3
:1054A000FF23E372A372B8F1000F0DD10D4803B0D2
:1054B000BDE8F04F19F070BD0B48FFF761FFC1E781
:1054C0000948FFF713FFBDE703B0BDE8F08F00BF49
:1054D000BC9B0020200000202877040859ED040818
:1054E00015A7040825A7040836EF0408022838B5D4
:1054F0000D460FD8084CE07208481AF09BFE084889
:10550000FFF73EFF19F0E7FC2946082019F0E8FCF8
:10551000FF23E37238BD00BF200000200DA7040860
:1055200036EF040838B5044619F0F8FAA0B3244B56
:10553000DB680133172B25D822490C2202FB03120A
:105540001C46D2F8345655B91E4A0C210134172C8A
:105550001ADD002401FB0420D0F83456ADB1184BFD
:10556000DC6024F05DFD2A462146174819F036FD1F
:10557000144B0C2202FB043494F82C06BDE838408E
:1055800024F068BD1C46DFE7E4D99C42DED10F4819
:10559000BDE8384019F000BD2046F7F7DBFF1728BB
:1055A000044607D8074A0C2303FB0023D3F83456DC
:1055B000002DD4D121460648BDE8384019F00EBD73
:1055C00020000020246A04085CA7040832A704080D
:1055D00046A704082DE9F341054619F09FFA044651
:1055E00020B119F0F7FC02B0BDE8F081284601AA0D
:1055F0002A49DFF8A8802FF052FD274605462646A7
:1056000075B9022CEDD1A7F57A73B3F57A7F1FD95E
:105610004FF4FA624FF47A71214819F0D3FCE2E7B3
:105620004CB1012C0FD001AA414600202FF037FDCC
:1056300001340546E4E701212846FFF7A9FB431C96
:105640000646F0D1CFE72846F7F784FF0746EAE79A
:10565000B8B21DF01BFDFF2EBCEEC00A114B0BD1E2
:10566000114AF8EE407A1278AA4212DC10EE101AB3
:105670000E4819F0B3FCB6E7F8EE407A03EB860368
:1056800010EE102A31460A48C3ED007A19F0A6FC44
:10569000A9E7E3EC017A0135E6E700BF5FDF040824
:1056A000FEAB040848320020AD4800207EA7040865
:1056B00071A704082DE9F04F014691B006468648CF
:1056C000864D19F08BFC864B8649C3F800D0002329
:1056D0002B70854B097840241C700622012330462C
:1056E00023F054F80A20F4F7A7FF2B78DBB20C2B39
:1056F00040F2ED809DF80C90B9F1FE0F2ED0B9F17B
:10570000FF0F15BF0F241524002601269C4240F0F0
:10571000DE80611EC9B268460EF02CFD10AB1C4441
:1057200014F8413C834240F0CE8006F1FF38B8F1D6
:10573000010F9DF80D4013D904F01F07650961376B
:105740004C466A4819F02EFB022E71D0013D042D03
:105750006AD8DFE805F00A5D616965000226D5E7D1
:105760009DF80E709DF80F50EBE761481AF0E2FBD0
:105770006048DFF8D491DFF8D4B119F013FB0025AD
:105780004FF0030A1DF805104846013519F0F5FAE7
:105790000C2D55D119F09FFB022E5BD06422B4FB77
:1057A000F2F102FB11423B46D2B2C9B2524819F0A3
:1057B00015FC5FFA88F8B8F1010F7BD84F4A504BBF
:1057C0009DF810104F48504D00290CBF1146194646
:1057D00019F004FC9DF811104C4B4D4800290CBFEA
:1057E0002946194619F0FAFB022E63D19DF81240A2
:1057F000484819F0D7FA9CB3FF2C41D00A22B4FBD9
:10580000F2F102FB1142D2B2434819F0E7FB2AE061
:1058100042481AF08FFBABE741481AF08BFBA7E731
:1058200040481AF087FBA3E73F481AF083FB9FE745
:1058300000230DF11F008DF83F301AF07BFB97E736
:1058400095FBFAF303EB43039D429BD1584619F0B5
:10585000A9FA97E73A462146344819F0BFFBA8E772
:1058600028461AF067FB9DF81340314819F09AFA60
:1058700054B1FF2C21D021462E4819F0AFFB06E091
:105880002D481AF057FBEEE71F481AF053FB1E4D48
:105890001E4E294F00240DEB04031A7D8AB1FF2A06
:1058A00014BF32463A4621462448013419F096FB8B
:1058B000042CF0D111B0BDE8F08F1F481AF03AFB6C
:1058C000E5E72A46EFE71E4819F066FBF2E71D48B8
:1058D0001AF030FBEEE700BFADA70408CA4800206D
:1058E000BC480020AD480020CB480020BEA70408DB
:1058F000C9A70408F7A704080EA8040896A7040877
:105900008DA7040845A804089DA70408BEAC040898
:105910005CA8040863A8040877A80408D0A70408B2
:10592000D8A70408E0A70408EFA704082AA80408D9
:105930007FA80408A5ED0408A1A704088FA80408FF
:105940009AA80408AAA8040809A804082BDC0408DB
:105950002DE9F74F054619F0E1F8044618B9374B21
:105960009B78042B04D819F035FB03B0BDE8F08F09
:1059700001AA3349DFF8E080DFF8E090DFF8E0A02B
:1059800028462FF08CFB0127264640B92D4B2E4A86
:105990001B689B1A2D4A18BF01231370E5E766B9EF
:1059A0000121FFF7F5F9421C0446DED001AA244983
:1059B000002001362FF073FBE7E7F7F7CBFD2F2828
:1059C000054636D807B323F0CFF8062D0CD10520B5
:1059D000F4F732FEDAF800301B0126D5FF2C20D078
:1059E000E0B2FFF767FE09E00120F4F725FE184951
:1059F0000123EAB20978E0B222F0C8FE29464846FF
:105A000019F0ECFA0027D1E70628F0D1E2E7FFF71A
:105A100051FE9BF80030F8B2834207F10107F6D837
:105A2000ECE70027DFF828B0F3E70A481AF082FA1B
:105A3000E4E72F21404619F0AFFAB7E788A5002028
:105A40005FDF0408A4A50020497D030838B20020C8
:105A5000AD480020B3A80408D3A80408C2A80408CD
:105A600084A3002013B5204C237C022B2FD10123CB
:105A70000DF10702F52104F11000F5F775FB40B3B5
:105A80009DF80710194819F0A9FA237C022B22D19E
:105A900001230DF107029A211548F5F765FBE0B1E6
:105AA0009DF80710134819F099FA237C022B16D1A0
:105AB00001230DF107029B210D48F5F755FB80B13D
:105AC0009DF807100C4819F089FA02B010BD0021AA
:105AD000D8E70146D6E70021E4E70146E2E70021E6
:105AE000F0E70146EEE700BFFC9C0020F3A80408A5
:105AF0000C9D002006A9040819A90408024BD3F83C
:105B00008C0515F0CBBD00BFDC2C00200A4C08B57D
:105B100005460A4819F046F9D4F84C05F5F754FC47
:105B2000D4F88C0524F036F81DF024FB0DB1F8F7FD
:105B3000A5FFFAF7A7FF00BFDC2C00202CA9040862
:105B4000094C0A4808B51AF075FB94F890250AB17B
:105B5000F3F7BAF994F891350BB1F3F795F9FAF731
:105B600059FC0020FFF7D2FFDC2C002038A90408E4
:105B70000A4D0B4808B51AF05DFBD5F84C05F5F752
:105B800023FC084B002485F89245C5F894461C7008
:105B90001DF07EFC2046FFF7B9FF00BFDC2C002083
:105BA0003FA90408DC530020034808B51AF042FB63
:105BB0000120FFF7ABFF00BF66A904082DE9F04FF5
:105BC0004A4085B098461D4FD34306460D460024F3
:105BD0000393204624F012FA0E9B184228D0039B10
:105BE000174ADFF860A0034214BF4FF001094FF0DD
:105BF000000910EA050302934FF00C0303FB042392
:105C00004946D3F808B0CDF800B014BF3A46524622
:105C10004346304619F042FA029ACDF800B04346A6
:105C2000002A14BF52463A464946304619F04EFA09
:105C30000134172CCDD105B0BDE8F08F7EEE0408FD
:105C40005070040884A90408F8B5084F4D1E064694
:105C500001F11F0415F8012F30463946F7F7A8F86F
:105C6000A54206F10206F5D1F8BD00BF09A8040857
:105C70002DE9F0419AB007462EF0B4FA01AD064680
:105C800020220021284630F0C9FD16B3402E07D04F
:105C9000402231462D4819F07FF91AB0BDE8F08155
:105CA0000024A046022207EB4401684630F0F4FDD0
:105CB0000023102209A968468DF80280F7F7D2FB6D
:105CC000099B0DF1020293421FD128550134202C6B
:105CD000E8D14122002109A830F0A0FD1C4C46B3B8
:105CE00094F89836B3B1202204F29961284630F036
:105CF0006DFD78B104F2996109A8FFF7A5FF09AA23
:105D00001449154819F048F9C7E71978134819F0EC
:105D100043F9C2E72846F3F769F80123104984F8EC
:105D2000913509A8FFF790FF09A90E4819F056F917
:105D3000B3E794F891351BB994F89836002BF3D05B
:105D4000074909A8FFF780FFEEE700BF8BA9040809
:105D5000DC2C0020C9A90408D3A90408ADA90408B3
:105D600075330020FDA9040870B505462EF03AFAF7
:105D7000064600B3134C94F8B9369BB104F2BA60EE
:105D80002EF030FAB042024605D1294604F2BA603C
:105D900030F070FD60B10C4A0C490D48BDE8704010
:105DA00019F0FAB80422294604F2BA6030F074FD02
:105DB000012384F8903504490648BDE8704019F085
:105DC0000DB900BFDC2C0020963300200AAA04087D
:105DD000D3A904081AAA040870B505462EF002FAE1
:105DE000064600B3134C94F8B9369BB104F2BF6079
:105DF0002EF0F8F9B042024605D1294604F2BF6000
:105E000030F038FD60B10C4A0C490D48BDE87040D7
:105E100019F0C2B81422294604F2BF6030F03CFDEC
:105E2000012384F8903504490648BDE8704019F014
:105E3000D5B800BFDC2C00209B3300202DAA04081D
:105E4000D3A9040838AA040870B506462EF0CAF98A
:105E5000124C054690B111220021204630F0DEFCA4
:105E60002A460F49304630F005FD38B1102D2A463C
:105E7000314628BF1022204630F00EFD2378074A15
:105E8000002B08BF0121064B1CBF00211346012037
:105E9000044ABDE8704019F019B900BFD87200205B
:105EA0002BDC04083EAA04082DE9F04F8BB0834692
:105EB00018F034FE044638B100224B490120FEF7A9
:105EC00009FE0BB0BDE8F08F5846F7F743FB0928F1
:105ED000054600F38380860037180BF10100DFF8D8
:105EE00014A18DF81F4018F021FE0AF2D468544620
:105EF00008EB07098346C24658B1F7F72BFB0D287C
:105F000007D8E31983F8D4069DF81F3001338DF8C4
:105F10001F30584618F00AFE834660B1F7F71AFBA7
:105F2000052808D87319234483F8D5069DF81F3037
:105F300001338DF81F30584618F0F8FD834660B1E4
:105F4000F7F708FB082808D87319234483F8D60606
:105F50009DF81F3001338DF81F30F91C0DF11F0221
:105F60005144584618F0EFFD9DF81F20052A2DD109
:105F7000002308A9484608938DF8243030F026FC09
:105F80007319234493F8D51618B1F9B193F8D6369E
:105F9000E3B12E4434444FF4617094F8D8261923A9
:105FA00013FB0202049294F8D72613FB0203039317
:105FB00094F8D6360D4ACDE90113002194F8D43671
:105FC000009308462B4619F081F87AE7002348F839
:105FD000073089F8043018F0FDFF72E709222146E6
:105FE000034818F0EFFF6CE7B033002086A20408E6
:105FF00046AA0408DC2C00207F2810B5044607D9E7
:1060000064F07F00C0B2E40916F008FB7F2CF7D8DB
:10601000E0B2BDE8104016F001BB00BF38B5194D25
:106020000446472016F0FAFAD5F808371B0305D5C1
:10603000D5F800341868201AFFF7DEFF124CA07C58
:10604000FFF7DAFFD5F80C372068C01A16F0A1FB6D
:10605000D5F810376068C01A16F09BFBA068FFF7F0
:10606000CBFFA089FFF7C8FFE089FFF7C5FFD4E9A0
:106070000023A17C85F81C17C5F81427C5F818372C
:1060800038BD00BFDC2C002098540020F0B52B4C0C
:106090002B4DD4F82C77D4F830672A492A48D4F805
:1060A000203794F828272D78097890F82000B742F7
:1060B00085B027DB84F83857C4F8343784F83907BB
:1060C00084F83A1784F83B2701AD532016F0A6FA5E
:1060D000D4F83407FFF790FF94F83807FFF78CFFE8
:1060E00094F8391794F83A2794F83B3703932846E5
:1060F000CDE9011216F09AFA0023C4F82C370120DA
:1061000005B0F0BDD4F834678DF80850B3428DF86F
:106110000B2001938DF809008DF80A1001AD04F2EF
:10612000347204D095E8030082E80300CDE7696883
:1061300053689942F6D10020E2E700BFDC2C002032
:10614000B05400205D5C0020E05100201E4A1F4B2F
:10615000116800221F29C3F83C27A3F84027A3F8A1
:106160004227A3F84427C3F82C2723D03F291CD06B
:106170004FF4FA42B2FBF1F1A3F846171448B3F911
:106180004627018829B1914201DD1F2A17DC92FBC5
:10619000F1F1A3F8481781780E48003118BF0121AA
:1061A0001202C3F83027017070474FF40072A3F851
:1061B0004627E3E74FF48062A3F84627DEE7012194
:1061C000A3F84817E7E700BF88BB0020DC2C0020BD
:1061D000C0540020A26D0020194BB3F84027D3F81B
:1061E0002C07D3F83C1710B40132B3F9464792B2EA
:1061F00001300131A242C3F82C07C3F83C17A3F8C1
:1062000040270FDAB3F84427B3F948175DF8044B79
:10621000013292B28A42A3F84427A4BF0022A3F815
:1062200044277047B3F842275DF8044B0021013240
:10623000A3F84227A3F84017A3F84417704700BFFC
:10624000DC2C0020F0B5A44C04F24C738FB093ED1D
:10625000000A2EF0CFFF04F5EA6393ED000A05462D
:106260002EF0C8FF0646402016F078F9002858D1D5
:106270009A4AD4F8543757784F2B00F2F184DFE86C
:1062800013F01F0411040704F303EA03E003D60329
:10629000CC0346043C0432042804BD045004C80462
:1062A000C203BB03B103A7039D03900382037403DE
:1062B0006603550344033303250317030903FB0255
:1062C000A9029D02920286027B02700265025902B7
:1062D0004D02410235022A021F0213020502FA0191
:1062E000EF01E401D901CF01C501BB01B101A70153
:1062F0009D01930188017D016701200116010C01B8
:106300000201F800EE00E400DA00D000C600BC0094
:10631000B200A9009F00940089007C006F00620019
:10632000530000200FB0F0BD6D4B6E49D3F898209C
:106330006D48FCF723FFD4F8543701330020C4F82C
:1063400054370FB0F0BD664A6849B2F896306848D5
:10635000B2F89420FCF712FFD4F854370133EDE77C
:10636000644A624992F82A30634892F82920FCF77F
:1063700005FFD4F854370133E0E75E4A5B4992F8F1
:1063800027305E4892F82620FCF7F8FED4F8543700
:106390000133D3E7574B534993F828205848FCF76B
:1063A000EDFED4F854370133C8E7524B4D4993F80A
:1063B00025205448FCF7E2FED4F854370133BDE7FA
:1063C000514B48491A685148FCF7D8FED4F8543765
:1063D0000133B3E7927843494D48FCF7CFFED4F838
:1063E00054370133AAE74B4B3E49DA894A48FCF758
:1063F000C5FED4F854370133A0E7464B39491A8813
:106400004648FCF7BBFED4F85437013396E7414BBE
:1064100034499A784248FCF7B1FED4F85437013336
:106420008CE73C4B2F491A793E48FCF7A7FED4F87D
:106430005437013382E72F4B2A491A7A3A48FCF73E
:106440009DFED4F85437013378E72A4B25491A7F4B
:106450003648FCF793FED4F8543701336EE7254BEA
:1064600020499A7E3248FCF789FED4F8543701332C
:1064700064E7204B1B491A7E2E48FCF77FFED4F8B8
:10648000543701335AE794F8702716492A48FCF725
:1064900075FED4F85437013350E794F86327114957
:1064A0002648FCF76BFED4F85437013346E7244BFB
:1064B0000C495A792348FCF761FED4F8543701336C
:1064C0003CE794F80B2407491F48FCF757FED4F823
:1064D0005437013332E700BFDC2C0020BC9B002086
:1064E0008CBB0020A5ED0408C8B2040870B20408F3
:1064F000ACB204083CB2002090B2040878B20408A0
:1065000058B2040844B20408A070002038B204084D
:106510002CB2040888A5002018B2040808B20408A8
:10652000F4B10408E0B10408CCB10408B0B1040827
:1065300094B1040880B1040868B1040858B1040893
:106540005C5A002048B1040838B104080000C84271
:10655000B4F808341FED037AA449A54807EE903A31
:10656000F8EEE77A67EE877AFDEEE77A17EE902A83
:10657000FCF704FED4F854370133DFE69D4A9E4908
:10658000538A9E48D289FCF7F9FDD4F85437013379
:10659000D4E6984A9849138A99489289FCF7EEFD07
:1065A000D4F854370133C9E6924B90495A8995483B
:1065B000FCF7E4FDD4F854370133BFE68D4B8B492B
:1065C0001A7E9148FCF7DAFDD4F854370133B5E66A
:1065D000884B86491A898D48FCF7D0FDD4F854378A
:1065E0000133ABE6834B8149DA7D8948FCF7C6FD70
:1065F000D4F854370133A1E67E4B7C49DA788548DC
:10660000FCF7BCFDD4F85437013397E6824B774949
:106610005A788248FCF7B2FDD4F8543701338DE63E
:106620007D4B72491A787E48FCF7A8FDD4F85437A0
:10663000013383E67B4B6D491B687B485A8DFCF721
:106640009DFDD4F85437013378E6764B67491B68D3
:1066500076481A8DFCF792FDD4F8543701336DE675
:10666000704B62491B6872481A8FFCF787FDD4F89B
:106670005437013362E66B4B5C491B686D48DA8E18
:10668000FCF77CFDD4F85437013357E6654B6A4973
:106690001D686A486B8AAA892D8B0095FCF76EFDF0
:1066A000D4F85437013349E65E4B50491B686448BF
:1066B00093F84720FCF762FDD4F8543701333DE6E8
:1066C000584B4A491B685F489A8EFCF757FDD4F82F
:1066D0005437013332E6534B44491B685A485A8EAB
:1066E000FCF74CFDD4F85437013327E64D4B3F49B6
:1066F0001B68564893F83020FCF740FDD4F8543717
:1067000001331BE6474B39491B68514893F82C204D
:10671000FCF734FDD4F8543701330FE6414B3349CD
:106720001B684C4893F84620FCF728FDD4F85437F2
:10673000013303E63B4B2D491B68474893F827205C
:10674000FCF71CFDD4F854370133F7E5354B2749E6
:106750001B684248DA88FCF711FDD4F8543701333E
:10676000ECE5304B21491B683D489A88FCF706FD53
:10677000D4F854370133E1E52A4B1C491B683948EA
:106780001A88FCF7FBFCD4F854370133D6E5254BC7
:1067900016491B683448B3F84C20FCF7EFFCD4F8DA
:1067A00054370133CAE51F4B10491B682F485A88DC
:1067B000FCF7E4FCD4F854370133BFE5194B0B491F
:1067C0001B682B4893F82620FCF7D8FCD4F85437E4
:1067D0000133B3E5134B05491B68264893F8202085
:1067E000FCF7CCFCD4F854370133A7E5A5ED040839
:1067F0002CB10408CC9C002034AE040818B1040865
:1068000008B10408F4B00408E0B00408D0B00408EB
:10681000BCB00408A8B004083472002098B0040882
:106820009CB00408E456002084B0040874B0040846
:1068300068B0040858B00408F0AE040844B0040876
:106840002CB0040818B0040800B00408ECAF040829
:10685000D8AF0408C8AF0408B8AF0408A4AF040850
:1068600094AF040884AF040870AF04085CAF040858
:1068700048AF040840AF0408AD4BAE491D68AE48B0
:10688000EB7EAA7E2D7F0095FCF778FCD4F8543778
:10689000013353E5A64BA7491D68A8486B7D2A7DA7
:1068A000AD7D0095FCF76AFCD4F85437013345E51B
:1068B0009F4BA0491D68A248EB7BAA7B2D7C0095CD
:1068C000FCF75CFCD4F85437013337E5984B994911
:1068D0001D689C486B7A2A7AAD7A0095FCF74EFCCD
:1068E000D4F85437013329E5974B9249974807EB81
:1068F000C70703EB4707FD7ABB7A7A7A0095FCF766
:106900003DFCD4F85437013318E58F4B8949904842
:1069100007EBC70703EB47073D7AFB79BA79009588
:10692000FCF72CFCD4F85437013307E5864B81493A
:10693000884807EBC70703EB47077D793B79FA786F
:106940000095FCF71BFCD4F854370133F6E47E4B7A
:106950008149824807EBC70703EB4707FA89FCF731
:106960000DFCD4F854370133E8E4774B7A497C487E
:1069700007EBC70703EB47073A7BFCF7FFFBD4F8AD
:1069800054370133DAE4704B7349764807EBC70795
:1069900003EB47077A78FCF7F1FBD4F8543701335F
:1069A000CCE4694B6C49704807EBC70713F8172014
:1069B000FCF7E4FBD4F854370133BFE494F85225D4
:1069C00065496A48FCF7DAFBD4F854370133B5E47B
:1069D000674B61499A786748FCF7D0FBD4F8543785
:1069E0000133ABE4644B5C491A686448FCF7C6FBAE
:1069F000D4F854370133A1E4614B9B79012B00F0AB
:106A0000218111239AE4B4F85C275E495E48FCF7C3
:106A1000B5FBD4F85437013390E45C4B4E491A88E7
:106A20005B48FCF7ABFBD4F85437013386E4B4F988
:106A3000482749495748FCF7A1FBD4F8543701339C
:106A40007CE4B4F9462744495348FCF797FBD4F853
:106A50005437013372E4514A51495248FCF78EFBD6
:106A6000D4F85437013369E403A8F6F715FA4E4B0E
:106A700003A9B3F9002006A80023F6F731FA06AA05
:106A800047494A48FCF77AFBD4F85437013355E4B8
:106A9000474B484A48494948FCF770FBD4F85437FB
:106AA00001334BE4464A474B47494848CDE9003259
:106AB000474B484AFCF762FBD4F8543701333DE4B6
:106AC000454A37494548FCF759FBD4F85437013358
:106AD00034E4B3B2AAB242494248FCF74FFBD4F8BF
:106AE000543701332AE44FF07E523F493F48FCF7C8
:106AF00045FBD4F85437013320E43D4B16495A8AFC
:106B00003C48FCF73BFBD4F85437013316E4384BD0
:106B100011491A8A3848FCF731FBD4F8543701334D
:106B20000CE4D4F80837DB0400F18180102305E47D
:106B3000E4560020F0AE040834AF04082CAF04087B
:106B400020AF040818AF04081E6D002010AF040821
:106B500008AF0408FCAE0408A5ED0408E0AE040884
:106B6000D4AE0408C8AE0408C0AE0408ACAE040835
:106B7000CC9C00209CAE0408EC9C002090AE040845
:106B800020520020DCF2040878AE0408C054002033
:106B900000AE0408F4AD0408E8AD0408D872002083
:106BA00083A20408DCAD04081C710020C8AD0408F1
:106BB000EBA20408F4A204087EEE0408B8AD0408B1
:106BC0009CA20408E1A2040894AD0408A4AD040842
:106BD00000A30408A6A2040878AD040884AD040844
:106BE00034AE04083CAE040820AE040828AE040805
:106BF00088A5002014AE040808AE04081A4B1B49EF
:106C00009A8A1B48FCF7BAFAD4F854370133FFF7D5
:106C100095BB184818498378427800780090174847
:106C2000FCF7ACFAD4F854370133FFF787BB144BA9
:106C30000E491A781348FCF7A1FAD4F854370133F7
:106C4000FFF77CBB104A1149B2F900301048B2F985
:106C50000220FCF793FAD4F854370133FFF76EBBE8
:106C60000120FFF75FBB00BF40520020DCF20408A8
:106C700048AE0408205200205CAE040868AE040848
:106C8000416B002050AE0408466B002034AE04086F
:106C900080AE04082DE9F04F604D85B0D5F8584717
:106CA0000093904600290CBF04230623621C0F9F0B
:106CB00001936ED00E9BA34247DDDFF874A157B15C
:106CC000109BDA1B04FB02F20123B95CD5F80827FC
:106CD0008B40134231D0009BD5F854B7A3EB080387
:106CE00004FB03F408EB0406BBF1000F3AD158F89B
:106CF00004002DF077FA00F10509484615F02EFC46
:106D0000002836D1DAF8000095F87217A0EB0900D8
:106D1000CAF80000002936D1012385F87237BBF18B
:106D2000000F2AD158F8040015F064FC96F90410FD
:106D30004B1C02D03A48FCF70FFAD5F858470E9B87
